:102000000FE023000EFF24000E01880000000000F6
:10201000000020000000E00002003200000120006B
:1020200020028800140007008A0007000000E0007A
:1020300003003A00E0A7230021002000020037003F
:102040000000200001002000810F7000010032001C
:102050000F000700000020000000E0000200320036
:102060000000020000000000B65B0200000000005B
:102070000040DA000000FE0060A027000000E00041
:1020800002003200102020009001880000000600AD
:10209000A1028800800478000000EB001F003700D8
:1020A000E284440054A0B4009905BA00E2844400DC
:1020B00054A0B4009906BA00E284440054A0B400CD
:1020C0000006EB00476FDE00FD07B200AE0188009E
:1020D000636CE10003003A000AD801000000EB0045
:1020E0000E003700606CE10008003A00004DEB0084
:1020F0000A05E800020039003420EC000AF0A000D4
:102100008B05E900F9FF3E00040037006168E1003B
:10211000010032000086EB000B00070019C7BA006F
:102120000E04E0001905BA0003003A000A00E000BE
:10213000DBFF3A0000000600FE07B200AE02880096
:102140008A047800F5FF37000CD0A300E20F4D00A1
:102150001C003B0089027800354DBA000A05E800F2
:10216000020039003420EC000AF0A0008B05E900E1
:102170000F003200254DBA000A05E80002003900C0
:102180003420EC000AF0A0008B05E90008003200C2
:102190000C00E0000600320015CDBA000A05E80088
:1021A000020039003420EC000AF0A0008B05E900A1
:1021B0008984E80054A0B4000B00E000E2FF3A007C
:1021C000000006009902BA00055D78008B05E90061
:1021D000F7FF3200C82ADE00055D78008B05E900B4
:1021E000F3FF32000C00E000F1FF320019DDBA000D
:1021F000EEFF3700CE9F040001000000646704007A
:102200000000000088A0040001000000BAA0040043
:1022100001000000D8A0040001000000B6DB0400AB
:10222000010000007CDC04000100000056DB04001B
:1022300001000000286304000000000060A004000A
:1022400001000000826704000000000074DB04004D
:102250000100000000000500839F68000100E0000D
:1022600002003D0060001000E08018000300E00064
:1022700002003D0060011100E08119000500070027
:102280004F00E00002003B0060001000E0801800FA
:10229000000006006022B800060220000000D00006
:1022A0008180D2000482D2008582D2000000A0008A
:1022B0000202520083825A000300310002024200EF
:1022C00083824A000000A1000603E900F3FF3A0000
:1022D000000006000A00FA00300798004107980045
:1022E00000012000000F78000000EB0010079800AC
:1022F000160037001E007800C780DE001E00900028
:102300003E01900000004100104078000080FB007A
:1023100080806800F00F2000008060002007980097
:102320001E007800C800DD002E0090000001400073
:10233000204E2F000000410010007800008F680040
:102340001E0090000000E800100798009E0090001A
:102350004E009000808F5000E6FF35001E00780090
:10236000000040000080FA00000006000800FA00AB
:102370000040EB0020479800D0C0B30030479800E1
:102380000E80E80021002000D2FF0700000F780037
:102390000040EB0020479800F0C0B30030479800A1
:1023A0000E80E80021002000CAFF0700000F78001F
:1023B00070C0B3002047980010C1B30030479800A8
:1023C0000E80E80021002000C2FF0700000F780007
:1023D0000080FA00000006000000FA00002E230032
:1023E0000107200000280200020000000080FA001F
:1023F000000006000200FA00004F78009E80FB00FB
:10240000800320008088B90080007800002E23001F
:10241000008040000080FA00000006000000FA0082
:10242000004C23000080FA00000006000000FA00C3
:10243000709380000080FA00000006000200FA009D
:10244000004F78001E4078000004E00002003A00CF
:102450002C8EA9000100370019CEA9000080FA00D7
:10246000000006000200FA00004F78001E407800CD
:102470000004E00002003A002C8EA80001003700A2
:1024800019CEA8000080FA00000006000200FA0041
:10249000881F7800000F78000040EB00383C0200F5
:1024A000020000009E007800804878001E04E800CA
:1024B0000040EB00383C020002000000004C7800B5
:1024C0001E00E800104078000080FB00C800DD001E
:1024D0001E007800104078000080FB000080400063
:1024E0004F0478000080FA00000006000200FA00A5
:1024F000881F7800000F78000040EB00383C020095
:10250000020000009E007800804878001E04E80069
:102510000040EB00383C020002000000004C780054
:102520001E007800104078000080FB00C800DD002D
:102530001E00E800104078000080FB000080400092
:102540004F0478000080FA00000006000600FA0040
:10255000204798002107980013E1A9001221A90043
:1025600012C1A90091088000000320000100700042
:10257000900888000A21EF00AE009000B0AA2A005F
:102580000008B8004208DE00700888000108A900B1
:102590002E409000A9FF070040712000AC3C0200D3
:1025A00002000000C0362F00AC3C02000200000018
:1025B00013E1A8000040EB00383C020002000000DC
:1025C000004F78000040EB00383C020002000000A1
:1025D000004F7800040037000040EB00383C020058
:1025E00002000000004F7800014080000010200031
:1025F000008060000000E00003003A001E40780008
:10260000E14F4000F4FF3A002E40900095FF070094
:102610001E407800E14F400003003A0010C0B300B4
:1026200010479800020037000040EB001047980068
:102630001E4090000080FA00000006000600FA002C
:10264000004F780011079800220798001E4078007C
:102650007AFF07000000EB00AC3C02000200000023
:102660000000EB00AC3C0200020000000000EB00A8
:10267000AC3C0200020000000000EB00AC3C020099
:10268000020000001E40780076FF07001E40780020
:102690006AFF07001E009000AC3C02000200000030
:1026A0002E009000AC3C0200020000001E407800AA
:1026B0006CFF07001E80FB00810320008181B900B0
:1026C000012E230081004100910078008100E80084
:1026D000820320008281B900002E23000000410007
:1026E000010878000080FA00000006000000FA00EF
:1026F000E2852700517120000040EB00CFFF07006A
:10270000E28527005171200010C0B300CBFF070005
:10271000813821000040EB008CFF07008138210048
:1027200010C0B30089FF07000080FA000000060017
:102730000000FA0062492500317120000040EB00E2
:10274000BEFF0700624925003171200010C0B300B0
:10275000BAFF0700011920000040EB007BFF0700D3
:102760000119200010C0B30078FF07000080FA00B4
:10277000000006000000FA00029C2C0011712000ED
:102780000040EB00ADFF0700029C2C0011712000FF
:1027900010C0B300A9FF0700011920000040EB00A2
:1027A0006AFF07000119200010C0B30067FF07008F
:1027B0000080FA00000006002400FA00005F980084
:1027C000115F9800520F9800630F9800645F9800A3
:1027D00005179800161798000E5890008080FB008F
:1027E000800320008088B90080007800602E2300DC
:1027F00000804000DE089000010878001E5890001C
:102800000004E000EB0032000E5890000080FB0056
:10281000810320008181B900820078000181E800F5
:10282000012E230081004100910078008100E80022
:10283000820320008281B900202E23000000410085
:10284000010878000040EB00004F780020C0B30082
:1028500010479800D40037001E1090008000EB0055
:10286000010878000E589000F4FE07005E08900002
:10287000AC3C0200020000006E089000AC3C02007C
:10288000020000008E109000110798000040EB003D
:1028900040479800A30037001E01900032079800BF
:1028A000014C23004E4090000081FB000E58900028
:1028B0000080FB004300DD0000004100EA00B90099
:1028C0000080400040079800CE009000510798001B
:1028D0005E009000EDFE0700100F98005E00900073
:1028E0000000E800500798005E0090000000E8003B
:1028F000500798005E009000E4FE0700200F98004B
:102900005E0090000000E800500798005E00900014
:102910000000E800500798005E009000DBFE070012
:10292000300F98005E0090000000E800500798000B
:102930005E0090000000E800500798005E009000E4
:10294000EAFE0700600798005E0090000000E800C3
:10295000500798005E0090000000E80050079800C3
:10296000610020004E0090005AFE0700700798009A
:102970007E0090004800DE00804078005E009000FD
:10298000014878005E0090000000E80050079800C1
:102990007E009000804078005E0090000148780042
:1029A0005E0090000000E800500798000E5890006C
:1029B0008080FB00800320008088B900E800400090
:1029C000002E2300808040004E4090000080FB00DD
:1029D000E600B90000804000000F9800FE00900063
:1029E0006E009000808F500023003A009E089000F7
:1029F0003E009000010878003E0090000080E80052
:102A000030079800AE0890003E0090000108780062
:102A10003E0090000080E80030079800BE0890005B
:102A20003E009000010878003E0090000080E80021
:102A3000300798001E109000900078004E409000E3
:102A40000080FB00120020000010DD0081007000FB
:102A50001E1090000108780010C0B300004F7800ED
:102A60000E089000100078008000E8000E0890002A
:102A700001087800220037003E0090008000EB0043
:102A8000010878003E0090000080E80030079800C0
:102A90003E0090008000EB00010878003E009000AE
:102AA0000080E800300798003E0090008000EB00B6
:102AB000010878003E0090000080E8003007980090
:102AC0006E009000E10F400008003A000E089000F0
:102AD000100090008000E8000E089000110098009F
:102AE00010C0B300004F7800050037000E089000BA
:102AF000200090008000E8000E089000210098005F
:102B00006E5890000080FB00000040009E00900086
:102B100000804000100798004E4090000040E80000
:102B200040479800CE4090001E58900080CF500043
:102B300059FF39000E5890004AFE07001E407800E9
:102B40000004E00018003A001E4090000040E90038
:102B5000104798001E4090000004E00003003A0077
:102B600010C0B300004F78000F0037000E589000DF
:102B70000080FB00810320008181B9008200780081
:102B800064814000012E2300810041009100780003
:102B90008100E800820320008281B900402E2300DA
:102BA00000004100010878001E4078000004E000A9
:102BB00029FF32000080FA00000006001200FA002F
:102BC000404F9800514F980072079800030F9800EB
:102BD0006AD2BF000E037800FE0290000042780027
:102BE000237C200042002000DE4890004E489000E8
:102BF000F1FE07007E009000E60040006AD2BF00B0
:102C00000E81E8000203780081027800004278001B
:102C100043A9290062002000DE4890004E48900041
:102C2000E5FE07007E009000EC0040006AD2BF0085
:102C300064014700020378008102780000427800B6
:102C400023E5250082002000DE4890004E489000D9
:102C5000D9FE07007E009000F20040006AD2BF005B
:102C60006601470002037800810278000042780084
:102C700043302C00A2002000DE4890004E48900017
:102C8000CDFE07009E0078001E009000808060004E
:102C90002E009000808060003E00900080806000E8
:102CA0000E089000010878006AD2BF00F24F500071
:102CB00020003A007E009000F80040006AD2BF0079
:102CC0006801470002037800810278000042780022
:102CD00003562D0092002000DE4890004E489000E0
:102CE000B5FE07007E009000FE0040006AD2BF00E3
:102CF0006A014700020378008102780000427800F0
:102D000063832400B2002000DE4890004E4890000B
:102D1000A9FE07000E089000900078004E00900079
:102D2000808060005E009000808060000E0890004F
:102D3000010878000080FA00000006000800FA0090
:102D40004047980051479800624798005E409000C5
:102D50000004E000990032004E409000B7FD0700EB
:102D600010002000AC3C020002000000E0D623006E
:102D7000AC3C020002000000DE40900011479800C9
:102D80003B0037006E4090000004E0002800320055
:102D90004E4090000004E0000A003A001E409000FF
:102DA0000080FB000000E900004078004300DD00E7
:102DB000204798001E4090004300DD0030479800F7
:102DC0000C0037001E4090000080FB0067004000B0
:102DD000004078004300DD00204798001E4090002E
:102DE0000080FB0068004000004078004300DD00E8
:102DF00030479800AE409000014F78000700370040
:102E00001E80FB00013B2300008040001040780042
:102E1000383C0200020000001E4FE8003E409000D7
:102E20009E40780080CF5000F5FF39000D0037003C
:102E30000040EB00004F7800070037001E80FB00C9
:102E4000014B23000080400010407800383C020015
:102E5000020000001E4FE8001E407800E74F5000BF
:102E6000F6FF36001E4090000040E9001047980031
:102E70001E4090000004E000C2FF3A004E40900067
:102E800078FD07006AD2BF00F24F500049003A00B7
:102E90004E40900069FD070040022000AC3C02005B
:102EA00002000000E0192B00AC3C02000200000010
:102EB000DE409000114798003B0037006E409000C4
:102EC0000004E000280032004E4090000004E000C2
:102ED0000A003A001E4090000080FB000000E9005C
:102EE000004078004300DD00204798001E4090001D
:102EF0004300DD00304798000C0037001E40900072
:102F00000080FB0067004000004078004300DD00C7
:102F1000204798001E4090000080FB0068004000A1
:102F2000004078004300DD0030479800AE4090003C
:102F3000014F7800070037001E80FB00014323008B
:102F40000080400010407800383C02000200000081
:102F50001E4FE8003E4090009E40780080CF500019
:102F6000F5FF39000D0037000040EB00004F7800FE
:102F7000070037001E80FB00814B230000804000CB
:102F800010407800383C0200020000001E4FE800AC
:102F90001E407800E74F5000F6FF36001E409000BC
:102FA0000040E900104798001E4090000004E00037
:102FB000C2FF3A004E4090002AFD07000080FA0050
:102FC000000006000E00FA00300798004107980044
:102FD00052079800630798000000EB001007980064
:102FE0000000EB00200798006BD2BF000004E00057
:102FF00018003200810C20000040EB0053FD070058
:103000004E019000BE0090000040EB008BFD0700D9
:1030100001FA20000040EB004CFD0700004F780053
:103020006CD2BF000004E000030032004106200023
:1030300010C0B30045FD07006BD2BF008E80E800D2
:10304000810178005E019000804078000040EB0034
:10305000DAFE07006CD2BF000004E0001600320068
:10306000810C200010C0B30038FD07004E01900015
:10307000BE00900010C0B30070FD070001FA2000F0
:1030800010C0B30031FD07006AD2BF000080FB0012
:103090004400DD00DE009000808040006CD2BF0064
:1030A00064014700820178000101780080407800C7
:1030B00010C0B300C1FE07002E009000C800DD0064
:1030C0001E009000808040006E0090000108780093
:1030D0000080FA00000006000A00FA00400798008D
:1030E0000000EB00000F78000000EB0010079800D4
:1030F0000000EB00200798000000EB00300798006C
:10310000810C20000040EB0010FD0700810C200026
:1031100010C0B3000DFD0700023A2D00015620003B
:103120000040EB0045FD0700023A2D00015620004B
:1031300010C0B30041FD070001FA20000040EB0081
:1031400002FD070001FA200010C0B300FFFC0700D9
:103150004E0090000080E800800078006BD2BF0035
:103160000E0378008102780034C0B300C3FC2E0047
:10317000C2002000804078000040EB008EFD070078
:103180004E0090002006B000800078006BD2BF0097
:103190000E81E800020378008102780034C0B30099
:1031A000A3292700E2002000804078000040EB00C7
:1031B00081FD07004E0090000080E8000103200020
:1031C000808040006CD2BF00640147000203780099
:1031D0008102780034C0B300C3FC2E00C20020007E
:1031E0008040780010C0B30073FD07004E009000CF
:1031F0002006B00001032000808040006CD2BF0098
:1032000066014700020378008102780034C0B300F1
:10321000A3292700E20020008040780010C0B300FE
:1032200065FD0700AE0090003E0090000080600049
:10323000C800DD001E0178001E0090000000610043
:10324000810070004E009000010878000080FA00B4
:10325000000006000A00FA00400798000000EB009A
:10326000000F78000000EB00100798000000EB0052
:10327000200798000000EB0030079800810C200028
:103280000040EB00B1FC0700810C200010C0B3002F
:10329000AEFC0700023A2D00015620000040EB0072
:1032A000E6FC0700023A2D000156200010C0B300D2
:1032B000E2FC070001FA20000040EB00A3FC07003D
:1032C00001FA200010C0B300A0FC07004E009000DF
:1032D0000080E800800078006BD2BF000E03780009
:1032E0008102780034C0B300E34F2600D2002000F2
:1032F000804078000040EB002FFD07004E0090005A
:103300002006B000800078006BD2BF000E81E8007C
:10331000020378008102780034C0B300839A2F0042
:10332000F2002000804078000040EB0022FD070002
:103330004E0090000080E8000103200080804000E3
:103340006CD2BF006401470002037800810278005C
:1033500034C0B300E34F2600D20020008040780044
:1033600010C0B30014FD07004E0090002006B0000E
:1033700001032000808040006CD2BF00660147003E
:10338000020378008102780034C0B300839A2F00D2
:10339000F20020008040780010C0B30006FD070056
:1033A000AE0090003E00900000806000C800DD008C
:1033B0001E0178001E009000000061008100700076
:1033C0004E009000010878000080FA00000006001E
:1033D0000E00FA0040079800510798006207980015
:1033E000810C20000040EB0058FC0700810C2000FD
:1033F00010C0B30055FC07005E019000CE009000A5
:103400000040EB008DFC07005E019000CE009000B4
:1034100010C0B30089FC070001FA20000040EB0057
:103420004AFC070001FA200010C0B30047FC070067
:103430000000EB00000F78000000EB001007980080
:103440000000EB00200798000000EB003007980018
:103450006E0090000080E800800078006BD2BF0012
:103460000E0378008102780034C0B30023D72E0009
:1034700002012000804078000040EB00CEFC0700F5
:103480006E0090002006B000800078006BD2BF0074
:103490000E81E800020378008102780034C0B30096
:1034A0004302270022012000804078000040EB000A
:1034B000C1FC07006E0090000080E80001032000BE
:1034C000808040006CD2BF00640147000203780096
:1034D0008102780034C0B30023D72E0002012000FF
:1034E0008040780010C0B300B3FC07006E0090006D
:1034F0002006B00001032000808040006CD2BF0095
:1035000066014700020378008102780034C0B300EE
:1035100043022700220120008040780010C0B30041
:10352000A5FC0700AE0090003E0090000080600007
:10353000C800DD001E0178001E0090000000610040
:10354000810070006E009000010878000080FA0091
:10355000000006000A00FA00400798000000EB0097
:10356000000F78000000EB00100798000000EB004F
:10357000200798000000EB00300798004E009000F4
:1035800064004000800078006BD2BF000E0378001A
:103590008102780034C0B300A3B0220022002000D2
:1035A000804078000040EB0083FC07004E00900054
:1035B0006400400001032000808040006CD2BF0006
:1035C00064014700020378008102780034C0B30030
:1035D000A3B02200220020008040780010C0B30079
:1035E00075FC07004E0090004006B0008000780097
:1035F0006BD2BF000E81E8000203780081027800E0
:1036000034C0B30083CC22006202200080407800E6
:103610000040EB0068FC07004E0090004006B00040
:1036200001032000808040006CD2BF00660147008B
:10363000020378008102780034C0B30083CC2200FA
:10364000620220008040780010C0B3005AFC0700DE
:103650002E009000C800DD001E0078008100700080
:103660004E009000010878003E009000C800DD0088
:103670001E009000810070004E0090001100980024
:103680000080FA00000006001400FA00000F980005
:10369000110F98000040EB00004F78001500370034
:1036A0000040EB0065FB070000362000AC3C020048
:1036B00002000000C0462F00AC3C020002000000E7
:1036C0000040EB0067FB070010C0B3005BFB070086
:1036D00000362000AC3C020002000000C0462F0073
:1036E000AC3C02000200000010C0B3005DFB07000C
:1036F0001E4FE8001E407800E94F5000E8FF3600FA
:103700000040EB00104798007B0037000040EB00C2
:103710002047980000352300200798001E409000A5
:10372000E14F500003003A00003523000003B000D1
:10373000200798001E40900040FB0700200020005A
:10374000AC3C020002000000A0B02200AC3C020031
:10375000020000000040EB00304798004E003700A8
:10376000AE00900031079800014C23003E409000CD
:103770000080FB00EA00B90000804000500798007C
:103780000040EB00004F9800100037005E009000F2
:103790003EFB0700BE009000800878003E009000CD
:1037A0000080E800300798005E0090000000E8000C
:1037B000500798005E0090000000E8005007980055
:1037C0000E4890000040E800004F98000E4890001E
:1037D000E24F5000EDFF36005E00900043FB070013
:1037E000600798005E0090000000E8005007980015
:1037F0005E0090000000E800500798000E4890001E
:103800000080FB000000400080007800024C230094
:103810003E4090000080FB00EA00B900000041003B
:10382000ACFA0700700798007E0090004800DE00A8
:10383000804078005E009000014878005E009000B3
:103840000000E800500798007E009000804078005B
:103850005E009000014878005E0090000000E800E3
:1038600050079800FE0090006E009000808F50007E
:1038700003003A003E4090000040E80020479800D6
:103880002E00900066004000200798003E40900007
:103890000040E800304798003E409000E74F50005D
:1038A000AFFF36001E409000EEFA07001E40900069
:1038B0000004E00007003A00AE409000B22621006C
:1038C000014978000E0890002E41900002487800CF
:1038D000060037002E419000C12621008248780062
:1038E0001E089000AE409000014878001E409000F5
:1038F0000040E800104798001E409000E14F500043
:1039000082FF36006BD2BF000080FB001100200058
:103910000008DD008000E9006CD2BF000080FB00E1
:10392000120020000010DD000000E9004800DD006A
:10393000010070007093880010C0B30002000700FF
:103940000080FA00000006000200FA00004F780034
:103950006BD2BF001E417800804078000040EB0031
:10396000F6FC07006CD2BF001E4178008040780052
:1039700010C0B300F1FC07000080FA000000060050
:103980001400FA00889FBE008A9FBE008C9FBE0074
:103990004047980032079800430798004E40900037
:1039A0004300DD00004F78009E40780011479800EA
:1039B0001E4090000080FB00013B2300008040007F
:1039C000C1CFB300014878001E4090000040E800DD
:1039D000104798001E4090000080FB00013B230030
:1039E000008040008040EB00014878001E409000BD
:1039F0000040E800104798001E4090000080FB0047
:103A0000013B2300008040008040EB00014878002B
:103A10001E4090000040E800104798001E409000B3
:103A20000080FB00013B2300008040008040EB0051
:103A3000014878001E4090000040E80010479800C0
:103A40001E4090000081FB003E0090008040780006
:103A5000003B230002004000014878001E40900017
:103A60000040E800104798001E4090000080FB00D6
:103A7000500798003E009000CE00900002F0200019
:103A8000030020000002780064079800010278001B
:103A90007407980082007800030078006E0190009F
:103AA000810061007E0290000000620080037800C7
:103AB000010378000600BE004809DD004802DE0070
:103AC00004027100C88ADE0084407800003B2300B5
:103AD0005E02900004004000014878001E40900003
:103AE0000040E800104798009E80FB00003B230048
:103AF0000080400061002000F6F9070010079800E0
:103B00001E4090000080FB009E009000C808DE0070
:103B100081407800023B230000004100014878000A
:103B20001E4090000040E800104798001E409000A2
:103B30000080FB009E00900081407800023B230043
:103B400000004100014878001E4090000040E8005D
:103B5000104798004E4090004300DD00004F780071
:103B60009E407800114798001E4090000082FB00A4
:103B70003E019000CE01900000002F0001002000C7
:103B800082027800030178008001780081007800CB
:103B90000380620081006100110F9800000F9800FF
:103BA0000E0890009E0890004809DD004806DE00DF
:103BB0000C067100C88EDE000C407800F040B300A7
:103BC0008040780000432300040040000148780052
:103BD0001E4090000040E800104798001E409000F2
:103BE0000082FB003E019000CE019000000020000A
:103BF0003100200082027800030178008001780003
:103C000081007800038062008100610081057800F6
:103C1000000578000A00BE00408CDE00CF8CDE007C
:103C200088407800004323000400400001487800E9
:103C30001E4090000040E800104798001E40900091
:103C40000080FB0001432300008040008040EB0027
:103C5000014878001E4090000040E800104798009E
:103C60001E4090000080FB000143230000804000C4
:103C70008040EB00014878001E4090000040E800C2
:103C8000104798001E4090000080FB000143230075
:103C9000008040008040EB00014878001E4090000A
:103CA0000040E800104798001E4090000080FB0094
:103CB00001432300008040008040EB000148780071
:103CC0001E4090000040E800104798009E80FB00D6
:103CD0000043230000804000610020007DF90700C0
:103CE000100798001E4090000080FB009E0090008E
:103CF000C808DE0081407800024323000000410034
:103D0000014878001E4090000040E80010479800ED
:103D10001E4090000080FB009E00900081407800D3
:103D20000243230000004100014878001E4090003B
:103D30000040E800104798004F06BE004F05BE0047
:103D40004F04BE000080FA00000006000600FA00E2
:103D5000404798004E419000A126210082487800FB
:103D600082F907000040EB00004F78001E80FB0046
:103D7000014B230000804000C1CFB3000148780010
:103D80001E4FE8001E80FB00014B23000080400016
:103D90008040EB00014878001E4FE8001E80FB00C9
:103DA000014B2300008040008040EB000148780078
:103DB0001E4FE8001E80FB00014B230000804000E6
:103DC0008040EB00014878001E4FE8001E80FB0099
:103DD000014B2300008040008040EB000148780048
:103DE0001E4FE8001E80FB00014B230000804000B6
:103DF0008040EB00014878001E4FE8006100200081
:103E0000004B230033F90700100798001E80FB00C9
:103E10009E009000C808DE0081407800024B23001D
:103E200000004100014878001E4FE8001E80FB00A2
:103E30009E00900081407800024B2300000041006A
:103E4000014878001E4FE8000040EB00004F78006A
:103E50001E80FB00814B230000804000F1C0B300B6
:103E6000014878001E4FE8001E80FB00814B2300B4
:103E7000008040008040EB00014878001E4FE800C1
:103E80001E80FB00814B2300008040008040EB003F
:103E9000014878001E4FE8001E80FB00814B230084
:103EA000008040008040EB00014878001E4FE80091
:103EB0001E80FB00814B2300008040008040EB000F
:103EC000014878001E4FE8001E80FB00814B230054
:103ED000008040008040EB00014878001E4FE80061
:103EE00061002000804B2300FAF8070010079800BB
:103EF0001E80FB009E009000C808DE008140780014
:103F0000824B230000004100014878001E4FE8006A
:103F10001E80FB009E00900081407800824B2300B1
:103F200000004100014878001E4FE8000040EB000F
:103F3000004F7800040037006011B8001E40780080
:103F40008FFE07001E4FE8001E407800EF4F500024
:0C3F5000F9FF36000080FA0000000600B7
:104000003600F800809FBE00829FBE00849FBE00E5
:10401000869FBE000000FA00CC28020000000000CD
:104020000080FA004F03BE004F02BE004F01BE00E9
:0C4030004F00BE003600F9000040060002
:104040000000FA002248A9000248A9000080FA00F6
:044050000040060026
:104080000000FA002268A9000268A9000080FA0076
:0440900000400600E6
:1040C0003600F800809FBE00829FBE00849FBE0025
:1040D000869FBE000000FA007A3A0200020000004B
:1040E0000080FA004F03BE004F02BE004F01BE0029
:0C40F0004F00BE003600F9000040060042
:104100003600F800809FBE00829FBE00849FBE00E4
:10411000869FBE000000FA00763A0200020000000E
:104120000080FA004F03BE004F02BE004F01BE00E8
:0C4130004F00BE003600F9000040060001
:104140003600F800809FBE00829FBE00849FBE00A4
:10415000869FBE000000FA00723A020002000000D2
:104160000080FA004F03BE004F02BE004F01BE00A8
:0C4170004F00BE003600F90000400600C1
:104180000000FA000088A9000080FA000040060044
:1041C0000000FA0001C8A9000080FA0000400600C3
:104200003600F800809FBE00829FBE00849FBE00E3
:10421000869FBE000200FA002028A900210A800023
:10422000010F7800E08480000000E00017003200F9
:10423000E08480000000E900E0848800E0848000E1
:10424000E10F500009003600E0848000E50F5000C7
:1042500006003E00E08480000080E900C1082100E3
:1042600000004000008040001E087800E0848000CC
:104270000000E000030032000028A9002028A80068
:1042800002003700B2620200010000000080FA0064
:104290004F03BE004F02BE004F01BE004F00BE00E4
:0842A0003600F90000400600A1
:104300003600F800809FBE00829FBE00849FBE00E2
:10431000869FBE000200FA0020A8A900610A800062
:10432000010F7800F08480000000E00017003200E8
:10433000F08480000000E900F0848800F0848000B0
:10434000E10F500009003600F0848000E50F5000B6
:1043500006003E00F08480000080E9004109210051
:1043600000004000008040001E087800F0848000BB
:104370000000E0000300320000A8A90020A8A80067
:1043800002003700B2620200010000000080FA0063
:104390004F03BE004F02BE004F01BE004F00BE00E3
:0843A0003600F90000400600A0
:10440000809FBE000200FA00101180006100600071
:104410000000E0002900320030118000004F7800D9
:1044200030928000EE0F500003003E00309280007A
:104430000000E800010037000000EB00419280001E
:10444000810F500004003A0080C981000000E8009C
:1044500080C98900190037004AD2BF000004E0007B
:10446000070032001E4078000004E00004003A001B
:10447000D0C981000000E800D0C989000F003700D2
:1044800090C981000000E80090C989003092800046
:1044900001922300008040001E4878003092800086
:1044A000EE0F500003003E00309280000000E80054
:1044B000010037000000EB00309288000168A9007D
:1044C00010118000610060000000E0000100320077
:1044D0000168A8000080FA004F00BE0000400600FE
:10458000809FBE000200FA000188A9000F003700DA
:1045900070928000C193230000804000104F78008B
:1045A00071928000E00F2000808F500003003E00D9
:1045B000709280000000E800010037000000EB006E
:1045C000709288001E80FB0020118800111180006D
:1045D00000202000008060000000E00004003A009D
:1045E0006192800070928000808F5000E8FF3A0056
:1045F0002188A8000080FA004F00BE00004006009D
:10468000801F78000000FA0010118000A0C9890086
:10469000B0C981000000E800B0C989001011800095
:1046A000620060000000E000010032002222A90048
:1046B00010118000640060000000E0000100320082
:1046C0002242A90010118000680060000000E00094
:1046D000010032002262A90021E2A90021E2A80023
:1046E0000828A9000080FA004F007800004006006A
:104780003600F800809FBE00829FBE00849FBE005E
:10479000869FBE000200FA00408E80000000E0000C
:1047A00003003200408E80000000E900408E880047
:1047B000508E80000000E00003003200508E800028
:1047C0000000E900508E8800508E80000000E0005C
:1047D0001C003A00D0002000508E880010C0B300AA
:1047E000CCF1B7000040EB00004F7800120037001A
:1047F0001E80FB0080004000C0EF220000804000CF
:10480000100078000000E0000A0032001E80FB006B
:1048100000014000C1EF22008100410091007800BA
:104820008100E90000014000C0EF220000004100CB
:10483000010878001E4FE8001E407800ED4F500040
:10484000EBFF3600CED1BF000040E800CEF1B7004C
:10485000CED1BF00E34F500001003600CE71EF0013
:10486000CED1BF000004E00018003A00C08D8000E7
:104870000000E800C08D8800A08D8000B18D800010
:1048800061004000E0804800A08D8800B18D880064
:1048900007003700D08D80000000E800D08D880030
:1048A000C18D800000102F0000804000C08D880066
:1048B000C18D8000F0EF2000808F5000F5FF3E009A
:1048C0005A5D0200000000000E003700CED1BF008C
:1048D000E14F500003003A00A07A020001000000FE
:1048E00008003700CED1BF00E24F500003003A006D
:1048F000B2F102000100000002003700685C020013
:1049000001000000318E8000F00F2000808F5000E9
:1049100016003E00C3D1BF008080FB00C4D1BF00A1
:104920000080FB00EC09B900000141008201410058
:10493000C2CB220002814100120178000201E8008E
:10494000EC0AB9008400780000804000800040003C
:10495000C0CB22000080400002087800308E80002A
:104960000000E800308E880028003700C5D1BF0065
:104970000004E00025003200C3D1BF000040E80081
:10498000C3F1B700C3D1BF00E74F500001003600AC
:10499000C371EF000040EB00004F780017003700B4
:1049A000C3D1BF008080FB001E80FB00EC09B90072
:1049B000820078000080400080004000C0CB2200D0
:1049C000008040008000EB0001087800C3D1BF00E8
:1049D0008080FB001E80FB00EC0AB9008400780098
:1049E00000804000C200DD00C0D7220000814000EE
:1049F0006000B8000089BE001E4FE8001E4078002D
:104A0000EB4F5000E6FF3600C631EF000068A9000A
:104A10000080FA004F03BE004F02BE004F01BE00EF
:0C4A20004F00BE003600F9000040060008
:104B80000000FA0000E8A9000080FA0000400600DA
:104BC0000000FA000080FA00004006000000FA0031
:104BD00000402A0021002000008C01000080FA0023
:104BE000000006000000FA000080FA000000060045
:104BF0000000FA00FBFF07000080FA00000006003A
:0C4C00000000FA000080FA0000400600EE
:0C4C40000000FA000080FA0000400600AE
:104CC0003600F800809FBE00821F78000800FA00BE
:104CD00040002000000F7800470037001E007800D9
:104CE000110020000008DD0020079800012180004D
:104CF0002E009000008060000000E0003D003200C7
:104D000001D823001E0078004400DD000080400030
:104D100030079800408281000000E800408289004E
:104D20009E00780064805000EB004000018140004C
:104D30004103230081004100910078008100E800D8
:104D40006B004000000140004003230000004100D0
:104D50000108780080908000F60F500003003E00AC
:104D6000809080000000E800010037000000EB00A8
:104D700091908000810F500006003A0070828100FF
:104D80000000E80070828900001D230010079800D1
:104D90000D00370080908000C400DD000005230076
:104DA000008040001007980080908000F60F5000AF
:104DB00003003E00809080000000E8000100370002
:104DC0000000EB00809088001E009000BE00900064
:104DD00007000900311878000001B1000101B1009D
:104DE0002E0090008080EA0000218000008060009A
:104DF000002188001E0FE8001E007800E50F50001B
:104E0000B6FF36000A24A9000468A9000080FA0051
:104E10004F0178004F00BE003600F9000040060048
:104E20000000FA00B431EF00B631EF00B831EF0006
:104E3000BA31EF00C371EF00C471EF0010C0B300CE
:104E4000C5F1B700C631EF00C831EF00CA31EF003D
:104E5000CC71EF0005E1A9000421A90004C1A9005B
:104E60002108800000032000010070002008880055
:104E70000021EF0020262000100888000142800059
:104E8000F0FF280080806000000023000100700017
:104E9000004288000068A9002068A80005E1A80079
:104EA0001FE1A9001E21A9001EC1A900F108800070
:104EB0000003200001007000F00888001421EF00BA
:104EC0000080EB00D00888000368A9002368A900CF
:104ED0001FE1A8000080FA00000006000000FA00B0
:104EE000C08D80000080FA00000006000000FA007B
:104EF000A08D8000B18D8000808E8800918E88000A
:104F00000080FA00000006000600FA004047980002
:104F1000A28D8000B38D8000808E8000918E8000F5
:104F2000001F510001975900C3D1BF008080FB00D2
:104F30004E4090000080FB00EC09B9008200780030
:104F400000804000C200DD00C0D722000080400089
:104F50009000900010007800BE0F5000AE8F5800F7
:104F60000C003D00C3D1BF008080FB004E4090008C
:104F70000080FB00EC09B90082007800008040004E
:104F8000C200DD00C0D72200008040003E1878003B
:104F90002E107800A08D8000B18D8000808E88005A
:104FA000918E88000080FA00000006000200FA00DE
:104FB000004F78001E4078000004E000110032002D
:104FC000154EA90015AEA90015EEA900292EA900BD
:104FD00000EEA900282EA900284EA900014EA90024
:104FE000156EA900280EA90014CEA900288EA900CC
:104FF00015CEA900002EA9000B2EA8001E0EA80099
:1050000010003700154EA80015AEA80015EEA80038
:10501000292EA80000EEA800282EA800284EA800DF
:10502000014EA800156EA800280EA80014CEA800F6
:10503000288EA80015CEA800002EA8000B2EA900CF
:105040001E0EA9000080FA00000006000000FA0011
:10505000213A8000F0F32F0000806000203A8800A1
:10506000213A800000FE2F0000806000203A880076
:1050700060022000303A880040A7A9000028EF0015
:105080000228EF000428EF000628EF000828EF00B0
:105090000E2EEF00222EEF00362EEF00230EA8007A
:1050A000232EA80036CEA80036EEA800370EA800A2
:1050B0000E0EA800194EA90019AEA90019EEA900FC
:1050C0002D2EA90004EEA9002C4EA8002C2EA9001C
:1050D000054EA9002C8EA80019CEA80018CEA80055
:1050E000042EA800C0C2B300AEE6B700C0C2B30031
:1050F000AFE6B70020EEA800222CEF00422CEF0014
:10510000622CEF00242CEF00442CEF00642CEF0005
:10511000202CEF00402CEF00602CEF00000024005A
:10512000206088001000200010608800836AA900B9
:10513000834AA9001154800000F82F00808060008D
:1051400000032000010070001054880083EAA800CA
:1051500083CAA9009C8AA800E1548000C0FF2F00E8
:10516000008060000010A000E05488009DAAA90003
:10517000E1548000F0F32F0000806000E0548800CC
:105180009DCAA9009D2AA9002248A9009DEAA9005C
:105190000080FA00000006000200FA00414680008C
:1051A000F00F2000008F6000E00420009E007800D7
:1051B000808F500004003A002E1D02000200000003
:1051C0000080FA00000006000046800068006000D1
:1051D0000000E0003F003200C068A900910180009B
:1051E000010F7800D0C0B300FE38020002000000BA
:1051F000A0C0B300FE3802000200000040C4B300AB
:10520000FE3802000200000030C5B300FE38020084
:105210000200000020C5B300FE38020002000000BA
:1052200000C5B300FE3802000200000010C4B30045
:10523000FE3802000200000070C4B300FE38020015
:1052400002000000D0C3B300FE38020002000000DC
:1052500000F020001E0060004800DE0000407800E2
:105260009821020002000000FE3802000200000047
:105270001E0078008040780000CFB30000C06000BE
:1052800098210200020000000080FB004400DE00C4
:1052900000407800FE380200020000001E00780086
:1052A000004078006F40600098210200020000007A
:1052B000FE38020002000000D0C0B300FE38020039
:1052C00002000000A0C0B300FE380200020000008F
:1052D000FFFF3700D0C0B300FE380200020000001C
:1052E000A0C0B300FE3802000200000060C5B30099
:1052F000FE38020002000000D0C3B300FE380200F6
:1053000002000000000F20001E0060004400DE00CC
:10531000004078009821020002000000FE380200E0
:10532000020000001E007800004078006F4060001E
:105330009821020002000000FE3802000200000076
:10534000D0C0B300FE38020002000000A0C0B300CD
:10535000FE38020002000000FFFF37000000FA00E4
:1053600005E1A9002068A90011E1A90020E8A90031
:1053700013E1A9002108A9001FE1A9002368A900E1
:105380002168A9002188A9002828A9002342A90092
:1053900021E2A90003C8A90023C8A90023E8A900A5
:1053A0002848A9003342A90031E2A9002088A900B9
:1053B00021C8A90001EBA90011EBA9000080FA00A7
:1053C000000006000000FA00F07781000000E00015
:1053D00004003A0020002000F0778900E28C0200EF
:1053E000010000000080FA00000006000000FA0042
:1053F000F07781000000E00006003A002000200065
:10540000F07789007C8702000100000048870200D5
:1054100001000000007881000000E00004003A0074
:105420006000200000788900DA8602000100000098
:10543000107881000000E00004003A0080002000A5
:105440001078890016870200010000002078810092
:105450000000E00004003A0090002000207889005D
:10546000DA870200010000000080FA000000060058
:105470000200FA00000F7800C4D1BF00D4F1B700D9
:1054800050C0B300C4F1B70013E1A9001221A90074
:1054900012C1A900910880000003200001007000E3
:1054A000900888000A21EF009E007800B0AA2A0028
:1054B0000008B8004208DE00700888000108A90052
:1054C00013E1A8000000000001408000001020004F
:1054D000008060000000E000FBFF3200D4D1BF007C
:1054E000C4F1B7000080FA00000006000800FA00CE
:1054F0001007980021079800320798001E009000BE
:10550000004078006F4F60001E00900080407800DF
:1055100000CFB30080C060003E00900001487800DA
:105520002E00900011C0B300014878001E407800A2
:10553000F14F500006003E001E80FB0081C3220098
:1055400000804000904078002E00900001487800D4
:1055500010C0B3000080FA00000006000400FA004A
:10556000004F7800110798001E4078000004E0000A
:1055700009003200F18D80001E00900001007000D3
:105580008000780020002000943802000200000013
:10559000F08D88000B0037001E0090008080EA002C
:1055A000F08D800000806000F08D8800F08D80001C
:1055B00080007800200020009438020002000000E3
:1055C000F08D88000080FA00000006000000FA005C
:1055D000402A2A0096390200020000000080FA00EA
:1055E000000006000000FA00102D2A009639020083
:1055F000020000000080FA00000006000000FA002F
:10560000E02F2A0096390200020000000080FA0014
:10561000000006000000FA00B0322A0096390200AD
:10562000020000000080FA00000006000000FA00FE
:1056300080352A009639020002000000D0392A0085
:1056400096390200020000000080FA000000060007
:105650000000FA00A03C2A00963902000200000077
:10566000203F2A009639020002000000A0412A00D3
:10567000963902000200000040442A0096390200D8
:1056800002000000E0482A009639020002000000F3
:10569000804D2A009639020002000000B0512A0015
:1056A0009639020002000000E0552A0096390200F7
:1056B00002000000005A2A00963902000200000091
:1056C0000080FA00000006000200FA00004F780097
:1056D0001E4078000004E0000500320080352A00FA
:1056E0009639020002000000D9FF070009003700C8
:1056F000D0392A009639020002000000205E2A00FC
:105700009639020002000000F0602A00963902007B
:10571000020000000080FA00000006000000FA000D
:1057200000642A009639020002000000A06B2A00E3
:10573000963902000200000050722A0096390200D9
:10574000020000000080FA00000006000000FA00DD
:10575000C0792A0096390200020000000080FA0099
:10576000000006000000FA0098FF070080802A0071
:10577000963902000200000050892A009639020082
:1057800002000000C0912A009639020002000000C9
:10579000E2FF070090942A00963902000200000000
:1057A000ABFF070060972A00963902000200000054
:1057B000309A2A0096390200020000009BFF070081
:1057C000E2FF070000A22A00963902000200000052
:1057D0000080FA00000006000000FA00C0A42A00C1
:1057E00096390200020000000080FA000000060066
:1057F0000200FA00004F7800C2D1BF000080FB0019
:10580000E20F50001E003200E20F500005003C0085
:105810000000E00008003200E10F500015003200E7
:1058200025003700E30F500019003200E40F50004C
:105830001B003200200037001E407800A2FF070046
:105840001E407800905B0200010000001E407800BE
:105850000004E000170032001E407800BAA20200E7
:10586000010000001E4078006ACE02000100000026
:10587000110037001E40780093FF07000E0037002C
:105880001E407800905B0200010000000A00370013
:105890001E407800BAA20200010000000600370096
:1058A0001E4078006ACE02000100000000000000E7
:1058B00001003700000000000080FA000000060030
:1058C0000000FA0090A72A009639020002000000AA
:1058D0000E8B0200010000000004E0000300320013
:1058E000E0AF2A009639020002000000B0B02A00A2
:1058F00096390200020000000080FA000000060055
:105900000000FA0040B12A009639020002000000AF
:10591000C2D1BF000080FB00E20F50001400320033
:10592000E20F500005003C000000E00008003200DB
:10593000E10F50000A00320019003700E30F500059
:105940000F003200E40F5000110032001400370045
:1059500040B32A0096390200020000001000370010
:1059600080B32A0096390200020000000C003700C4
:10597000C0B32A0096390200020000000800370078
:1059800000B42A009639020002000000040037002B
:1059900050B42A0096390200020000000000000006
:1059A000A0B42A00963902000200000060B62A0066
:1059B000963902000200000060B92A009639020000
:1059C000020000000080FA00000006000200FA0059
:1059D000004F78001E80FB00E20F50001A003200DA
:1059E000E20F500005003C000000E000080032001B
:1059F000E10F5000120032001C003700E30F50008E
:105A000014003200E40F5000150032001700370078
:105A1000EEFE070041FF0700F2FE0700825B020076
:105A200001000000F5FE070094A202000100000042
:105A3000F8FE070062CE0200010000000B003700F4
:105A400036FF070009003700825B020001000000FA
:105A50000600370094A20200010000000300370096
:105A600062CE020001000000000000000080FA0089
:105A7000000006000000FA0060BC2A00963902000F
:105A80000200000040CB2A0096390200020000000C
:105A900000D62A0096390200020000000080FA00B9
:105AA000000006000800FA0020479800210798002F
:105AB000320798008E01780032DE2A00BE00900086
:105AC0002E00900064020200000000000004E000CC
:105AD000220032001E4078000004E0001E003A0060
:105AE0002E4090000080FB00E20F500010003200BA
:105AF000E20F500005003C000000E000080032000A
:105B0000E10F50000800320014003700E30F50008E
:105B10000A003200E40F50000B0032000F00370083
:105B2000D4FF07000D0037000EFF07000B00370001
:105B3000AC5B02000100000008003700E6A2020092
:105B4000010000000500370092CE020001000000B5
:105B500000000000010037001FFF07000080FA006E
:105B6000000006000600FA0040479800311C2100A2
:105B700091407800114798000040EB00004F7800FA
:105B80003F0037001E4090000004E0000400320097
:105B90001E4090000040E9001047980002003700C6
:105BA00070C0B300104798004E409000EB4F50007B
:105BB00011003A001E4090000080FB00F800B90080
:105BC000F6004000C0CB220000804000900078002A
:105BD000D0CC2C000008B8004208DE0051C0B30051
:105BE000EE28020002000000E0DE2A0096390200E2
:105BF00002000000210037001E4090008080FB0062
:105C00004E4090000080FB00EC09B9008200780053
:105C10000080400080004000C0CB22000080400097
:105C2000100078008000EB00420620008289B90055
:105C3000E002B9008401780003014100430620001E
:105C40000300B800010141008200780092012000A9
:105C5000030020002C110200000000001007980033
:105C600031C0B3001E00900076290200020000003F
:105C700030DF2A0096390200020000001E4FE800C3
:105C80001E407800E74F5000BEFF36000080FA004B
:105C9000000006000400FA0020479800311C210093
:105CA00091407800114798000040EB00004F7800C9
:105CB000200037001E4090000004E0000400320085
:105CC0001E4090000040E900104798000200370095
:105CD00070C0B300104798002E409000EB4F50006A
:105CE000130032001E4090008080FB002E40900088
:105CF0000080FB00EC09B9008200780000804000C1
:105D0000C200DD00C0D7220000804000900090005B
:105D1000100078000000780061C0B300EE28020097
:105D20000200000080DF2A00963902000200000015
:105D30001E4FE8001E407800E74F5000DDFF3600A0
:105D40000080FA00000006000000FA00C571EF00B4
:105D5000C0DF2A009639020002000000B0E42A00E9
:105D60009639020002000000B0C0B3007DFF0700BA
:105D700030E52A00963902000200000060E52A00A2
:105D8000963902000200000050C0B30075FF070002
:105D900030E52A009639020002000000E0E52A0002
:105DA000963902000200000010C0B3006DFF07002A
:105DB00030E52A00963902000200000060E62A0061
:105DC000963902000200000020C0B30065FF070002
:105DD00030E52A009639020002000000E0E62A00C1
:105DE000963902000200000020C0B300A9FF07009E
:105DF00030E52A00963902000200000060E72A0020
:105E0000963902000200000030C0B30055FF0700C1
:105E100030E52A009639020002000000E0E62A0080
:105E2000963902000200000030C0B30099FF07005D
:105E300030E52A009639020002000000E0E72A005F
:105E4000963902000200000060C0B30045FF070061
:105E500030E52A009639020002000000E0E62A0040
:105E6000963902000200000060C0B30089FF0700FD
:105E700030E52A00963902000200000060E82A009E
:105E8000963902000200000090C0B30035FF070001
:105E900030E52A009639020002000000E0E62A0000
:105EA000963902000200000090C0B30079FF07009D
:105EB00030E52A009639020002000000E0E82A00DE
:105EC000963902000200000070C0B30025FF0700F1
:105ED00030E52A009639020002000000E0E62A00C0
:105EE000963902000200000070C0B30069FF07008D
:105EF00030E52A00963902000200000060E92A001D
:105F0000963902000200000080C0B30015FF0700B0
:105F100030E52A009639020002000000E0E62A007F
:105F2000963902000200000080C0B30059FF07004C
:105F300030E52A00963902000200000010C0B300CC
:105F4000C5F1B7000080FA00000006000000FA006A
:105F5000E0E92A00963902000200000070EA2A00F7
:105F60009639020002000000A0EA2A0096390200D9
:105F70000200000060EB2A009639020002000000D7
:105F800080EB2A009639020002000000B62C0200C5
:105F9000020000000080FA00000006000A00FA007B
:105FA0004047980031079800420798004E40900003
:105FB0000004E00002003A00C0D1BF000100370039
:105FC000C1D1BF00104798000E80E8008001780022
:105FD00012EC2A00CE0090003E0090006402020005
:105FE000000000000004E000470032002E40900056
:105FF0000004E0000B003A004E4090000004E00076
:1060000004003A00D0EC2A00963902000200000099
:106010003F00370020EF2A009639020002000000FE
:106020003B0037000040EB00004F78002E4090000E
:10603000E14F500002003A0020C0B300004F78004A
:106040002E409000E24F500002003A0030C0B300F2
:10605000004F78002E409000E34F500002003A00BD
:1060600040C0B300004F78001E4090009E4F50008B
:1060700004003A0070F12A00963902000200000084
:10608000230037001E4078000004E00020003200AA
:1060900030F32A0096390200020000004E409000C2
:1060A0000004E0000E003A009E407800400020000E
:1060B0007E38020002000000C0F1B700F08D8000C1
:1060C00000407800E1406000C0D1BF000080FB00CC
:1060D00082C322009E1A0200020000000C0037005A
:1060E0009E407800500020007E3802000200000030
:1060F000C1F1B7001E80FB00A1C42200A410020061
:106100000200000002003700C22C02000200000062
:106110000080FA00000006001000FA005007980006
:1061200061079800624F9800734F98000040EB00A1
:10613000404798007E4890000004E00003003200D1
:106140007E489000E14F500053003A00C1C4220045
:106150007E4890000080FB00F400B9000080400001
:106160004101200000280200020000007E4890004B
:106170000004E00005003A0030C0B300104798006A
:10618000006A2000100798000400370050C0B300D8
:1061900010479800406B20001007980010C0B30013
:1061A000404798000040EB00004F78001C0037008B
:1061B0001E4078000004E0000A003A007E4890008B
:1061C0000081FB003E009000CE009000F411B90069
:1061D00082017800C2C42200028141000089BE0011
:1061E0000E0037007E4890008081FB001E80FB007F
:1061F0000001E9003E009000CE009000E51AB900D1
:1062000084017800028141000201E800C211DD0032
:10621000C2C42200028141000089BE001E4FE80076
:106220006600470000017800EE0090005E009000DC
:1062300092060200000000000004E00004003200AA
:106240001E4090009E40780080CF5000D8FF39005B
:106250004E4090000004E0000F003200C1C4220054
:106260007E4890000080FB00F400B90000804000F0
:1062700042012000800078001E00900020380200BB
:1062800002000000C1D1BF000080FB00A1C42200B9
:10629000A4100200020000000080FA0000000600C6
:1062A0000A00FA00404798005147980032079800CA
:1062B00043079800C11B210091407800014F7800EE
:1062C0006300470080017800D2F42A00CE009000DD
:1062D0003E00900064020200000000000004E000A4
:1062E0000C0132003E4090000080FB00CF80DE00B9
:1062F000D200200003002000820F5000838F58003E
:10630000F6003E00000601000D00370010003700C7
:106310006200370071003700F3003700F2003700E9
:106320007E0037008F0037008E0037009F00370057
:10633000B0003700EC003700C0003700D500370050
:1063400040F82A009639020002000000E7003700FA
:1063500088A30200010000001047980046C3020015
:106360000100000020479800BCD1BF000004E000FD
:1063700006003A001E4090000004E00003003A00CE
:106380002E4090000004E00040003200E0072B00A7
:106390009639020002000000BCD1BF000080FB0063
:1063A000620060000000E0000300320060082B0083
:1063B0009639020002000000BCD1BF000080FB0043
:1063C000640060000000E00003003200C0082B0001
:1063D00096390200020000001E4090000080FB0081
:1063E000620060000000E0000300320020092B0082
:1063F00096390200020000001E4090000080FB0061
:10640000640060000000E00003003200A0092B00DF
:1064100096390200020000001E4090000080FB0040
:1064200061006000004078000004E00003003200DA
:10643000100A2B0096390200020000001E40900056
:106440000080FB00680060000000E00003003200F4
:10645000A00A2B0096390200020000002E40900096
:106460000080FB00620060000000E00003003200DA
:10647000300B2B00963902000200000030E52A00A4
:10648000963902000200000098003700800B2B00B4
:10649000963902000200000094003700100D2B0016
:1064A00096390200020000004E4090000004E00017
:1064B000050032001E14A000600E2B009639020069
:1064C00002000000890037001E14A100B00E2B004E
:1064D000963902000200000084003700100F2B00E4
:1064E00096390200020000004E4090000004E000D7
:1064F000050032001E24A000600E2B009639020019
:1065000002000000790037001E24A100B00E2B000D
:1065100096390200020000007400370060102B0062
:1065200096390200020000004E4090000004E00096
:1065300004003200600E2B009639020002000000B9
:1065400003003700B00E2B00963902000200000055
:10655000410020004E40900050A3020001000000C6
:1065600062003700C0112B009639020002000000C3
:106570004E4090000004E00004003200600E2B004A
:10658000963902000200000003003700B00E2B0015
:106590009639020002000000210020004E409000C9
:1065A00050A30200010000005000370030132B0000
:1065B00096390200020000004E4090000004E00006
:1065C00004003200600E2B00963902000200000029
:1065D00003003700B00E2B009639020002000000C5
:1065E000810020004E40900050A3020001000000F6
:1065F0003E003700B0142B00963902000200000064
:106600004E4090000004E00004003200600E2B00B9
:10661000963902000200000003003700B00E2B0084
:106620009639020002000000210020004E40900038
:106630000EC30200010000002C003700F0152B00F3
:1066400096390200020000004E4090000004E00075
:1066500004003200600E2B00963902000200000098
:1066600003003700B00E2B00963902000200000034
:10667000110020004E40900050A3020001000000D5
:10668000110020004E409000185702000100000049
:1066900016003700800B2B00963902000200000024
:1066A0000040EB00004F7800F10F20000040EB00AD
:1066B0001857020001000000F10F20000040EB001D
:1066C00050A3020001000000F10F20000040EB0089
:1066D0000EC302000100000004003700C22C0200BB
:1066E000020000000100370000000000BCD1BF0024
:1066F0009E40780080CF5000080032009E40780015
:106700000000EB007E38020002000000BCF1B70080
:1067100002003700C22C0200020000000080FA00D4
:10672000000006000200FA00004F780011479800B0
:106730001E4090000004E000090032009E407800F6
:106740001E4090008A7302000000000011C0B300D8
:106750001E409000027A0200000000000300370093
:1067600070172B0096390200020000000080FA002A
:10677000000006000A00FA00404798003107980020
:10678000420798000040EB00004F78000040EB000B
:10679000104798000E80E8008001780022192B0035
:1067A000CE0090003E009000640202000000000055
:1067B0000004E000560032002E4090000080FB00F4
:1067C000CF80DE003201200003002000820F500045
:1067D000838F58003C003E00000601003C0037005B
:1067E0001200370011003700100037000F0037008B
:1067F0000E0037000D0037000C0037000E00370088
:106800001000370012003700140037001600370060
:10681000180037001A0037001C0037001E00370030
:10682000200037002200370024003700AE409000DF
:10683000014F78002700370060C0B3001047980070
:106840002400370010C0B300104798002100370023
:1068500080C0B300104798001E00370020C0B3006E
:10686000104798001B00370030C0B3001047980055
:106870001800370040C0B3001047980015003700DB
:1068800050C0B300104798001200370070C0B3002A
:10689000104798000F00370090C0B30010479800D1
:1068A0000C003700A0C0B300104798000900370063
:1068B000B0C0B3001047980006003700E0C0B30036
:1068C0001047980003003700000000000100370067
:1068D000000000002E4090000004E00002003A009A
:1068E000F7FB07000C0037009E4090001E40780028
:1068F000365E0200000000000004E00006003A00DE
:10690000901F2B00963902000200000002003700A1
:10691000C22C0200020000000080FA000000060005
:106920000400FA00881F7800204798002E4090004D
:106930000004E00003003200C0202B009639020062
:1069400002000000F0012000843702000200000075
:10695000BDF1B7002E4090000004E00006003A00B0
:10696000BDD1BF000004E00003003200BDD1BF0074
:10697000E44F50000500360011C0B300F0012000C4
:106980007E38020002000000BDF1B7000000EB00FD
:106990008437020002000000BCF1B7002E409000D6
:1069A0000004E00006003A00BCD1BF008080FB007C
:1069B000000F2000008060000000E00005003200B1
:1069C0008040EB000000EB007E3802000200000077
:1069D000BCF1B70020002000963702000200000042
:1069E000F08D88002E4090000004E00005003A0081
:1069F000F18D800000F82F00008060000000E000B2
:106A00000500320021002000200020009438020000
:106A100002000000F08D8800400020008437020052
:106A200002000000C0F1B7002E4090000004E0001A
:106A300003003A00C0D1BF00E14F400005003A001A
:106A400031C0B300400020007E3802000200000088
:106A5000C0F1B7005000200084370200020000009F
:106A6000C1F1B7002E4090000004E00003003A009E
:106A7000C1D1BF00E14F400005003A0041C0B30062
:106A8000500020007E38020002000000C1F1B70073
:106A9000C0C422004201200080007800006A20006B
:106AA0003A370200020000002E4090000004E0008F
:106AB00007003A0062628100736281000080EB008F
:106AC0008080EB00800F5100818F59000A003A004E
:106AD000C0C4220041012000002802000200000082
:106AE000C0C422004201200080007800006A20001B
:106AF0002038020002000000C0C4220074004000E0
:106B00004201200080007800406B20003A370200EC
:106B1000020000002E4090000004E00007003A0050
:106B200002638100136381000080EB008080EB0032
:106B3000800F5100818F59000C003A00C0C4220020
:106B40007400400041012000002802000200000003
:106B5000C0C4220074004000420120008000780080
:106B6000406B20002038020002000000F18D800000
:106B7000000420000080600000F0A7000000EA0090
:106B80000000EA004F00DE00004078000080FB00BB
:106B900061006000516281000100A10001007000ED
:106BA000506289002201200081C322006000200081
:106BB0003A370200020000000040EB00004F78006E
:106BC000180037001E80FB0081C3220000804000B7
:106BD00090407800114798002E4090000004E0009B
:106BE00003003A001E409000F14F50000C003600A8
:106BF0001E84FB001E80FB00016C2300008040000F
:106C0000904078001E80FB00660040007E38020045
:106C10000200000081C32200888040008048780084
:106C20001E4FE8001E407800F14F5000E5FF36008F
:106C3000B0C322008040EB000148780020C422004D
:106C40008040EB00014878002E4090000C6002006C
:106C5000000000002E409000B46B02000000000015
:106C60002E4090000004E0000300320090212B0031
:106C700096390200020000004F0478000080FA00FC
:106C8000000006000200FA00004F78001E40780065
:106C900023FF07001E4078003C12020001000000A4
:106CA0001E407800447F0200010000001E40780072
:106CB00086C80200010000001E4078003AF502007C
:106CC000010000000080FA00000006000600FA0043
:106CD000F0850200010000000004E0000100320025
:106CE000C2F90700228B0200010000000004E0004E
:106CF00001003200B3F9070064004700E6FB020020
:106D0000010000000004E00007003200307881003C
:106D10000000E00004003A002E0090003078890066
:106D20009CFC0200010000006400470000FC02001F
:106D3000010000000004E0000700320040788100FC
:106D40000000E00004003A002E0090004078890026
:106D5000F2FC020001000000640047001AFC02007F
:106D6000010000000004E0000700320050788100BC
:106D70000000E00004003A002E00900050788900E6
:106D80005EFD0200010000006400470034FC0200C8
:106D9000010000000004E00007003200607881007C
:106DA0000000E00004003A002E00900060788900A6
:106DB0009AFD020001000000640047004EFC020042
:106DC000010000000004E00007003200707881003C
:106DD0000000E00004003A002E0090007078890066
:106DE00028FD0200010000006400470068FC02006A
:106DF000010000000004E0000900320080788100FA
:106E00000000E00004003A002E0090008078890025
:106E1000D0FE020001000000DAFE020001000000C6
:106E20006400470082FC0200010000000004E00052
:106E300009003200907881000000E00004003A0070
:106E40002E009000907889003EFF020001000000B3
:106E500044FF020001000000CDD1BF000004E000AB
:106E600081003200CCD1BF000004E0007E0032007F
:106E7000CC71EF000040EB0020479800770037000E
:106E80002E4090000080FB0081F122000080400035
:106E9000104078000004E0006D0032002E409000A9
:106EA0000080FB0081F1220080804000914078004A
:106EB0008140E90082F12200000041000148780091
:106EC0002E4090000080FB0081F1220000804000F5
:106ED000104078000004E0005D003A002E40900071
:106EE0000004E00003003A0000F22F00000F7800D9
:106EF000200037002E409000E14F500003003A0080
:106F000010F22F00000F78001A0037002E4090007A
:106F1000E24F500003003A0020F22F00000F7800EB
:106F2000140037002E409000E34F500003003A0059
:106F300030F22F00000F78000E0037002E40900036
:106F4000E44F500003003A0040F22F00000F780099
:106F5000080037002E409000E54F500003003A0033
:106F600000F32F00000F7800020037000000EB0054
:106F7000000F78002E4090000080FB0061F222009C
:106F800000804000104078000004E000180032004B
:106F90002E4090000080FB00D1F2220000804000D3
:106FA000104078000041EB009E007800F10B0700D4
:106FB0002E4090000080FB0061F222000080400023
:106FC00010407800E14F4000090032002E40900050
:106FD0000080FB0061F22200808040009140780038
:106FE0008140E90062F2220000004100014878007F
:106FF0002E4090000080FB0061F2220000804000E3
:10700000104078000004E0000B0032002E40900099
:107010000080FB00AE4090008180FB00F2F1220076
:10702000810041009140780082F12200000041007F
:1070300001487800060037002E4090000080FB00D9
:10704000F1F12200008040008040EB000148780010
:107050002E4090000040E800204798002E4090000D
:10706000E64F500086FF36000205020001000000D6
:107070000080FA00000006000000FA00AA200200CA
:1070800002000000721A0200020000000080FA00F4
:10709000000006000600FA00004F78001107980073
:1070A000220798004658020001000000F2FF070086
:1070B0000080FA00000006000200FA00004F78008D
:1070C0001E4078000004E000030032001E407800FB
:1070D000E14F50000F003A00F08D80000040780032
:1070E000E1406000C0D1BF000080FB0082C32200ED
:1070F0009E1A020002000000C1D1BF000080FB0008
:10710000A1C42200A410020002000000247D02009D
:1071100000000000607F02000000000011C0B3000A
:107120000040EB0034740200000000001E407800B4
:107130000004E000030032001E407800E34F5000DE
:1071400002003A0088C00200010000001E407800E2
:107150000004E000030032001E407800E24F5000BF
:1071600004003A00F45C020001000000D4050200B3
:10717000020000001E4078000004E000030032001E
:107180001E407800E44F500002003A0074F1020003
:10719000010000000080FA00000006000200FA0072
:1071A000004F78001E80FB00E20F500019003200F3
:1071B000E20F500005003C000000E0000800320033
:1071C000E10F5000090032001A003700E30F5000B1
:1071D0000C003200E40F500012003200150037009E
:1071E00010C0B300A7FE07001200370010C0B300A4
:1071F000CBFD070010C0B3003AF50200010000000B
:107200000C00370010C0B300447F020001000000F2
:107210000800370010C0B3003C120200010000005B
:107220000400370010C0B30086C80200010000004F
:10723000000000001E4078009FFF07000080FA0059
:10724000000006000400FA00B17080000008200071
:10725000008060000000E0001F00320010222B00C0
:107260009639020002000000A0222B00963902008D
:107270000200000030272B009639020002000000B7
:10728000C02B2B00963902000200000050302B006A
:107290009639020002000000A08D8000B18D8000B0
:1072A0000204200003002000021F40000397480052
:1072B00000000000A08D8000B18D8000BE0F500046
:1072C000AE8F5800FBFF350024F80700E6250200CA
:1072D000000000000300370000352B009639020043
:1072E000020000000080FA00000006000000FA0022
:1072F000020620008000EB0000002100AA310200FD
:10730000020000004C800200010000009A160200FA
:107310000100000028CB0200010000000080FA00FC
:10732000000006000200FA00004F78001E407800BE
:10733000E24F500004003A00F0372B00963902006B
:10734000020000000D0037001E407800E34F50009F
:1073500004003A0080382B00963902000200000039
:10736000060037001E407800E44F500003003A004A
:1073700010392B0096390200020000000080FA004C
:10738000000006000400FA00004F78001107980082
:107390001E80FB006101B900D0FF2F00F1FF2F001C
:1073A0000200400083804800E2002000030020002B
:1073B000820F5000838F5800D8003E000006010065
:1073C0000E0037001B003700280037003900370057
:1073D0008000370091003700A2003700B30037006B
:1073E000460037005700370068003700CD003700EF
:1073F000CC003700CB003700BA0037001E009000E9
:10740000104078000004E00003003200A0392B0097
:107410009639020002000000D0392B009639020094
:10742000020000001E00900011C0B3000148780067
:10743000CD0037001E009000104078000004E000EE
:1074400003003200A0392B00963902000200000030
:10745000303A2B0096390200020000001E00900016
:1074600011C0B30001487800BF0037000E8B020046
:10747000010000000004E000AC0032001E0090009B
:10748000104078000004E00003003200A0392B0017
:107490009639020002000000C03A2B009639020023
:1074A000020000001E00900011C0B30001487800E7
:1074B000AD0037008AC20200010000000004E000B5
:1074C0009C0032001E009000104078000004E00094
:1074D00003003200A0392B009639020002000000A0
:1074E000503B2B0096390200020000001E00900065
:1074F00011C0B300014878009B0037009EC2020013
:10750000010000000004E0008C0032001E0090002A
:10751000104078000004E00003003200A0392B0086
:107520009639020002000000B03B2B0096390200A1
:10753000020000001E00900011C0B3000148780056
:1075400089003700AAC20200010000000004E00028
:107550007C0032001E009000104078000004E00023
:1075600003003200A0392B0096390200020000000F
:10757000303C2B0096390200020000001E009000F3
:1075800011C0B3000148780077003700BEC2020086
:10759000010000000004E0006C0032001E009000BA
:1075A000104078000004E00003003200A0392B00F6
:1075B0009639020002000000B03C2B009639020010
:1075C000020000001E00900011C0B30001487800C6
:1075D00065003700D2C20200010000000004E00094
:1075E0005C0032001E009000104078000004E000B3
:1075F00003003200A0392B0096390200020000007F
:10760000303D2B0096390200020000001E00900061
:1076100011C0B300014878005300370006FA020099
:10762000000000000004E0004C0032001E0090004A
:10763000104078000004E00003003200A0392B0065
:107640009639020002000000803D2B0096390200AE
:10765000020000001E00900011C0B3000148780035
:1076600041003700F0850200010000000004E00046
:107670003C0032001E009000104078000004E00042
:1076800003003200A0392B009639020002000000EE
:10769000D03D2B0096390200020000001E00900031
:1076A00011C0B300014878002F0037001E00900081
:1076B000104078000004E00003003200A0392B00E5
:1076C0009639020002000000403E2B00963902006D
:1076D000020000001E00900011C0B30001487800B5
:1076E000210037001E009000104078000004E000E8
:1076F00003003200A0392B0096390200020000007E
:10770000C03E2B0096390200020000001E009000CF
:1077100011C0B300014878001300370000000000DA
:1077200011003700000000000F00370000000000CB
:107730000D003700000000000B00370000000000C3
:1077400009003700000000000700370000000000BB
:1077500005003700000000000300370000000000B3
:1077600001003700000000000080FA000000060061
:107770000200FA00503F2B00963902000200000080
:10778000C0D1BF00E7FE070030E52A0096390200AD
:1077900002000000F08D8000610060000040780071
:1077A0000004E0000600320040402B009639020041
:1077B0000200000010412B00963902000200000078
:1077C000D0412B009639020002000000C1D1BF0059
:1077D000D4FE070030E52A009639020002000000BE
:1077E000F18D800000042000008060000000E000B7
:1077F00006003200C0422B00963902000200000051
:1078000010412B00963902000200000060628100E6
:107810007162810000007800000F78001E0078007F
:107820000000E0001900320090432B00963902005E
:1078300002000000110020000E0078001C2B020046
:1078400002000000A0442B00963902000200000054
:1078500000C52200110020001C2B020002000000C5
:10786000F0442B00963902000200000000C52200FF
:1078700064004000110020001C2B020002000000E8
:1078800030E52A0096390200020000000063810002
:107890001163810000007800000F78001E0078005E
:1078A0000000E0002900320040452B00963902001C
:1078B00002000000110020000E0078001C2B0200C6
:1078C00002000000A0442B009639020002000000D4
:1078D00040C62200110020001C2B02000200000004
:1078E000F0442B00963902000200000040C622003E
:1078F00064004000110020001C2B02000200000068
:1079000050462B00963902000200000040C62200BB
:1079100068004000110020001C2B02000200000043
:10792000A0462B00963902000200000040C622004B
:107930006C004000110020001C2B0200020000001F
:1079400030E52A0096390200020000000080FA00AB
:10795000000006000A00FA00004F9800114F98003E
:107960000E4890000004E0002B003A00503F2B002E
:107970009639020002000000C0D1BF0069FE070076
:1079800030E52A009639020002000000F0462B0084
:1079900096390200020000000040EB0060479800AA
:1079A00020C0B300204798000E0037002E40900002
:1079B0000080FB0081C3220000804000104078005E
:1079C000E14F500004003A00660047008000780054
:1079D0002E4090006BFE07002E4090000040E80013
:1079E000204798002E409000F14F5000EFFF3600E6
:1079F00030E52A00963902000200000064004700CA
:107A00006A2002000200000078200200020000004C
:107A1000000F78002A003700D0412B009639020071
:107A200002000000C1D1BF003EFE070030E52A0081
:107A30009639020002000000F0462B009639020041
:107A4000020000000040EB006047980020C0B30037
:107A5000204798000E0037002E4090000080FB0069
:107A600081C322000080400010407800E24F5000A7
:107A700004003A0066004700800078002E40900025
:107A800040FE07002E4090000040E800204798008C
:107A90002E409000F14F5000EFFF360030E52A00F5
:107AA000963902000200000064004700541A0200E8
:107AB00002000000621A020002000000000F7800BD
:107AC0001E4890000004E000D4003200E0472B0084
:107AD00096390200020000002E009000100078008D
:107AE00051C0B300EE28020002000000D0482B0075
:107AF00096390200020000002E0090001000900055
:107B000011C0B300EE28020002000000A0392B00D3
:107B100096390200020000002E0090002000900024
:107B200011C0B300EE28020002000000A0392B00B3
:107B300096390200020000002E00900030009000F4
:107B400011C0B300EE280200020000000E489000B1
:107B50000004E00008003A00A0392B00963902002A
:107B6000020000002E0090004000900011C0B30001
:107B7000EE2802000200000000492B0096390200A6
:107B800002000000000022001E0060000000E00073
:107B90000400320020492B00963902000200000048
:107BA0000F003700000021001E0060000000E00010
:107BB00004003200B0492B00963902000200000098
:107BC00007003700004020001E0060000000E000B9
:107BD00003003200804A2B009639020002000000A8
:107BE0002E009000100890000000E0000800320015
:107BF000204B2B0096390200020000002E0090005E
:107C00001008900011C0B300EE280200020000002E
:107C10002E009000500090000000E00008003200AC
:107C2000D04B2B0096390200020000002E0090007D
:107C30005000900011C0B300EE28020002000000C6
:107C40002E009000600090000000E000080032006C
:107C5000A04C2B0096390200020000002E0090007C
:107C60006000900011C0B300EE2802000200000086
:107C70002E009000000890000000E0000800320094
:107C8000204D2B0096390200020000002E009000CB
:107C90000008900011C0B300EE28020002000000AE
:107CA0002E009000700090000000E00008003200FC
:107CB000B04D2B0096390200020000002E0090000B
:107CC0007000900011C0B300EE2802000200000016
:107CD00030E52A009639020002000000404E2B00D9
:107CE00096390200020000002E009000200890004B
:107CF00051C0B300EE28020002000000D0482B0063
:107D000096390200020000002E009000300890001A
:107D100011C0B300EE28020002000000A0392B00C1
:107D200096390200020000002E00900040089000EA
:107D300011C0B300EE2802000200000000492B0031
:107D400096390200020000002E00900050089000BA
:107D50000000E00008003200304F2B00963902008E
:107D6000020000002E0090005008900011C0B300E7
:107D7000EE28020002000000008020001E006000CB
:107D80000000E00004003200F04F2B0096390200A2
:107D9000020000000F003700002020001E006000DD
:107DA0000000E00004003200C0502B0096390200B1
:107DB0000200000007003700001020001E006000D5
:107DC0000000E0000300320060512B0096390200F1
:107DD000020000009E007800648060000000E00067
:107DE0000400320060522B009639020002000000AD
:107DF000070037009E007800688060000000E00007
:107E00000300320090532B0096390200020000005C
:107E100030E52A0096390200020000000080FA00D6
:107E2000000006000A00FA00881F7800404798000A
:107E300051479800320798004307980010C0B300DC
:107E4000004F78004E4090000004E000280032000F
:107E50000E80E80080017800F2542B00CE009000E4
:107E60003E00900064020200000000000004E000F8
:107E70001A0032002E4090000004E00003003A0097
:107E800010C0B30010479800080037002E40900043
:107E9000E14F500003003A0010C0B30010479800B3
:107EA0000200370020C0B300104798005E409000E9
:107EB0000084FB005E4090000080FB0066004000F4
:107EC0009E4090007E3802000200000081C3220024
:107ED0008880400080487800100037000040EB00A8
:107EE000004F7800C22C0200020000000B00370097
:107EF0005E4090000084FB005E4090000080FB002C
:107F0000660040008040EB007E3802000200000066
:107F100081C3220088804000804878001E4078009D
:107F20004F0478000080FA00000006000800FA0004
:107F30002047980021079800320798008E017800AA
:107F400092552B00BE0090002E00900064020200AB
:107F5000000000000004E000120032001E40780023
:107F60000004E00003003A00A2A2020001000000A9
:107F70000E0037001E407800E14F500006003A0026
:107F80003E019000AE00900010C0B300E0AC0200D3
:107F90000100000005003700C22C020002000000B2
:107FA00002003700C22C0200020000000080FA002C
:107FB000000006000800FA002047980021079800FA
:107FC000320798008E01780092552B00BE00900079
:107FD0002E00900064020200000000000004E00097
:107FE000120032001E4078000004E00003003A0056
:107FF000AEA20200010000000E0037001E40780013
:10800000E14F500006003A003E019000AE009000A3
:108010000040EB00E0AC020001000000050037006A
:10802000C22C02000200000002003700C22C020035
:10803000020000000080FA00000006000800FA00BC
:10804000204798003147980022079800330798008E
:108050000E00E8008001780012562B00BE00900050
:108060002E00900064020200000000000004E00006
:108070004D0132001E4090000080FB00CF80DE00EA
:108080008202200003002000820F5000838F5800DE
:1080900048013E0000060100280037002A00370092
:1080A0002D0037003000370033003700360037002E
:1080B00039003700430037004200370046003700E0
:1080C0003E013700490037004E0037004D003700B1
:1080D0003A0137005100370054003700570037008D
:1080E0005A0037005D003700680037007300370022
:1080F000780037007D003700880037008B0037009C
:10810000900037009B003700A6003700B100370011
:10811000BC003700C0003700C4003700CF00370074
:10812000E5003700EB003700F1003700F5003700BD
:10813000F9003700040137000F0137002E4090008E
:10814000ABF507003201370011C0B3002E4090009C
:1081500074F907002E01370021C0B3002E409000B3
:1081600070F907002A01370031C0B3002E4090009B
:108170006CF907002601370041C0B3002E40900083
:1081800068F907002201370051C0B3002E4090006B
:1081900064F907001E01370010C0B300004F7800DB
:1081A000040037009E4078002E4090005DF90700E3
:1081B0001E4FE8001E407800E54F5000F9FF3600E2
:1081C00013013700010120002E4090001CAA02007C
:1081D000010000000E013700010220002E40900037
:1081E0001CAA020001000000090137003E019000B6
:1081F000AE0090002E4090001C52020001000000D2
:10820000030137003E019000AE0090002E40900028
:108210005252020001000000FD0037000101200061
:108220002E409000CDF40700F90037000102200035
:108230002E409000C9F40700F5003700210020000F
:108240002E409000C5F40700F100370041002000E7
:108250002E409000C1F40700ED003700BE019000F1
:108260002E01900051C0B3002E409000EDFE07009B
:108270000004E000D3003200810020002E40900076
:108280001CAA020001000000E1003700BE019000BE
:108290002E01900061C0B3002E409000E1FE070067
:1082A0000004E000C9003200810020002E40900050
:1082B00010F0020001000000D5003700BE01900060
:1082C0002E01900071C0B3002E409000D5FE070033
:1082D000CF003700BE0190002E01900081C0B30096
:1082E0002E409000CFFE0700C9003700BE0190006D
:1082F0002E01900091C0B3002E409000C9FE0700EF
:108300000004E000B3003200010420002E40900081
:108310001CAA020001000000BD00370081002000FF
:108320002E4090008DF40700B9003700BE01900088
:108330002E01900041C0B3002E409000B9FE07000E
:10834000B3003700BE0190002E019000B1C0B30011
:108350002E409000B3FE07000004E0009F003200B2
:10836000110020002E40900010F0020001000000DB
:10837000A7003700BE0190002E019000C1C0B300DD
:108380002E409000A7FE07000004E0009500320098
:10839000210020002E40900010F00200010000009B
:1083A0009B003700BE0190002E019000C1C0B300B9
:1083B0002E4090009BFE07000004E0008B0032007E
:1083C000012020002E40900010F00200010000006B
:1083D0008F003700BE0190002E019000D1C0B30085
:1083E0002E4090008FFE07000004E0008100320064
:1083F000410020002E40900010F00200010000001B
:1084000083003700010021002E40900010F0020090
:10841000010000007E003700010820002E4090007F
:1084200010F0020001000000790037001100200068
:108430002E40900049F40700F08D80000040780045
:10844000E1406000C0D1BF000080FB0082C3220079
:108450009E1A0200020000006D0037000104200097
:108460002E4090003DF40700F18D800000042000B4
:108470000080600000F0A7000000EA000000EA00B1
:108480004F00DE00004078000080FB0061006000CB
:10849000516281000100A10001007000506289005A
:1084A000C1D1BF000080FB00A1C42200A4100200C3
:1084B0000200000056003700BE0190002E0190001F
:1084C00011C0B3002E4090000CF602000100000025
:1084D0004F003700BE0190002E01900021C0B30074
:1084E0002E4090000CF6020001000000480037000A
:1084F000011020002E40900010F00200010000004A
:1085000043003700010022002E40900010F00200CE
:10851000010000003E003700BE0190002E019000D7
:1085200001C1B3002E4090003EFE07000004E000B1
:1085300032003200014020002E40900010F0020076
:108540000100000032003700BE0190002E019000B3
:10855000F1C0B3002E40900032FE07000004E0009E
:1085600028003200018020002E40900010F0020010
:108570000100000026003700BE0190002E0190008F
:1085800011C1B3002E40900026FE07000004E00059
:108590001E003200010024002E40900010F0020066
:1085A000010000001A003700C22C02000200000087
:1085B0001700370000000000150037000000000021
:1085C0001300370000000000110037000000000019
:1085D0000F003700000000000D0037000000000011
:1085E0000B00370000000000090037000000000009
:1085F0000700370000000000050037000000000001
:1086000003003700000000000100370000000000F8
:108610000080FA00000006000800FA0020479800D9
:1086200021079800320798008E01780052672B00CE
:10863000BE0090002E0090006402020000000000C6
:108640000004E000210032001E4078000080FB00A2
:10865000E30F500011003200E30F500005003C0012
:108660000000E000080032000000E0001A003500C1
:1086700007003700E50F50000D003400E60F5000F2
:108680000E003200150037009DF40700130037007C
:108690002E409000C1FA0700100037003E01900004
:1086A000AE0090002E4090007AFA07000B003700D1
:1086B0000A6702000100000008003700EC11020008
:1086C000000000000000000004003700C22C02007F
:1086D0000200000001003700000000000080FA00E6
:1086E000000006000E00FA0050079800610798008D
:1086F0000040EB00204798006400470080017800AC
:108700000081EB00EE0090005E0090008A360200CF
:10871000020000000004E00025003200660047006F
:1087200080017800F20F2000EE0090005E009000C3
:108730008A360200020000000004E0001C00320043
:108740006800470000017800EE0090005E00900095
:108750000E040200000000000004E00002003A00E5
:1087600010002000400798000000EB00000F780088
:10877000090037003E009000804078002E009000F5
:108780007E380200020000002E0090000000E80089
:10879000200798001E0FE8004E0090009E00780011
:1087A000808F5000F3FF390010C0B30020479800BD
:1087B0000080FA00000006000800FA002047980038
:1087C00021079800320798008E01780072692B000B
:1087D000BE0090002E009000640202000000000025
:1087E0000004E000B80132001E4078000080FB0069
:1087F000CF80DE006204200003002000820F5000C2
:10880000838F5800B3013E00000601004600370088
:10881000480037004C003700500037005500370043
:108820005A0037005F0037006400370068003700E7
:108830006C0037007000370074003700A701370064
:10884000770037007B0037007F0037008300370058
:10885000870037008B0037008F0037009300370008
:10886000970037009B0037009F003700A3003700B8
:10887000A7003700AB003700AF003700B300370068
:10888000B7003700BB003700BF003700C300370018
:10889000C7003700CB003700CF003700D3003700C8
:1088A000D7003700DB003700DF003700E300370078
:1088B000E7003700EB003700EF003700F400370027
:1088C000F9003700FD0037000101370005013700CE
:1088D0000901370081013700800137000B013700A3
:1088E0000F01370014013700190137001E0137004E
:1088F00023013700280137002D01370032013700EE
:10890000370137003C01370041013700450137008E
:108910004A0137004F013700540137005901370031
:108920005E013700630137002E40900027F40700F6
:108930006B0137003E019000AE0090000040EB005C
:1089400096F50700660137003E019000AE009000EA
:1089500010C0B30091F50700610137003E0190009F
:10896000AE0090000040EB006CAD02000100000082
:108970005B0137003E019000AE00900010C0B300D4
:108980006CAD020001000000550137003E0190006F
:10899000AE00900020C0B3006CAD020001000000EA
:1089A0004F0137003E019000AE00900030C0B30090
:1089B0006CAD02000100000049013700BE009000CC
:1089C0002E00900030B0020001000000440137008A
:1089D000BE0090002E0090001AB1020001000000BD
:1089E0003F013700BE0090002E00900082B10200CF
:1089F000010000003A013700BE0090002E009000F8
:108A0000D8B102000100000035013700BE0090001F
:108A10002E00900042B20200010000003001370039
:108A2000BE0090002E00900098B2020001000000ED
:108A30002B013700BE0090002E009000EEB2020025
:108A40000100000026013700BE0090002E009000BB
:108A500072B302000100000021013700BE00900047
:108A60002E009000C8B30200010000001C01370076
:108A7000BE0090002E0090001EB402000100000015
:108A800017013700BE0090002E00900074B4020061
:108A90000100000012013700BE0090002E0090007F
:108AA000CAB40200010000000D013700BE009000B2
:108AB0002E00900020B502000100000008013700E0
:108AC000BE0090002E00900090B502000100000052
:108AD00003013700BE0090002E009000C6AF0200D8
:108AE00001000000FE003700BE0090002E00900044
:108AF000C04B020001000000F9003700BE009000EA
:108B00002E009000824D020001000000F4003700AA
:108B1000BE0090002E0090003A4E020001000000BE
:108B2000EF003700BE0090002E0090009A4E020029
:108B300001000000EA003700BE0090002E00900007
:108B4000524F020001000000E5003700BE00900017
:108B50002E0090002050020001000000E0003700CD
:108B6000BE0090002E009000B24F020001000000F5
:108B7000DB003700BE0090002E009000385102004C
:108B800001000000D6003700BE0090002E009000CB
:108B9000CE51020001000000D1003700BE0090005D
:108BA0002E009000F04D020001000000CC003700C4
:108BB000BE0090002E009000084F0200010000004F
:108BC000C7003700BE0090002E009000B2310200B6
:108BD00001000000C2003700BE0090002E0090008F
:108BE000180F020002000000BD003700BE00900018
:108BF0002E0090008050020001000000B8003700F5
:108C0000BE0090002E009000DC5002000100000029
:108C1000B3003700BE0090002E009000B4CE0200DA
:108C200001000000AE003700BE0090002E00900052
:108C3000B0CF020001000000A9003700BE00900084
:108C40002E009000F2CF020001000000A4003700C7
:108C5000BE0090002E00900090D0020001000000A5
:108C60009F003700BE0090002E00900004D102004B
:108C7000010000009A0037003E019000AE00900015
:108C800010C0B30038CB0200010000009400370090
:108C90003E019000AE0090000040EB0038CB020097
:108CA000010000008E003700BE0090002E009000F2
:108CB000EACB02000100000089003700BE009000EE
:108CC0002E009000D0EE020001000000840037006A
:108CD000BE0090002E00900014EF02000100000082
:108CE0007F003700BE0090002E00900082EF02004F
:108CF000010000007A003700BE0090002E009000B6
:108D000078D102000100000075003700BE0090001D
:108D10002E009000C4EF0200010000007000370038
:108D200012C0B300BE0090002E0090004663020007
:108D3000000000006A00370022C0B300BE009000AF
:108D40002E0090004663020000000000640037001F
:108D500032C0B300BE0090002E00900046630200B7
:108D6000000000005E00370042C0B300BE0090006B
:108D70002E009000466302000000000058003700FB
:108D800052C0B300BE0090002E0090004663020067
:108D9000000000005200370012C0B300BE00900077
:108DA0002E0090002C6E0200000000004C003700E6
:108DB00022C0B300BE0090002E0090002C6E020076
:108DC000000000004600370032C0B300BE00900033
:108DD0002E0090002C6E02000000000040003700C2
:108DE00042C0B300BE0090002E0090002C6E020026
:108DF000000000003A00370052C0B300BE009000EF
:108E00002E0090002C6E020000000000340037009D
:108E1000BE0090002E0090005432020001000000BD
:108E20002F0037000041EB00BE0090002E009000A4
:108E3000E8320200010000002900370012C0B30030
:108E4000BE0090002E009000E832020001000000F9
:108E50002300370022C0B300BE0090002E00900017
:108E6000E8320200010000001D00370032C0B300EC
:108E7000BE0090002E009000E832020001000000C9
:108E8000170037008041EB0022C0B300BE00900005
:108E90002E009000A0F407001100370013C0B300AB
:108EA00022C0B300BE0090002E0090009AF407008C
:108EB0000B003700BE0090002E00900009FE070056
:108EC0000000000006003700C22C02000200000073
:108ED0000300370000000000010037000000000020
:108EE0000080FA00000006000200FA000000EB001B
:108EF000000F78000E017800216D23000040EB0088
:108F00002DFE07000040EB00A4F807000000EB0076
:108F1000000F78000E017800D16D23000040EB00B7
:108F200025FE07000000EB00000F78000E0178001E
:108F3000816E23000040EB001FFE07000000EB00E5
:108F4000000F78000E017800316F23000040EB0025
:108F500019FE07000000EB00000F78000E017800FA
:108F6000D16F23000040EB0013FE07000000EB0070
:108F7000000F78000E017800717023000040EB00B4
:108F80000DFE07000000EB00000F78000E017800D6
:108F9000317123000040EB0007FE07000000EB00EA
:108FA000000F78000E017800D17123000040EB0023
:108FB00001FE07000000EB00000F78000E017800B2
:108FC000917223000040EB00FBFD07000000EB0066
:108FD000000F78000E017800317323000040EB0091
:108FE000F5FD07000000EB00000F78000E0178008F
:108FF000D17323000040EB00EFFD07000000EB0001
:10900000000F78000E017800717423000040EB001F
:10901000E9FD07000000EB00000F78000E0178006A
:10902000117523000040EB00E3FD07000000EB009A
:10903000000F78000E017800B17523000040EB00AE
:10904000DDFD07000000EB00000F78000E01780046
:10905000C17623000040EB00D7FD07000080FA0036
:10906000000006000000FA00D0862B0096390200AE
:109070000200000020882B00963902000200000048
:10908000F08B2B00963902000200000040902B006C
:109090009639020002000000B0932B0096390200BE
:1090A0000200000090972B00963902000200000099
:1090B000609B2B009639020002000000209E2B00CE
:1090C000963902000200000030A12B009639020000
:1090D00002000000C0A62B0096390200020000002A
:1090E00020A92B009639020002000000F0AB2B00F3
:1090F0009639020002000000B0B22B00963902003F
:109100000200000070B52B0096390200020000003A
:10911000B0B82B00963902000200000020BB2B00E3
:1091200096390200020000000080FA0000000600EC
:109130000200FA00004F78001E407800E14F500016
:1091400004003A00E0BD2B00963902000200000046
:10915000060037001E407800E24F500003003A003E
:1091600070BE2B0096390200020000000080FA0059
:10917000000006000200FA00F08D8000620060002E
:109180000000E0000600320000BF2B00963902000C
:109190000200000010412B0096390200020000007E
:1091A000F08D8000640060000000E00006003200E6
:1091B000D0BF2B00963902000200000010412B00A6
:1091C0009639020002000000F08D80006800600007
:1091D0000000E00006003200A0C02B00963902001B
:1091E0000200000010412B0096390200020000002E
:1091F000B2F7020001000000C0C32200104F780047
:109200001E4078000004E0000500320070C12B0011
:1092100096390200020000001E407800C4FF0700DB
:1092200010C42200104F78001E4078000004E000B7
:109230000500320040C22B009639020002000000F7
:109240001E407800BAFF0700D0C32200104F7800FC
:109250001E4078000004E0000500320010C32B001F
:1092600096390200020000001E407800B0FF07009F
:10927000E0C32200104F78001E4078000004E00098
:1092800005003200E0C32B00963902000200000006
:109290001E407800A6FF070030C42200104F78005F
:1092A0001E4078000004E00005003200B0C42B002E
:1092B00096390200020000001E4078009CFF070063
:1092C00040C42200104F78001E4078000004E000E7
:1092D0000500320080C52B00963902000200000014
:1092E0001E40780092FF070050C42200104F780003
:1092F0001E4078000004E0000500320050C62B003C
:1093000096390200020000001E40780088FF070026
:1093100090C42200104F78001E4078000004E00046
:109320000500320020C72B00963902000200000021
:109330001E4078007EFF070000C42200104F780016
:109340001E4078000004E00005003200F0C72B004A
:1093500096390200020000001E40780074FF0700EA
:10936000D2C20200010000000004E0000700320049
:10937000F0C32200104F7800C0C82B0096390200BD
:10938000020000001E40780069FF070070C4220040
:10939000104F78001E4078000004E0000500320005
:1093A00090C92B0096390200020000001E40780090
:1093B0005FFF07000080FA00000006000000FA00CE
:1093C00060CA2B0096390200020000000040EB004A
:1093D000446902000000000030CD2B0096390200E5
:1093E000020000000040EB00A67C0200000000002C
:1093F00000D02B009639020002000000DCF80700C4
:1094000090942A00963902000200000059FF0700DC
:109410000080FA00000006000000FA0060CA2B007D
:10942000963902000200000010C0B3004469020037
:109430000000000030CD2B00963902000200000031
:1094400010C0B300A67C020000000000D0D22B00A8
:10945000963902000200000011C0B3000040EB008A
:109460003CF90700A0D52B0096390200020000004D
:1094700011C0B30010C0B30036F907000080FA0035
:10948000000006000200FA00004F78001E80FB007A
:10949000E20F500017003200E20F500005003C00C0
:1094A0000000E00008003200E10F50000F00320021
:1094B00019003700E30F500011003200E40F500094
:1094C0001200320014003700BCFF070045F007000F
:1094D0001E390200010000009CA3020001000000F0
:1094E00000EB0200010000000B003700B3FF070093
:1094F000090037001E390200010000000600370095
:109500009CA30200010000000300370000EB0200F2
:1095100001000000000000000080FA0000000600CA
:109520000200FA00004F78001E80FB00E20F50009E
:109530001C003200E20F500005003C000000E0007B
:1095400008003200E10F5000140032001E00370006
:10955000E30F500016003200E40F500017003200F5
:109560001900370056BC020001000000A2380200BA
:10957000010000008AEA02000100000070D82B0000
:109580009639020002000000C18D8000D08D80005D
:109590006E2A0200020000000B0037009EFF070049
:1095A00009003700EA34020001000000060037001D
:1095B0007EB902000100000003003700F8E8020055
:1095C00001000000000000000080FA00000006001A
:1095D0000800FA00204798002107980032079800F9
:1095E0008E01780022D92B00BE0090002E00900042
:1095F00064020200000000000004E0005A00320093
:109600001E4078000080FB00CF80DE009201200029
:1096100003002000820F5000838F580055003E0049
:1096200000060100190037001B0037001A00370040
:109630001C0037001B0037001D0037001F003700DB
:1096400021003700230037002500370027003700AE
:1096500026003700280037002A0037002B0037008B
:109660002A0037002B0037002A0037002900370076
:109670002C0037002B0037002A0037002D00370060
:109680003E0037003D0037003C0037002E40900080
:10969000A3FF07003A0037002E40900079FF070033
:1096A0003700370078B702000100000034003700AF
:1096B0009C3B02000100000031003700BE3D02006B
:1096C000010000002E00370066410200010000008A
:1096D0002B0037003C440200010000002800370046
:1096E000F84502000100000025003700F2470200A3
:1096F0000100000022003700DA4A020001000000E9
:109700001F00370090F107001D0037000FF207001F
:109710001B00370010C0B3004469020000000000C5
:109720001700370010C0B300A67C02000000000044
:1097300013003700D0D22B0096390200020000003F
:1097400011C0B3000040EB0082F80700A0D52B0049
:10975000963902000200000011C0B30010C0B3002F
:109760007CF8070006003700C22C0200020000004F
:109770000300370000000000010037000000000077
:109780000080FA00000006002000FA00600F980038
:10979000710F98000040EB00204798007A004700C6
:1097A0008001780042E22B00FE0890006E089000D5
:1097B00064020200000000000004E0007D003200AE
:1097C00010C0B300204798002E5890000080FB0086
:1097D000CF80DE00A200200003002000820F500096
:1097E000838F580070003E00000601000A00370019
:1097F0000F0037001700370020003700290037001E
:10980000320037003B003700440037004B00370080
:10981000520037005900370010E52B00963902003E
:10982000020000000040EB00204798007300370062
:109830006000B8002007980031079800000620005B
:1098400040079800D0E92B00963902000200000082
:109850006A0037000008200001002000200798005F
:1098600031079800400220004007980040EA2B0092
:10987000963902000200000060003700000C200052
:109880000100200020079800310798000004200004
:1098900040079800C0EA2B00963902000200000041
:1098A000560037000010200001002000200798001B
:1098B00031079800400920004007980030EB2B004A
:1098C00096390200020000004C003700001C200006
:1098D0000100200020079800310798008003200035
:1098E00040079800B0EB2B00963902000200000000
:1098F00042003700002020000100200020079800CF
:1099000031079800400120004007980030EC2B0000
:10991000963902000200000038003700E8004700D6
:10992000640047000266020001000000B0EC2B005A
:10993000963902000200000030003700E8004700BE
:10994000640047001A6602000100000030ED2B00A1
:10995000963902000200000028003700E8004700A6
:1099600064004700B6F5020001000000B0ED2B00D6
:10997000963902000200000020003700006A200033
:109980000100200020079800310798008002200085
:109990004007980020EE2B009639020002000000DC
:1099A00000000000150037000040EB002047980041
:1099B000120037006400470000017800FE089000A4
:1099C0006E08900092060200000000000004E00013
:1099D0000A0032006800470000017800FE0890008D
:1099E0006E0890000E040200000000000004E00079
:1099F0000200320010C0B300204798002E409000B3
:109A00000004E00028003200240037004E009000DF
:109A1000F00F50000300360000012000000F780016
:109A200002003700CE009000010F78002E00900059
:109A3000BE00900000007800EA0047001E01780098
:109A40003A370200020000006400470011002000C5
:109A50001C2B0200020000006A0047009E007800F4
:109A6000E62A020002000000B62C020002000000FC
:109A70004E0090001E005000400798001E00780025
:109A80006101B8002E009000BE009000020040006E
:109A90008380480020079800310798004E0090000E
:109AA0000000E000D9FF3A00B62C020002000000DE
:109AB0000080FA00000006000800FA003007980055
:109AC0000000EB00100798003E00900090407800E6
:109AD000A0C3B30080CF50000A003A001E009000DF
:109AE0000000E800100798000E80E8008000780071
:109AF0003E0090008C32020002000000D8F1B70056
:109B0000C3003700E40047000E80E80081017800C0
:109B100092EE2B00800078003E009000640202006C
:109B200000000000004F78001E4078000004E000B4
:109B3000B00032004E4090000080FB00CF80DE007D
:109B40006202200003002000820F5000838F580023
:109B5000AC003E0000060100AC00370025003700D5
:109B6000240037002900370028003700270037007D
:109B7000280037002A0037002C0037002E0037005D
:109B800030003700350037003A0037003900370021
:109B90003E0037003D0037004200370041003700EB
:109BA00046003700450037004C0037004B003700B7
:109BB0005200370051003700580037005700370077
:109BC0005E0037005D003700620037006300370039
:109BD00064003700690037006F0037008B003700E2
:109BE00073003700740037008800370074003700B6
:109BF00078003700C2D1BF008E80E80001017800F4
:109C0000BE009000A7EF070081003700C271EF008F
:109C10007F00370010C0B300C2F1B7007C003700EE
:109C200020C0B300C2F1B7007900370030C0B300E4
:109C3000C2F1B7007600370040C0B300C2F1B700F0
:109C400073003700C2D1BF008E80E80001017800A8
:109C5000BE009000B5F807006D003700C2D1BF000C
:109C60008E80E80001017800BE009000D1F8070066
:109C700067003700C2D1BF008E80E8000101780084
:109C8000BE00900052FE070061003700C2D1BF0045
:109C90008E80E80001017800BE009000C6FA07003F
:109CA0005B003700C2D1BF008E80E8000101780060
:109CB000BE00900058FA070055003700C2D1BF001F
:109CC0008E80E800810178003E019000804078009D
:109CD00010C0B300D9F807004D003700C2D1BF0053
:109CE0008E80E800810178003E019000804078007D
:109CF0000040EB00D1F8070045003700C2D1BF009B
:109D00008E80E800810178003E019000804078005C
:109D100010C0B30062F107003D003700C2D1BF00A0
:109D20008E80E800810178003E019000804078003C
:109D30000040EB005AF1070035003700C2D1BF00E8
:109D40008E80E80001017800BE00900089F20700D3
:109D50002F00370064FC07002D003700C1FC07000E
:109D60002B0037000E80E800800078003E00900055
:109D7000325A020001000000250037000E80E80082
:109D800012C0B300800078003E0090004E580200E0
:109D9000010000001E0037000E80E80080007800FF
:109DA0003E009000505702000100000018003700EC
:109DB00024F50700160037004CF5070014003700A3
:109DC0000E80E800800078003E0090006EFE0700E4
:109DD0000F0037000E80E8000041EB0080007800A3
:109DE0003E0090004E5802000100000000000000FC
:109DF00007003700F0FA2B0096390200020000003D
:109E000003003700000000000100370000000000E0
:109E10000080FA00000006003C00FA00207F980055
:109E200071022C0038000900315F78009E03B100F8
:109E300080FC2B009639020002000000D0FC2B00B1
:109E400096390200020000000E00780096390200E8
:109E500002000000F0FC2B00963902000200000016
:109E600090002C009639020002000000E0E92A0070
:109E7000963902000200000070EA2A0096390200BA
:109E800002000000A0EA2A00963902000200000049
:109E900060EB2A00963902000200000080EB2A00E5
:109EA000963902000200000060012C009639020081
:109EB000020000000E007800963902000200000047
:109EC0000080FA00000006000000FA00C2D1BF00C6
:109ED0000080FB00E20F500018003200E20F50003B
:109EE00005003C000000E00008003200E10F5000D7
:109EF0000A00320019003700E30F50000B00320057
:109F0000E40F5000110032001400370000062C004E
:109F100096390200020000001400370060062C0091
:109F2000963902000200000010003700C0062C0025
:109F300096390200020000000C00370030072C00A8
:109F400096390200020000000800370090072C003C
:109F500096390200020000000400370000082C00BF
:109F60009639020002000000000000000080FA00A4
:109F7000000006001E00FA00881F7800005F9800AD
:109F8000510F9800425F9800680047008100200050
:109F900000280200020000005E08900000407800E7
:109FA000F043B20040479800CE409000014F980027
:109FB0006000B800008FBE00DE08900000FA2F009D
:109FC0008080600000FA2F00808F50007C003A00F3
:109FD0005E089000004078006F4060005047980095
:109FE0005E4090000080FB004800DD006101B90088
:109FF000000D2A00F14F2100001F41000197490088
:10A0000070004700000178008040EB005E40900047
:10A010001A000200010000000E5890000080FB00B2
:10A02000F000470084C0B3001E0178009E0190003C
:10A03000402102000200000070004700000178008B
:10A0400011C0B3005E4090001A0002000100000041
:10A050000E5890000080FB00F000470084C0B30061
:10A060001E0178009E0190004021020002000000C5
:10A07000700047000001780021C0B3005E409000EE
:10A080001A000200010000000E5890000080FB0042
:10A09000F000470084C0B3001E0178009E019000CC
:10A0A000402102000200000070004700000178001B
:10A0B00031C0B3005E4090001A00020001000000B1
:10A0C0000E5890000080FB00F000470084C0B300F1
:10A0D0001E0178009E019000402102000200000055
:10A0E000E607020001000000604798006E40900003
:10A0F0000004E0001D003A007000470000017800F5
:10A1000041C0B3005E4090001A0002000100000050
:10A110000E5890000080FB00F000470084C0B300A0
:10A120001E0178009E019000402102000200000004
:10A13000700047000001780051C0B3005E409000FD
:10A140001A000200010000000E5890000080FB0081
:10A15000F000470084C0B3001E0178009E0190000B
:10A160004021020002000000510137006E409000C3
:10A17000E14F50004E0132006E409000E24F50001F
:10A180004B013A00700047000001780041C0B30065
:10A190005E4090001A000200010000000E5890007E
:10A1A0000080FB00F000470084C0B3001E0178006F
:10A1B0009E01900040210200020000003C01370097
:10A1C000DE08900000FC2F008080600000FC2F0063
:10A1D000808F50002F003A005E0890000040780009
:10A1E0006F406000504798005E4090000080FB0088
:10A1F0004800DD006101B900000D2C00F14F210085
:10A20000001F4100019749007000470000017800DD
:10A210008040EB005E4090009800020001000000CA
:10A220000E5890000080FB00F000470084C0B3008F
:10A230001E0178009E0190004021020002000000F3
:10A24000E607020001000000604798006E409000A1
:10A250000004E00016013A00700047000001780099
:10A2600011C0B3005E4090009800020001000000A1
:10A270000E5890000080FB00F000470084C0B3003F
:10A280001E0178009E0190004021020002000000A3
:10A29000070137005E0890006101B800001020003F
:10A2A000F1FF2F00020040008380480002032000DD
:10A2B00003002000820F5000838F5800EA003E0008
:10A2C000000601003000370037003700410037003A
:10A2D0004B003700550037005F003700690037003A
:10A2E000E3003700E2003700E1003700E00037000C
:10A2F000DF003700DE003700DD003700DC0037000C
:10A30000DB0037006A0037007D0037008700370028
:10A31000D7003700D6003700D5003700D40037000B
:10A32000D30037008C00370096003700A0003700BC
:10A33000CF003700CE003700CD003700CC0037000B
:10A34000CB003700A5003700AB003700B100370065
:10A35000B7003700BD003700C5003700C400370024
:10A36000C3003700C2003700C1003700C00037000B
:10A37000BF003700BE003700BD003700BC0037000B
:10A38000BB003700BA003700F00047006800470004
:10A390004AFF020001000000000D2000F14F2100E3
:10A3A000008FBE00B300370068004700CE58900011
:10A3B00011409800F000470068004700209A020012
:10A3C00001000000001D2000F14F2100008FBE00A1
:10A3D000A800370068004700CE5890001140980050
:10A3E000F000470068004700609B02000100000089
:10A3F000002D2000F14F2100008FBE009D0037008E
:10A4000068004700CE58900011409800F0004700C7
:10A4100068004700329C020001000000003D20005F
:10A42000F14F2100008FBE00920037006800470006
:10A43000CE58900011409800F00047006800470097
:10A44000169D020001000000004D2000F14F210088
:10A45000008FBE008700370068004700CE5890008C
:10A4600011409800F0004700680047002A9E020053
:10A4700001000000005D2000F14F2100008FBE00B0
:10A480007C00370068004700CE58900011409800CB
:10A49000F000470068004700FC9E02000100000039
:10A4A000006D2000F14F2100008FBE0071003700C9
:10A4B0007000470001C1B3002140980070004700C0
:10A4C00021C1B3003140980070044700E607020044
:10A4D0000100000040449800700047008040EB00FD
:10A4E00011409800700047008000EB003100980098
:10A4F000000D2100F14F2100008FBE005D003700EC
:10A500006800470011C1B30001487800F00047001F
:10A51000680047006C06020001000000001D2100D9
:10A52000F14F2100008FBE00520037006800470045
:10A5300021C1B30001487800F000470068004700DF
:10A54000E006020001000000002D2100F14F210073
:10A55000008FBE00470037006800470081C1B3008C
:10A5600001487800F00047006800470074070200C7
:10A5700001000000008D2100F14F2100008FBE007E
:10A580003C0037006800470091C1B30001487800E3
:10A59000F000470068004700740702000100000057
:10A5A000009D2100F14F2100008FBE0031003700D7
:10A5B00068004700A1C1B30001487800F0004700DF
:10A5C00068004700740702000100000000AD210090
:10A5D000F14F2100008FBE002600370070004700B9
:10A5E00026FE020001000000000D2200F14F2100B4
:10A5F000008FBE001F0037007000470068FE020099
:10A6000001000000001D2200F14F2100008FBE005C
:10A61000180037007000470090FE020001000000A3
:10A62000002D2200F14F2100008FBE0011003700E5
:10A6300070004700AEFE020001000000003D220055
:10A64000F14F2100008FBE000A0037007000470064
:10A650007CFE020001000000004D2200F14F2100AD
:10A66000008FBE000300370000000000010037002B
:10A67000000000001E0078009E009000E00F5000D7
:10A68000E08F58000A0032000040EB0000579800AD
:10A690000E5890000080FB00F000470084C0B3001B
:10A6A0001E0178009E01900040210200020000007F
:10A6B0001E0090001E00700000F0A7000000EA00DD
:10A6C0000000EA004F00DE00004078004F047800F0
:10A6D0000080FA00000006001600FA0000579800FB
:10A6E000110F9800425798001E0890009040780083
:10A6F00011479800680047008100200000280200F0
:10A70000020000009E409000014F98001E0890003B
:10A71000104090000080FB00C800DD001E4090004B
:10A720000080FB0000804000100798001E08900089
:10A73000A0409000414798001E089000B040900053
:10A74000514798001E089000F04090006147980023
:10A750004E4090000004E0005E00320000C0EB00BC
:10A76000004F78001E00900021F22F00810F500052
:10A770001A00320021F22F00810F500007003E0026
:10A7800001F22F00810F50000E00320011F22F0055
:10A79000810F50000E0032001C00370041F22F00E4
:10A7A000810F50001300320041F22F00810F500042
:10A7B0000D00390001F32F00810F5000100032000E
:10A7C000120037000040EB00004F78000F00370008
:10A7D00010C0B300004F78000C00370020C0B30059
:10A7E000004F78000900370030C0B300004F7800F8
:10A7F0000600370040C0B300004F78000300370068
:10A8000050C0B300004F7800000000001E407800E8
:10A81000E14F40002F00320010C0B300CDF1B7006F
:10A820005E409000E14F500010003E001E80FB0093
:10A83000F1F12200008040008040EB0001487800E8
:10A840001E80FB0081F12200008040008040EB0070
:10A85000014878001E80FB0061F222000080400069
:10A860008040EB00014878001A0037001E80FB0092
:10A87000F1F1220000804000CE40900001487800B5
:10A880001E80FB0081F1220000804000CE4090003D
:10A89000014878009E80FB005E409000E14F400040
:10A8A000030032005E4090000040E90001003700E4
:10A8B00000C0EB0062F22200810041008048780075
:10A8C0001E80FB00D1F22200008040008E509000DC
:10A8D000014878006E4190009E0090000E5090005C
:10A8E000A4FD0700704798009E00900080F12F00A3
:10A8F000808F500008003A006E41900091F12F00C7
:10A900000E5090009BFD07006E419000A1F12F00BA
:10A910000E50900097FD07007E4090000080FA00E6
:10A92000000006002A00FA00889FBE008A9FBE0031
:10A93000405F9800515F9800720F980003179800CD
:10A940001417980045679800361798004717980025
:10A9500070772300500F98000040EB00004F780004
:10A960005E5890000004E000C0003200F08D8000CE
:10A97000680060000000E0002A0032007E099000BC
:10A980008E119000800D2D00B14E2100800F5100DE
:10A99000818F59000E003A00307E2300500F98003E
:10A9A0004E6190009E1090004E5890004AFF0700A4
:10A9B0000004E00003003200A06581000000E80010
:10A9C000A065890010C0B300004F78001500370063
:10A9D0007E0990008E119000800D2D00F14E210017
:10A9E000800F5100818F59000E003A00C07E230075
:10A9F000500F98004E6190009E1090004E589000AD
:10AA000086FF0200010000000004E00003003200A5
:10AA1000A06581000000E800A065890010C0B300B7
:10AA2000004F78001E4078000004E00082003A00E9
:10AA300080C42200904078004E58900080CF500093
:10AA40000D003A007E0990008E119000000E230048
:10AA5000F14F2100800F5100818F590006003A000C
:10AA60001E109000800078004E5890004EC30200E7
:10AA700001000000004F78007E0990008E119000C8
:10AA800000002000F1FF2F0002027800030178008F
:10AA9000800178008100780003006200810061007D
:10AAA00081057800000578000A01BE000000200042
:10AAB000E11D2000800F5100818F590027003A00CE
:10AAC000FE08900000F02F00008060001007980042
:10AAD000FE08900000032000008060004400DE00BB
:10AAE000404798007E089000004078006F4060006A
:10AAF000504798009E00900000802000808F5000FA
:10AB000009003A004E5890000080FB005E41900022
:10AB1000CE409000DEFC02000000000010C0B30038
:10AB2000004F7800440037009E00900000C02000D5
:10AB3000808F500040003A004E5890000080FB008B
:10AB40005E419000CE409000B2FE02000000000086
:10AB500010C0B300004F780037003700C0C3220098
:10AB6000904078004E58900080CF500032003A005C
:10AB70007E0990008E11900000F02F00F1FF2F0051
:10AB800002027800030178008001780081007800DB
:10AB900003006200810061008104780000047800F5
:10ABA0000800BE003007980041079800FE0890009A
:10ABB000510798003E019000CE0190000040220015
:10ABC000B18E2100800F5100818F59000A003A0098
:10ABD00090782300500F98001E109000800078009D
:10ABE0005E009000187002000100000010C0B30069
:10ABF000004F7800100037003E019000CE01900019
:10AC000000002500F18F2100800F5100818F590035
:10AC100009003A0020792300500F98001E10900080
:10AC2000800078005E0090002271020001000000A8
:10AC300010C0B300004F78001E4078000004E00010
:10AC4000D8003A00CE6290001E1290007E0990005B
:10AC50008E11900011C0B3004E58900076F802009B
:10AC600001000000004F7800CE003700FE08900081
:10AC7000610798000040EB00004F780000C42200FC
:10AC8000904078004E58900080CF50000F003A005E
:10AC9000CE6190001E119000EE0090004E58900082
:10ACA000F806020002000000004F78001E40780005
:10ACB0000004E00005003200406581000000E8006B
:10ACC00040658900F07B2300500F98001E407800FB
:10ACD0000004E00014003A0010C422009040780004
:10ACE0004E58900080CF50000F003A00CE61900087
:10ACF0001E119000EE0090004E5890000686020053
:10AD000001000000004F78001E4078000004E000C1
:10AD100005003200506581000000E80050658900A0
:10AD2000107D2300500F98001E4078000004E000C2
:10AD30001A003A00D0C32200904078004E5890008C
:10AD400080CF500015003A00EE00900080102000E7
:10AD5000808F500004003200EE0090009010200020
:10AD6000808F50000D003A00CE6190001E119000BF
:10AD7000EE0090004E589000CA72020001000000E0
:10AD800010C0B300004F7800106581000000E8009B
:10AD900010658900607B2300500F98001E407800EA
:10ADA0000004E00013003A00F08D800062006000B3
:10ADB0000000E0000F0032007A0047000002780037
:10ADC000CE6190001E119000EE0090004E58900051
:10ADD000EC00020002000000004F78001E407800E6
:10ADE0000004E00003003200606581000000E8001C
:10ADF000606589001E4078000004E00014003A00FD
:10AE0000E0C32200904078004E58900080CF500060
:10AE10000F003A007A00470000027800CE619000EF
:10AE20001E119000EE0090004E589000D2040200D7
:10AE300002000000004F78001E4078000004E0008F
:10AE400003003200206581000000E80020658900D1
:10AE50001E4078000004E00013003A00F08D8000EE
:10AE6000640060000000E0000F003200807C2300DE
:10AE7000500F9800CE6190001E119000EE009000DF
:10AE80004E58900080FA020001000000004F780048
:10AE90001E4078000004E00003003200F0648100EE
:10AEA0000000E800F06489001E4078000004E00023
:10AEB0003C003A00CE6290001E1290007E09900085
:10AEC0008E1190008040EB004E58900076F8020002
:10AED00001000000004F78006E00900041522000F9
:10AEE000810F50000A003E0011522000810F5000D7
:10AEF0001F00310021212000810F50001600320078
:10AF000011512000810F50001F0032002500370032
:10AF1000015F2000810F50000900320071612000A4
:10AF2000810F50001E003A00B0792300500F9800A6
:10AF30001E1090000072020001000000190037008E
:10AF4000407A2300500F98001E10900038720200C3
:10AF50000100000013003700D07A2300500F980042
:10AF60001E1090007C720200010000000D003700EE
:10AF70001E109000800078004E58900068C50200B6
:10AF800001000000070037001E10900080007800CC
:10AF90004E58900062C4020001000000010037001A
:10AFA00000000000BCD1BF000080FB006200600018
:10AFB0000000E000430032004E589000E14F500086
:10AFC00040003A008A20020002000000604F980012
:10AFD000D9D1BF000004E00017003200D08E8000FD
:10AFE0000000E800D08E88006E489000E14F5000CD
:10AFF00034003E00CE1090003E109000EE2902007A
:10B000000200000020082C00963902000200000017
:10B01000D08E800011C0B300EE28020002000000B4
:10B0200080092C009639020002000000D971EF005F
:10B03000DA31EF00230037006E489000EF4F5000E8
:10B0400015003E0010C3B300704F980000C2B3005B
:10B05000005798005E089000EF0047008180E800EC
:10B06000920020002A280200020000006F00470022
:10B070004E6390009E1190007E0A90008E12900008
:10B0800000017800CE1090003E109000DA2C0200F3
:10B09000020000000B003700CE1090003E10900020
:10B0A000EE29020002000000B00A2C0096390200CE
:10B0B0000200000010C0B300D9F1B700100020005A
:10B0C000D08E8800BCD1BF000080FB00640060000F
:10B0D0000000E000460032004E589000E24F500061
:10B0E00043003A00801A020002000000604F9800FE
:10B0F000DCD1BF000004E000130032006E48900075
:10B10000E14F500010003E00CE1090003E10900025
:10B11000EE29020002000000300C2C0096390200DB
:10B1200002000000F08E800011C0B300EE28020083
:10B130000200000080092C00963902000200000085
:10B14000DC71EF00DE31EF00DCD1BF000004E00075
:10B1500024003A006E489000E74F500015003E0072
:10B1600020C3B300704F980000C2B300005798008E
:10B170005E089000EF0047008180E8009200200008
:10B180002A280200020000006F0047004E63900072
:10B190009E1190007E0A90008E12900000017800AF
:10B1A000CE1090003E109000DA2C02000200000049
:10B1B0000F003700CE1090003E109000EE290200E4
:10B1C00002000000900D2C009639020002000000E1
:10B1D00010C0B300DCF1B70010002000F08E880032
:10B1E00003003700F08E80000000E800F08E880039
:10B1F0004F05BE004F04BE000080FA0000000600AC
:10B200000000FA0010C0B300E4F1B700E031EF0035
:10B21000E231EF00E571EF00003A80004300DE000C
:10B2200061406000FCFA07000080FA0000000600A0
:10B230000200FA00E4D1BF000004E0000400320084
:10B24000E471EF00B62C0200020000001EFB0700B4
:10B25000265E0200000000000004E000030032004F
:10B26000B62C02000200000017FB07000E00E800E9
:10B270001E3A020002000000004F78001E407800D5
:10B280000004E00073003200865E0200000000004F
:10B290000004E00002003200D0C0B3001047980064
:10B2A000E5D1BF000004E00008003A001E40900015
:10B2B000FB4F500003003A0010C0B300E5F1B700A7
:10B2C0001B003700E571EF0019003700E5D1BF0022
:10B2D000E14F500009003A009E409000B0C5B30015
:10B2E00080CF500003003A0020C0B300E5F1B70062
:10B2F0000F003700E571EF000D003700E5D1BF000A
:10B30000E24F500009003A009E40900010C4B30084
:10B3100080CF500003003A0030C0B300E5F1B70021
:10B3200003003700E571EF0001003700E571EF0021
:10B330009E409000F0C7B30080CF50000300320061
:10B340001E409000E84F50000A003A00008F800035
:10B350000000E0003F0032001E409000583902001B
:10B3600002000000008F80000000E900008F8800CC
:10B37000380037001E409000ED4F500003003200AF
:10B380001E409000EA4F500015003A00D0C0B300B4
:10B390005839020002000000A0C0B3005839020072
:10B3A00002000000008F80000000E0000A00320070
:10B3B000008F8000108F8800008F800041F32200F2
:10B3C000008040008040EB000148780040F32200FC
:10B3D000B9F90700E031EF00BBFA07001D003700A4
:10B3E000E5D1BF000004E00011003A001E409000CB
:10B3F0005839020002000000008F80009E4090003B
:10B400000141780041F322008080400082487800AA
:10B410000000E800008F8800018F800000102000ED
:10B42000808F50000B003600E031EF00090037003C
:10B43000E5D1BF00E34F500006003A0040F3220080
:10B440009639020002000000108F8000008F8800F3
:10B45000E571EF000080FA00000006000200FA002B
:10B46000C2FB020001000000142EA900182EA90042
:10B4700010C0B300CDE607002C2EA80068E6070038
:10B4800000712200FAE70700DE5C02000000000005
:10B490005C3C020002000000D03C02000200000000
:10B4A000004F780011C0B30050052000B6380200EC
:10B4B0000200000052FF0700E85C020001000000EB
:10B4C0001E4078000004E00003003A00100F2C003A
:10B4D00096390200020000000080FA000000060019
:10B4E0000400FA0020479800CC5F02000100000031
:10B4F000004F78002E4090000004E000160032005B
:10B50000E1548000F0F32F00008060000060A00094
:10B51000E05488001E407800E14F500007003A00D8
:10B520001154800000F82F0080806000F00520009A
:10B5300001007000105488001C0037001154800076
:10B5400000F82F0080806000600220000100700081
:10B550001054880015003700E1548000F0F32F00EC
:10B56000008060000070A000E05488001E40780059
:10B57000E14F500007003A001154800000F82F00FE
:10B5800080806000E00620000100700010548800F8
:10B59000060037001154800000F82F008080600002
:10B5A0002005200001007000105488009D2AA90089
:10B5B0002248A8009DEAA8000080FA0000000600CA
:10B5C0000200FA00142EA800182EA8000040EB007C
:10B5D00076E607000E0EA9000080EB00003B880015
:10B5E0000080EB00103B88006547A9000040EB009D
:10B5F000004F78009D2AA9001C003700E15480000C
:10B6000000202000008060000000E0000800320000
:10B61000E154800000102000008060000000E00085
:10B6200003003A0010C0B300004F78000F0037004D
:10B630000040EB00AAFF07002268A8001CEEA8004B
:10B64000B170800000082000008060000000E00071
:10B6500006003A00E15480000020200000806000D5
:10B660000000E00001003A000040FE00B1708000E0
:10B6700000082000008060000000E00003003A00A5
:10B680001E4078000004E000DCFF32009D2AA90083
:10B690000F00370010C0B30091FF07002268A80018
:10B6A0001CEEA800B170800000082000008060003F
:10B6B0000000E00006003A00E15480000020200075
:10B6C000008060000000E00001003A000040FE0041
:10B6D000B170800000082000008060000000E000E1
:10B6E00005003A00E1548000002020000080600046
:10B6F0000000E000E7FF32006027EF006227EF0064
:10B700006547A9000080FA00000006000200FA0068
:10B71000411C210091407800014F780010C0B30017
:10B72000C4F1B700707F020000000000A25D0200BB
:10B7300000000000408E80000000E00004003A009D
:10B740008E1802000200000010002000408E8800C9
:10B7500010C0B300ECE507009E407800421C2100B9
:10B76000014978000080FA00000006001400FA0089
:10B77000881F780035E6070038FF07000040EB001F
:10B7800040ED07000040EB004BEE0700BC71EF00FE
:10B79000D871EF00C271EF00F085020001000000D7
:10B7A0000004E0000A00320020012000F077890048
:10B7B00020012000007889002001200010788900F5
:10B7C00020012000207889000100370000000000DF
:10B7D00010C0B300C4F1B700CCFF070010C0B30025
:10B7E000C9E5070020C0B300C4F1B700105E020035
:10B7F0000100000020C0B300C3E5070070C0B30023
:10B80000C4F1B7008AFE070070C0B300BEE50700B0
:10B81000C18D80001E009000808F50000800320013
:10B8200030C0B300C4F1B700E0C002000100000066
:10B8300030C0B300B4E50700C18D80001107980047
:10B8400060C0B300C4F1B700A05E020000000000B9
:10B8500060C0B300ACE5070090C0B300C4F1B7000E
:10B8600060F202000100000090C0B300A6E50700EE
:10B8700080C0B300C4F1B70014ED07000040EB0036
:10B88000004F780010003700C28D8000D58D8000F9
:10B890002E5290003E009000CE0090004E4490004A
:10B8A000EA014700820378000503780084427800AB
:10B8B000030278000001BE008840780010C0B30089
:10B8C00018FC07001E4FE8001E407800E14F5000B2
:10B8D00008003E00F20147006A014700E600470009
:10B8E00064004700D81B0200020000000004E000D2
:10B8F000E5FF3A000040EB00004F780010003700F1
:10B90000C28D8000D58D80002E5290003E009000A8
:10B91000CE0090004E449000EA0147008203780078
:10B920000503780084427800030278000001BE001D
:10B930008840780020C0B300FAFB07001E4FE800E3
:10B940001E407800E14F500008003E00F201470021
:10B950006A014700E6004700640047006E160200D7
:10B96000020000000004E000E5FF3A0080C0B300E0
:10B9700065E50700318E8000F00F2000808F5000B9
:10B9800092FF3E00C3D1BF000080FB00F801B90068
:10B990008200780076814000C1CB22008100410006
:10B9A000910078008100E800F801B90020CD220064
:10B9B000000041000108780085FF37000200FA000E
:10B9C0002143A80001198000F0CF2F000080600003
:10B9D0000019880001198000000E2000010070008D
:10B9E000001988002083A9002043A90011198000B4
:10B9F000F0FF2100008060001019880000C0EB00FB
:10BA000024E3B70021E3A8000040EB00004F7800DA
:10BA1000070037001E80FB008000400080BE23002E
:10BA2000008040008000EB00010878001E4FE80015
:10BA30001E407800E64F5000F6FF360060C0B300AD
:10BA400027F2B70027D2BF000080FB0081C62E007E
:10BA50000080400010407800F043B2008080FB007E
:10BA6000F0032000008060004219800001FC2F00DC
:10BA70008100610001007000401988002003A900C6
:10BA80002023A80010C0B30026F2B7002003200036
:10BA9000109188002832EF002432EF002F72EF005F
:10BAA0002A72EF002C32EF002E72EF000080FA00B5
:10BAB000000006000000FA00109180000000E00085
:10BAC00003003200109180000000E900109188000E
:10BAD000209180000000E0000300320020918000EF
:10BAE0000000E90020918800609180000000E000E3
:10BAF00009003200609180000000E9006091880038
:10BB0000609180000000E00003003A002A72EF001C
:10BB100010C0B3002EF2B7000080FA00000006004B
:10BB20000000FA001091800000F0A7000000EA0079
:10BB30000000E9004F00DE00004078000080FA00BD
:10BB4000000006000000FA0026D2BF000004E0005A
:10BB50003500320000198000610060000000E00044
:10BB6000380032002672EF0027D2BF000080FB00B1
:10BB7000011880000001400080BE23000000410049
:10BB80000108780027D2BF000080FB0011002000D0
:10BB90000008DD0080007800409180000100700006
:10BBA0004091880027D2BF00E64F500002003A00C3
:10BBB00010C0B3002FF2B70027D2BF000040E8004A
:10BBC00027F2B70027D2BF00E64F50000200360030
:10BBD00010C0B30027F2B70027D2BF000080FB00DF
:10BBE00081C62E000080400010407800F043B20073
:10BBF0008080FB00F003200000806000421980007C
:10BC000001FC2F00810061000100700040198800D4
:10BC1000109180000000E0000A003A0010002000AF
:10BC20002091880007003700209180000000E0008C
:10BC300004003A002003A9002023A80010C0B3008C
:10BC400026F2B7000080FA00000006000200FA00A9
:10BC5000E122210091407800014F78002E72EF0020
:10BC60001E4078000080FA00000006000400FA0080
:10BC700020479800314798000040EB00004F7800C3
:10BC80002E4090000004E000090032002E40900099
:10BC9000E84F500006003E002E419000A1222100F6
:10BCA0008248780010C0B300004F780014003700BD
:10BCB0003E4090000004E000110032003E40900041
:10BCC000EE4F50000E003E003E4090000080FB0012
:10BCD00061C2230000804000904078002147980016
:10BCE0002E4090000004E00005003200AE409000BD
:10BCF000A22221000149780010C0B300004F780053
:10BD00001E4078000080FA00000006000200FA00E1
:10BD10000040EB00004F78002AD2BF000004E00092
:10BD2000040032002A72EF002C32EF0010C0B30082
:10BD3000004F78001E4078000080FA0000000600E6
:10BD40000200FA002AD2BF000004E0001B0032000B
:10BD5000A122210091407800014F78001E40780018
:10BD6000E64F50000200360010C0B300004F7800CC
:10BD70001E80FB00110020000008DD00800078001C
:10BD800040918000008060000000E0000B00320065
:10BD90002AD2BF0011C0B300690407001E80FB0057
:10BDA000110020000008DD000080EA00800078001B
:10BDB0004091800000806000409188000080FA007F
:10BDC000000006000200FA00F122210091407800F4
:10BDD000014F78002F72EF001E4078000080FA00BB
:10BDE000000006000400FA00204798003147980040
:10BDF0000040EB00104798000040EB00004F780037
:10BE00003E4090000080FB00ED0F500011003E000E
:10BE1000110020000008DD00414C2000810060007E
:10BE20000100E00005003A008100230001006000ED
:10BE30000000E00004003A000700370010C0B30023
:10BE4000104798000400370010C0B300004F78007E
:10BE500001003700000000002E4090000080FB0031
:10BE6000E20F500022003200E20F500003003C00BD
:10BE7000E10F50000600320065003700E30F50006C
:10BE800033003200E40F50004900320060003700F8
:10BE90001E4090000080FB000000EA004F00DE0022
:10BEA000004078000080FB00610060004800DD0079
:10BEB000017180000180A100010070000071880004
:10BEC0001E80FB000000EA004F00DE00004078000A
:10BED0000080FB00610060004800DD00F170800020
:10BEE0000180A10001007000F07088004800370058
:10BEF0001E4090000080FB000000EA004F00DE00C2
:10BF0000004078000080FB00610060004900DD0017
:10BF1000017180000190A100010070000071880093
:10BF20001E80FB000000EA004F00DE0000407800A9
:10BF30000080FB00610060004900DD00F1708000BE
:10BF40000190A10001007000F070880030003700FF
:10BF50001E4090000080FB000000EA004F00DE0061
:10BF6000004078000080FB00610060004600DD00BA
:10BF7000A17180000160A10001007000A071880023
:10BF80001E80FB000000EA004F00DE000040780049
:10BF90000080FB00610060004600DD0091718000C0
:10BFA0000160A10001007000907188001800370046
:10BFB0001E4090000080FB000000EA004F00DE0001
:10BFC000004078000080FB00610060004700DD0059
:10BFD000A17180000170A10001007000A0718800B3
:10BFE0001E80FB000000EA004F00DE0000407800E9
:10BFF0000080FB00610060004700DD00917180005F
:10C000000170A10001007000907188000000000024
:10C010000080FA00000006000400FA0020479800A3
:10C020002E4090000004E00016003A0040C12300BA
:10C030002201200080007800000220003A37020030
:10C040000200000010C0B300004F78000A00370063
:10C050001E80FB008000400040C1230000804000A3
:10C0600010407800EE4F50000200360010C0B300C0
:10C07000204798001E4FE8001E407800E94F50000E
:10C08000F3FF360000C2230081C0B30001487800EE
:10C0900020C22300B1C0B3000148780040C2230091
:10C0A00091C0B300014878002E4090000004E000E9
:10C0B0001800320010C0B300004F78000C003700A9
:10C0C0001E80FB0001CA2E000080400090407800D6
:10C0D000114798001E80FB008000400040C12300F3
:10C0E000008040009E409000014878001E4FE8000C
:10C0F0001E407800E94F5000F1FF360040C1230098
:10C100002201200080007800000220002038020078
:10C110000200000060C22300F1002000002802009D
:10C120000200000010C0B300004F78001900370073
:10C130001E80FB008000400040C1230000804000C2
:10C1400090407800114798001E4090000004E000E5
:10C150000C0032001E409000EE4F500009003E00DF
:10C160001E4090000080FB0061C223000080400060
:10C170001E4878009E4090001E40780019FF07007E
:10C18000030037008040EB001E40780015FF0700D9
:10C190001E4FE8001E407800E84F5000E4FF3600D4
:10C1A0000080FA00000006000A00FA0060479800CC
:10C1B000410798006E409000E84F50002D003E006F
:10C1C00041C123006E4090000080FB000000400051
:10C1D0000080400010079800CE00900021079800D2
:10C1E00020C0B300004F78006E4090009E80FB009E
:10C1F0008088B900104798001B0037001E0090008F
:10C20000904078002E0090001040780080CF5000C1
:10C21000110032002E009000904078001E409000E7
:10C220000080FB000002B0007E3802000200000027
:10C230002E009000904078001E0090000148780089
:10C240001E0090000000E800100798002E009000EB
:10C250000000E800200798001E4090000040E80021
:10C26000104798001E4FE9001E4078000004E000CF
:10C27000E2FF3A000080FA00000006000600FA0023
:10C2800040479800514798000040EB002047980035
:10C290004E409000E84F5000020036000040EB0096
:10C2A000404798005E409000EE4F5000020036007C
:10C2B0000040EB00504798004E4090000080FB008B
:10C2C0008000400040C1230000804000104F7800F3
:10C2D0001E4078000004E000140032001E80FB00C5
:10C2E00061C2230000804000904078001147980010
:10C2F0001E4090000004E000070032000E80E800BD
:10C30000800078001E409000A7FF07008040EB00EF
:10C310001E409000B3FE07001E80FB0061C2230098
:10C32000008040008040EB00014878005E409000B3
:10C330000080FB0061C22300008040009040780034
:10C34000114798001E4090000004E00012003200E7
:10C350001E4090000080FB008000400040C1230090
:10C3600000804000104F78001E4078000004E0007C
:10C37000040032000E80E800800078001E4090002B
:10C3800089FF07001E80FB0061C22300008040007F
:10C390008040EB00014878004E4090000004E0002F
:10C3A00009003200DE409000214798000E80E8002E
:10C3B000800078004E4090007BFF0700DE40900038
:10C3C0004E40900087FE07005E4090000004E000B1
:10C3D000060032005E4090000080FB0061C2230036
:10C3E00000804000CE409000014878000080FA00B4
:10C3F000000006000200FA00004F78001E80FB00DB
:10C40000E40F50001E003200E40F500007003C0013
:10C41000E20F500012003200E20F500014003C0006
:10C42000E10F50000A00320029003700E60F5000EB
:10C430001B003200E60F500015003500E70F5000DA
:10C440001B003200E80F50001D00320020003700B2
:10C4500020D02E0096390200020000002000370094
:10C4600080D02E0096390200020000001C00370028
:10C47000E0D02E00963902000200000018003700BC
:10C4800040D12E009639020002000000140037004F
:10C49000A0D12E00963902000200000010003700E3
:10C4A00000D22E0096390200020000000C00370076
:10C4B00060D22E009639020002000000080037000A
:10C4C000C0D22E009639020002000000040037009E
:10C4D00020D32E0096390200020000000000000068
:10C4E0000080FA00000006000200FA00004F780009
:10C4F0001E80FB006101B9000080EB008080EB0032
:10C500000200400083804800D20020000300200089
:10C51000820F5000838F580047003E000006010044
:10C520001100370014003700170037001A003700D9
:10C530001D003700080037001F00370022003700B9
:10C5400025003700280037002B0037002E00370069
:10C55000310037003400370080D32E0096390200B6
:10C56000020000003800370010D42E009639020077
:10C570000200000034003700A0D42E0096390200DB
:10C58000020000003000370030D52E00963902003E
:10C59000020000002C003700C0D52E0096390200A2
:10C5A000020000002800370050D62E009639020005
:10C5B0000200000024003700E0D62E009639020069
:10C5C000020000002000370070D72E0096390200CC
:10C5D000020000001C00370000D82E00963902002F
:10C5E000020000001800370090D82E009639020093
:10C5F000020000001400370020D92E0096390200F6
:10C600000200000010003700B0D92E009639020059
:10C61000020000000C00370040DA2E0096390200BC
:10C620000200000008003700D0DA2E009639020020
:10C63000020000000400370060DB2E009639020083
:10C6400002000000000000000080FA000000060068
:10C650000400FA00000F7800110798001E009000F7
:10C66000E10F500004003A00F0DB2E009639020082
:10C67000020000000300370080DC2E009639020023
:10C68000020000000080FA00000006000E00FA0020
:10C690004007980051079800424F98004E4890007C
:10C6A0000080FB008000400000C72E00008040009A
:10C6B000900078002107980066004700800178000C
:10C6C00052DD2E00DE0090004E0090006402020059
:10C6D000000000000004E000C10032006E40900045
:10C6E0000004E00023003A0020E22E009639020008
:10C6F00002000000A0E22E009639020002000000B5
:10C700004E4890000080FB0011C0B300EE280200EC
:10C710000200000030E32E00963902000200000003
:10C720004E489000E44F50000B003E0060E32E00A6
:10C7300096390200020000000E8B0200010000008A
:10C740000004E00007003200C0E52E009639020028
:10C75000020000000300370090E62E009639020028
:10C760000200000060E72E0096390200020000007F
:10C770009D0037000040EB00004F78000040EB00C8
:10C78000104798006E4090000080FB00CF80DE00D4
:10C79000C200200003002000820F5000838F580049
:10C7A0004A003E00000601004A0037000B00370037
:10C7B0000F00370013003700170037001B00370049
:10C7C0001F00370023003700270037002B003700F9
:10C7D0002F00370033003700370037000040EB00F0
:10C7E000004F780050C3B300104798003A0037005C
:10C7F00060C0B300004F780050C3B30010479800EA
:10C800003500370010C0B300004F780050C3B300AC
:10C81000104798003000370020C0B300004F780068
:10C8200040C0B300104798002B00370030C0B30061
:10C83000004F780040C0B300104798002600370032
:10C8400040C0B300004F780040C0B30010479800CC
:10C850002100370050C0B300004F780040C0B30043
:10C86000104798001C00370070C0B300004F7800DC
:10C8700050C3B3001047980017003700A0C0B300A2
:10C88000004F780050C0B3001047980012003700E6
:10C89000C0C0B300004F780050C3B30010479800E9
:10C8A0000D003700D0C0B300004F780050C3B30074
:10C8B0001047980008003700E0C0B300004F780030
:10C8C00050C3B30010479800030037000000000079
:10C8D00001003700000000000040EB0020479800F6
:10C8E0002E009000E10F500009003A001E40900019
:10C8F0000080FB0061006000004078000004E00060
:10C900002400320010C0B3002047980021003700F7
:10C910002E009000E20F500008003A001E409000E8
:10C920000080FB00640060000000E000190032009D
:10C9300010C0B30020479800160037002E0090006A
:10C94000E30F500008003A001E4090000080FB00FA
:10C95000700060000000E0000E00320010C0B30064
:10C96000204798000B0037002E009000E40F500085
:10C9700008003A001E4090008080FB00000220006A
:10C98000008060000000E0000200320010C0B30030
:10C99000204798002E4090000004E000070032007D
:10C9A0009E4078004E48900034FE07008040EB0027
:10C9B0004E489000620107000B003700B0EA2E00DD
:10C9C00096390200020000001E407800C6FE0700F3
:10C9D00000ED2E0096390200020000000200370030
:10C9E000C22C0200020000000080FA0000000600D5
:10C9F0000400FA00004F7800110798001E407800EC
:10CA0000E84F500007003E001E80FB008000400001
:10CA100040C1230000804000904078001E0090003C
:10CA2000014878000080FA00000006000600FA00C5
:10CA300020479800210798000040EB00004F780045
:10CA40002E409000EE4F50000D003E002E40900012
:10CA50000080FB0061C2230000804000904078000D
:10CA60002E009000014878002E00900010407800C1
:10CA70000080FB000000EA004F00DE00004F78005D
:10CA80001E4078000080FA00000006000800FA004E
:10CA9000300798003E0090008000EB0082382100B3
:10CAA0008289B900E002B9008401780003014100E5
:10CAB000833821000300B8000101410082007800A2
:10CAC000008FBE001E0078009E0090004409DD002B
:10CAD0004C00DE0000007100CC08DE00200798004A
:10CAE0002E0090000080FA00000006000400FA000A
:10CAF000204798000000EB00000F78002E409000C7
:10CB0000E84F500006003E002E4090000080FB00E1
:10CB10008000400000C72E0000804000100F780009
:10CB20001E0078000080FA00000006000400FA00F1
:10CB3000204798002E409000E64F500007003E002E
:10CB40002E4090000080FB008000400080BE23004B
:10CB500000804000100F7800020037000000EB005A
:10CB6000000F78001E0078000080FA000000060028
:10CB70000400FA00204798002E409000E64F500035
:10CB800009003E002E4090000080FB008000400025
:10CB900080BE23000080400010007800BBFF07002B
:10CBA000000F7800020037000000EB00000F780053
:10CBB0001E0078000080FA00000006000A00FA005B
:10CBC000004F98000E4890000080FB00800040005D
:10CBD00000C72E00008040009000780021079800D8
:10CBE0000E489000E2FF0700300798002E009000EA
:10CBF000E30F500003003A0080382100000F780056
:10CC0000080037002E009000E40F500003003A00A7
:10CC1000802A2000000F7800020037000000EB009F
:10CC2000000F7800BE00900040192100808F500056
:10CC3000030036000080EB00100798001400370056
:10CC40001E0078006101B8003E0090008000EB00FB
:10CC5000809AB900828BB9008602780005024200F2
:10CC60000010B80001024200840078003E019000EC
:10CC70008001EB00843821000500200002015200F1
:10CC800083815A002C110200000000001007980058
:10CC90001E0090000080FA00000006000A00FA0062
:10CCA000004F98000040EB00004F78000E489000C5
:10CCB000E84F500030003E000E4890000080FB001E
:10CCC0008000400000C72E000080400090007800E7
:10CCD000110798001E009000E20F50000B003A0070
:10CCE0000E489000A2FF07002007980010C0B30074
:10CCF0002E019000419C2000810F510001003E0058
:10CD00000040EB00004F78001B0037001E00900031
:10CD1000E30F5000030032001E009000E40F5000AB
:10CD20000B003A000E489000A4FF0700300798005F
:10CD300010C0B3003E019000311F2000810F510050
:10CD4000010036000040EB00004F78000A00370079
:10CD50001E009000E10F500007003A000E489000BE
:10CD6000E84F500004003A00B07080004700DE0039
:10CD700061406000004F78001E4078000080FA009B
:10CD8000000006000600FA002047980021079800DE
:10CD90000040EB00004F78002E0090008040EB0038
:10CDA000014878000E00E800800078002E409000D6
:10CDB0001EFF07000004E0000600320010C0B300B0
:10CDC000004F78001E409000B4FF0700AE009000B6
:10CDD000804878001E4078000080FA0000000600BD
:10CDE0000600FA0020479800210798000040EB0059
:10CDF000004F78002E0090008000EB0001087800C2
:10CE00000E00E800800078002E40900007FF070029
:10CE10000004E000060032001E40900054FF0700AE
:10CE2000AE0090008008780010C0B300004F78007A
:10CE30001E4078000080FA00000006000600FA009C
:10CE400020479800210798000040EB00004F780031
:10CE50002E0090008000EB00010878000E00E80032
:10CE6000800078002E409000F0FE07000004E000F3
:10CE7000060032001E40900050FF0700AE009000F8
:10CE80008008780010C0B300004F78001E40780082
:10CE90000080FA00000006000200FA00B170800075
:10CEA000000820000080600000F0A7000000EA00F9
:10CEB0000000EA004F00DE00004F78001E407800BE
:10CEC0000080FA00000006000400FA00000F78005D
:10CED000110798001E0090000000E00004003200DE
:10CEE00030ED2E00963902000200000003003700EA
:10CEF00060ED2E0096390200020000000080FA006A
:10CF0000000006000400FA00000F780011079800E6
:10CF10001E0090000000E0000400320060ED2E00D2
:10CF200096390200020000000300370030ED2E00A9
:10CF300096390200020000000080FA00000006009E
:10CF40000E00FA00404F9800514F98004E48900054
:10CF5000E84F5000CA003E004E4890000080FB00A1
:10CF60008000400040C1230000804000104F780046
:10CF70004E4890000080FB008000400000C72E005B
:10CF80000080400090007800110798004E48900003
:10CF9000E54F500003003E001E4078000004E00012
:10CFA00003003A005E4890000004E000B400320044
:10CFB000D0ED2E0096390200020000004E4890008D
:10CFC0000CFD07005E4890000004E000770032008E
:10CFD0001E009000E10F500015003A004E489000EE
:10CFE0002EFF07000080FB004007980000EE2E0097
:10CFF00096390200020000004E0090000000E000A0
:10D000000400320050EE2E009639020002000000AB
:10D010000300370070EE2E00963902000200000077
:10D0200090EE2E00963902000200000062003700E8
:10D030001E009000E20F500012003A004E4890008F
:10D04000BAFE070091FE070040079800D0EE2E00C0
:10D050009639020002000000CE009000D0CC2C00D7
:10D060000008B8004308DE0011C0B300B029020078
:10D0700002000000F0EE2E009639020002000000CF
:10D080004D0037001E009000E30F500003003200F7
:10D090001E009000E40F500029003A004E48900016
:10D0A000C6FE0700400798004E009000E10F4000C8
:10D0B00004003A0030EF2E00963902000200000012
:10D0C0003D003700CE009000703E2000808F500061
:10D0D0000B003E00D0ED2E00963902000200000049
:10D0E0004E00900031C0B300EE28020002000000A4
:10D0F000C0EF2E0096390200020000002E0037001B
:10D10000D0EE2E0096390200020000004E00900082
:10D110002003B000C200DE00B04721000008B800C4
:10D120000100D10021C0B3007629020002000000F6
:10D1300000F02E0096390200020000001E003700A9
:10D140001E009000E60F500014003A0068004700EF
:10D150004EB90200010000000004E0000B003200A4
:10D16000D0EE2E0096390200020000004E00900022
:10D1700031C0B300EE2802000200000040F02E0093
:10D1800096390200020000000B00370090F02E00DC
:10D1900096390200020000000700370060DB2E0015
:10D1A000963902000200000003003700E0F12E0073
:10D1B00096390200020000004E4890000080FB00FB
:10D1C0008000400040C1230000804000104F7800E4
:10D1D0004E489000E54F500026003E001E4078006B
:10D1E0000004E000230032001E407800BEFC07006F
:10D1F0005E4890000004E0001E0032001E80FB002C
:10D200008000400020C82E00008040009000780080
:10D21000210798002E009000E10F500007003A000F
:10D220006A004700800078001E407800D5FE0700A5
:10D230002E4890000080FB00400798001E80FB00F5
:10D240008000400060BF2300008040009000780014
:10D25000310798003E0090000000E0000500320019
:10D260004E0090003E019000800078001E0090006B
:10D270000200010000ED2E009639020002000000BD
:10D280000080FA00000006000400FA002047980021
:10D2900010C0B300004F780004003700AE4090008B
:10D2A0001E40780026FF07001E4FE8001E40780051
:10D2B000E84F5000F9FF36000080FA000000060039
:10D2C0000600FA00404798004E409000E64F50009C
:10D2D0001E003E0061C323004E4090000080FB0012
:10D2E0004300DD00008040001007980080C0B300BC
:10D2F000004F78004E4090009E80FB008088B9006F
:10D30000104798000E0037001E00900090407800F3
:10D310001E4090000080FB00001CB0007E38020020
:10D32000020000001E0090000000E80010079800B6
:10D330001E4090000040E800104798001E4FE90092
:10D340001E4078000004E000EFFF3A000080FA0081
:10D35000000006000600FA00404798004E4090008A
:10D36000EF4F50001E003E00E1C623004E409000EB
:10D370000080FB0000004000008040001007980083
:10D3800020C0B300004F78004E4090009E80FB000C
:10D390008088B900104798000E0037001E009000EA
:10D3A000904078001E4090000080FB000004B00018
:10D3B0007E380200020000001E0090000000E8001D
:10D3C000100798001E4090000040E80010479800A9
:10D3D0001E4FE9001E4078000004E000EFFF3A0015
:10D3E0000080FA00000006000200FA00004F7800FA
:10D3F0001E407800E14F500005003A0001ECA90002
:10D4000063ECA900662CEF0001ECA8000F003700C8
:10D410001E407800E24F500005003A0001ECA900E0
:10D4200043CCA900462CEF0001ECA8000700370010
:10D430001E407800E34F500004003A0001ECA900C0
:10D4400023CCA900262CEF0001ECA8000080FA00F4
:10D45000000006000400FA002047980010C0B30046
:10D46000004F78002E409000E14F500006003A0037
:10D4700001ECA90063ECA80063ACA800662CEF00E7
:10D4800001ECA800140037002E409000E24F50003D
:10D4900006003A0001ECA90043CCA800438CA80088
:10D4A000462CEF0001ECA8000B0037002E40900046
:10D4B000E34F500006003A0001ECA90023CCA8007D
:10D4C000238CA800262CEF0001ECA80002003700F6
:10D4D0000040EB00004F78001E4078000080FA000A
:10D4E000000006000600FA00204798002107980077
:10D4F0002E4090000080FB0080004000E0C623002A
:10D5000000804000104F7800AE009000F0FF230034
:10D51000808F500002003600F0FF230020079800A3
:10D520002E4090000080FB0080004000E0C62300F9
:10D530000080400010409000E34F500011003A007E
:10D540001E407800E14F500003003A00AE0090000A
:10D55000316388000B0037001E407800E24F500016
:10D5600003003A00AE0090003162880005003700E9
:10D570001E407800E34F500002003A00AE009000D9
:10D58000316188000040EB000080FA0000000600D6
:10D590000400FA0020479800314798003E40900070
:10D5A0000080FB004600DD00000F78009E00780040
:10D5B0002E409000CBFF07000080FA00000006001C
:10D5C0000600FA0020479800210798000040EB0071
:10D5D000004F78002E0090008000EB0001087800DA
:10D5E0002E4090000080FB0080004000E0C6230039
:10D5F0000080400090407800114798002E40900035
:10D600000080FB0080004000E0C623000080400056
:10D6100010409000E34F50001A003A001E40900066
:10D62000E14F500006003A00316380002E00900068
:10D630000108780010C0B300004F780011003700D7
:10D640001E409000E24F500006003A003162800018
:10D650002E0090000108780010C0B300004F780041
:10D66000080037001E409000E34F500005003A00CC
:10D67000316180002E0090000108780010C0B300D6
:10D68000004F78001E4078000080FA00000006007D
:10D690000800FA0040479800310798003E009000CB
:10D6A0008040EB00014878000E80E80080007800A0
:10D6B0004E409000C2FF0700004F78001E407800E7
:10D6C0000004E000050032001E0090004600DE006D
:10D6D000804078003E009000014878001E407800AD
:10D6E0000080FA00000006000000FA0010C0B3003D
:10D6F0003DFF070020C0B3003BFF070030C0B30070
:10D7000039FF07000080FA00000006000200FA005E
:10D7100010C0B300004F78000E0037001E80FB00E1
:10D7200080004000E0C623000080400010409000D0
:10D73000E34F500006003A001E80FB0080004000CE
:10D74000E0C62300008040001040780041FF070041
:10D750001E4FE8001E407800EF4F5000EFFF3600EC
:10D760000080FA00000006000600FA00404798001A
:10D770004E4090000004E0002D003A00E0C6230077
:10D780000202200080007800000420003A370200E6
:10D790000200000060C323008203200080007800A4
:10D7A000001C20003A3702000200000010C0B30045
:10D7B000004F7800150037001E80FB0080004000FD
:10D7C000E0C6230000804000904078001147980098
:10D7D0001E80FB0080004000E0C623000080400067
:10D7E00090409000214798001E409000E64F500066
:10D7F00003003E002E409000E44F5000020036002F
:10D8000010C0B300404798001E4FE8001E4078004B
:10D81000EF4F5000E8FF360020C8230061C0B3007E
:10D820000148780030C8230041C0B30001487800A7
:10D830004E4090000004E0004B00320010C0B300E6
:10D84000E9FE070020C0B300E7FE070030C0B300C8
:10D85000E5FE0700E0C623000102200000280200C8
:10D860000200000060C323008103200000280200A2
:10D87000020000000040EB00004F78001700370066
:10D880001E80FB009E80FB0001814000A1CA2E008B
:10D89000810041009140900000014000E0C623005B
:10D8A00000004100114098001E80FB009E80FB009C
:10D8B00001814000A1CA2E00810041009140780002
:10D8C00000014000E0C6230000004100014878004C
:10D8D0001E4078009FFE07001E4FE8001E407800A3
:10D8E000EF4F5000E6FF36000040EB00004F78009D
:10D8F0001A0037001E81FB001E80FB00C300DD0004
:10D90000A0CC2E0000804000900090001000780015
:10D91000C311DD0062C32300028141000089BE0003
:10D920001E81FB001E80FB004300DD00E400400080
:10D93000A0CC2E00008040009000900010007800E5
:10D94000C311DD00A2C32300028141000089BE0093
:10D950001E4078005AFE07001E4FE8001E40780067
:10D96000E64F5000E3FF360010C0B300004F7800D0
:10D970000E0037001E80FB0080004000E0C6230040
:10D980000080400010409000E34F500006003A0035
:10D990001E80FB0080004000E0C6230000804000A5
:10D9A00010407800ABFE07001E4FE8001E407800D4
:10D9B000EF4F5000EFFF36000080FA000000060035
:10D9C0001000FA004047980051479800320798002D
:10D9D0004407980055079800660798007707980055
:10D9E0000040EB001047980010C0B300004F7800D3
:10D9F0001D0037001E80FB0080004000E0C62300B1
:10DA000000804000904078004E40900080CF500051
:10DA100014003A005E4090009E40780080CF500095
:10DA2000100032001E80FB0080004000E0C6230092
:10DA3000008040008040EB00014878001E80FB0021
:10DA400080004000E0C62300008040008040EB00E2
:10DA5000114098001E4078003EFE0700CE40900026
:10DA6000114798001E4FE8001E407800EF4F50000D
:10DA7000E0FF36005E4090000080FB008000400028
:10DA8000E0C6230000804000104178002247980043
:10DA90002E4090000004E00014003200AE409000E0
:10DAA0004E40900080CF5000100032005E40900049
:10DAB0000080FB0080004000E0C6230000804000A2
:10DAC0008040EB00014878005E4090000080FB0041
:10DAD00080004000E0C62300008040008040EB0052
:10DAE00011409800AE419000134798001E409000EE
:10DAF0000004E000190032003E009000E30F5000E7
:10DB000003003A001E40900037FE07000300370074
:10DB10008040EB001E409000FE0207001E40900077
:10DB20000080FB00C300DD0060C3230000814000D3
:10DB30006000B8000089BE001E4090000080FB001D
:10DB4000C300DD00A0C32300008140006000B800D6
:10DB50000089BE001E409000D9FD07005E40900085
:10DB60000080FB0080004000E0C6230000804000F1
:10DB7000CE409000014878005E4090000080FB009D
:10DB8000BE0090008140780000014000E0C6230004
:10DB900000004100114098005E409000EDFD07003C
:10DBA0004E4090000080FB00C300DD0060C32300F6
:10DBB000008040004E019000DE0190000288BE000F
:10DBC0004E4090000080FB00C300DD00A0C3230096
:10DBD000008040006E019000FE0190000288BE00AF
:10DBE0004E409000B6FD07005E409000E84F5000A8
:10DBF000030032005E409000E94F50000A003A00F6
:10DC000030002000300798004E40900011FE0700C1
:10DC10000004E0000E003A0060F22E009639020087
:10DC2000020000000A0037005E409000E14F500003
:10DC300004003A0011C0B3004E409000B502070046
:10DC4000030037008040EB004E409000B102070017
:10DC50000080FA00000006001800FA00100F98007B
:10DC6000210F9800625798000040EB00004F7800A9
:10DC70000000EB005007980070004700800178001A
:10DC800012F62E00AE0890001E08900064020200FA
:10DC9000000000000004E000BF0032000E509000C1
:10DCA0000004E00040003A00F0F92E00963902002E
:10DCB000020000006E5090000080FB0011C0B30015
:10DCC000EE2802000200000000FB2E009639020040
:10DCD0000200000060FD2E009639020002000000E4
:10DCE0006E509000E34F500003003E00B0FF2E0046
:10DCF00096390200020000000E8B020001000000B5
:10DD00000004E0000300320080002F00963902007A
:10DD10000200000050012F009639020002000000AE
:10DD200030022F00963902000200000030052F005B
:10DD3000963902000200000050092F0096390200B7
:10DD400002000000B00E2F00963902000200000011
:10DD5000700F2F00963902000200000060132F00A0
:10DD60009639020002000000C0172F009639020009
:10DD700002000000601B2F00963902000200000024
:10DD8000101F2F009639020002000000C0232F0050
:10DD9000963902000200000080282F009639020008
:10DDA00002000000280237000E5090000080FB00A7
:10DDB0006101B9000080EB008080EB0002004000B0
:10DDC000838048009200200003002000820F500052
:10DDD000838F58001B023E00000601000900370037
:10DDE0000F00370026003700170037001D003700EE
:10DDF0002300370022003700450037004E0037006F
:10DE0000570037006033B8006022B8000001EB0013
:10DE10008040EB006E509000E9FE07000A023700D8
:10DE20006033B8006022B8001200200011C0B300B7
:10DE30006E509000E2FE070011C0B30010C0B300A6
:10DE400015030700000237006033B8006022B800F5
:10DE50001200200061C0B3006E509000D8FE070091
:10DE6000F90137006033B8006022B80012002000CA
:10DE700071C0B3006E509000D1FE0700F201370070
:10DE80000E509000E34F500003003A0080C0B300F2
:10DE9000004F7800080037000E509000E64F500009
:10DEA00003003A0090C0B300004F78000200370032
:10DEB00020C0B300004F78006E509000E14F50003A
:10DEC000060032006E509000E24F50000300320016
:10DED0006E509000E34F500009003A006033B800E4
:10DEE0006022B800320020009E4078006E50900002
:10DEF000B3FE07006E50900056FD0700D2013700B8
:10DF000060F22E009639020002000000CE013700B8
:10DF10006E5090006A4040006033B80084D02F00FB
:10DF20004500200022002000804078006E509000C4
:10DF3000A3FE0700C40137006E5090006A40400005
:10DF40006033B80084F12F0045002000120020004B
:10DF5000804078006E50900099FE0700BA013700AB
:10DF60006033B8006022B8000001EB008040EB0095
:10DF70006E50900092FE07006033B8006022B80037
:10DF80001200200031C0B3006E5090008CFE0700DC
:10DF900000000000AC0137006E5090006A4F400056
:10DFA00010002000500798006000B800100798008B
:10DFB000210798006000B8003007980041079800DA
:10DFC00010C0B300404F980010C0B300504F9800ED
:10DFD00000C0EB00604F9800050037002E0890004D
:10DFE000100078008000E8002E08900001087800FA
:10DFF0002E089000100078009E08900000804000DD
:10E000009040780000C2B30080CF5000F3FF320090
:10E010002E089000100078009E08900000804000BC
:10E0200010407800704F9800FE48900080C2B30006
:10E0300080CF500009003A002E08900010007800B0
:10E040008000E8002E089000010878002E0890005B
:10E0500010007800604F980039003700FE489000AB
:10E06000D0C2B30080CF500035003A002E08900097
:10E07000100078000000E8009E089000008040003A
:10E080009040780080C2B30080CF50002C003A004E
:10E0900020002000500798002E0890001000780003
:10E0A0008000E8002E089000010878002E089000FB
:10E0B000100078008000E8002E0890000108780029
:10E0C0002E08900010007800604F98001C00370068
:10E0D0006E4890000080FB009E0890000080400089
:10E0E0009040780090C2B30080CF500009003A0001
:10E0F0006E4890000080FB009E0890000080400069
:10E100008040EB000148780000C0EB00604F9800B1
:10E110000B0037006E4890000080FB009E089000C6
:10E12000008040009040780000C3B30080CF5000D2
:10E13000030032006E4890000040E800604F9800F5
:10E140006E489000E14F4000E1FF3A00280137009F
:10E150002E089000100078008000E8002E08900043
:10E160000108780001003700000000002E08900030
:10E17000100078009E0890000080400090407800D9
:10E1800000C2B30080CF5000F1FF32002E08900093
:10E19000100078009E089000008040001040780039
:10E1A000704F9800FE48900090C2B30080CF50009E
:10E1B00004003200FE489000D0C5B30080CF50006C
:10E1C00003003A000040EB00404F98000801370080
:10E1D0000040EB0010479800FE489000D0C2B3000A
:10E1E00080CF500007003A002E0890001000780001
:10E1F0008000E8002E0890000108780010C0B300ED
:10E20000104798007000470080017800622D2F00B1
:10E21000AE0890001E08900064020200000000009A
:10E220000004E000EC0032000E5090000080FB0083
:10E23000CF80DE000201200003002000820F50008A
:10E24000838F580069003E0000060100100037006F
:10E2500012003700170037001C003700630037003A
:10E2600020003700250037002A0037002F00370034
:10E2700034003700390037003E00370043003700D4
:10E28000480037004D003700520037005A00370071
:10E290000040EB00404F9800580037001E009000EF
:10E2A000AE0090000020A000100798002107980001
:10E2B000520037001E009000AE0090000110A00038
:10E2C00010079800210798004C0037001E009000AE
:10E2D000AE0090000070A000100798002107980081
:10E2E000460037001E009000AE0090000080A000A5
:10E2F0001007980021079800400037001E0090008A
:10E30000AE0090000030A000100798002107980090
:10E310003A0037001E009000AE0090000040A000C0
:10E320001007980021079800340037001E00900065
:10E33000AE0090000090A000100798002107980000
:10E340002E0037001E009000AE00900000A0A0003C
:10E350001007980021079800280037001E00900041
:10E36000AE00900000B0A0001007980021079800B0
:10E37000220037001E009000AE00900000C0A000F8
:10E3800010079800210798001C0037001E0090001D
:10E39000AE00900000D0A000100798002107980060
:10E3A000160037001E009000AE00900000E0A000B4
:10E3B0001007980021079800100037001E009000F9
:10E3C000AE00900000F0A000100798002107980010
:10E3D0000A0037001E009000AE0090000120A0004F
:10E3E0001007980021079800040037000040EB0058
:10E3F000404F980001003700000000001E409000D0
:10E400000004E000770032000E5090000080FB0016
:10E41000CF80DE000201200003002000820F5000A8
:10E42000838F580069003E0000060100100037008D
:10E4300012003700170037001C0037006300370058
:10E4400020003700250037002A0037002F00370052
:10E4500034003700390037003E00370043003700F2
:10E46000480037004D003700520037005F0037008A
:10E470000040EB00404F98005D0037003E009000E8
:10E48000CE0090000020A0003007980041079800BF
:10E49000570037003E009000CE0090000110A00011
:10E4A0003007980041079800510037003E00900067
:10E4B000CE0090000070A00030079800410798003F
:10E4C0004B0037003E009000CE0090000080A0007E
:10E4D0003007980041079800450037003E00900043
:10E4E000CE0090000030A00030079800410798004F
:10E4F0003F0037003E009000CE0090000040A0009A
:10E500003007980041079800390037003E0090001E
:10E51000CE0090000090A0003007980041079800BE
:10E52000330037003E009000CE00900000A0A00015
:10E5300030079800410798002D0037003E009000FA
:10E54000CE00900000B0A00030079800410798006E
:10E55000270037003E009000CE00900000C0A000D1
:10E560003007980041079800210037003E009000D6
:10E57000CE00900000D0A00030079800410798001E
:10E580001B0037003E009000CE00900000E0A0008D
:10E590003007980041079800150037003E009000B2
:10E5A000CE00900000F0A0003007980041079800CE
:10E5B0000F0037003E009000CE0090000120A00028
:10E5C0003007980041079800090037000040EB0031
:10E5D000404F9800060037000040EB00504F980075
:10E5E00003003700000000000100370000000000B9
:10E5F0004E4890000004E000030032005E489000A6
:10E600000004E000D8FE3A005E4890000004E000FC
:10E61000090032003E039000CE0390001E029000DD
:10E62000AE0290005E0190009E4078006E50900017
:10E63000E3FC070004003700C22C020002000000C7
:10E6400001003700000000000080FA000000060012
:10E650000400FA00004F7800110798001E00900097
:10E660008040EB00014878001E407800EF4F5000DA
:10E6700007003E001E80FB0080004000E0C6230033
:10E6800000804000904078001E0090000148780013
:10E690001E009000104078000080FB000000EA009F
:10E6A0004F00DE00004078000080FA000000060005
:10E6B0000600FA0020479800210798002E009000DD
:10E6C0008040EB000148780010C0B300004F780094
:10E6D0000B0037001E80FB0080004000E0C62300D6
:10E6E00000804000904078002E40900080CF500085
:10E6F00002003A002E0090001E4878001E4FE800ED
:10E700001E407800EF4F5000F2FF36000080FA0004
:10E71000000006000400FA002047980031479800E6
:10E720003E4090000080FB000000EA004F00DE0049
:10E73000004F78002E4090000004E00048003200B6
:10E740002E409000E64F500045003E002E409000C5
:10E750000080FB00E20F500018003200E20F500072
:10E7600005003C000000E0003C003200E10F5000DA
:10E77000080032003A003700E40F50002200320057
:10E78000E40F500017003500E50F5000280032005C
:10E79000330037009E40780061C060000080FB00BD
:10E7A000610060004A00DD00C170800001A0A1008E
:10E7B00001007000C0708800290037009E4078007A
:10E7C00061C060000080FB00610060004D00DD0062
:10E7D000C170800001D0A10001007000C0708800ED
:10E7E0001F0037009E40780061C060000080FB0081
:10E7F0004F00DD00C170800001F0A1000100700039
:10E80000C0708800160037009E40780061C060002C
:10E810000080FB00610060004900DD006171800044
:10E820000190A10001007000607188000C003700A9
:10E830009E40780061C060000080FB0061006000C5
:10E840004700DD00217080000170A1000100700010
:10E850002070880000000000010037000000000068
:10E860000080FA00000006000A00FA00889FBE003F
:10E87000004F9800114F98001E4890000004E000DF
:10E88000150032000E4890000082FB0010002000AE
:10E8900001002000F002120004003B008502EA00A3
:10E8A0008501DD000001EB00040037008502DE0079
:10E8B0000401DD008409DD00838172008091800005
:10E8C000919180000000710081807100809188002A
:10E8D000919188001D0037000E4890000083FB00D6
:10E8E00014002000050020007001130004003B000C
:10E8F0000201EA008220DD000000EB000400370086
:10E900000221DE000620DD008628DD008100710086
:10E910000082EA008182EA0080918000919180006B
:10E9200004037800050278008002780081007800F6
:10E930000500630081006200810178000001780019
:10E940000200BE00809188009191880010C0B30041
:10E95000004F78003E0037001E80FB006A00400038
:10E9600080004000E0C6230000804000104090007E
:10E970000080FB00100798001E009000E10F50007F
:10E98000030032001E009000E20F50002F003A00FA
:10E990001E80FB004300DD00E400400060C3230054
:10E9A000008040001001780090019000809180006C
:10E9B0009191800000006900818069002007980023
:10E9C000310798001E80FB00C300DD0060C32300F8
:10E9D0000080400010017800900190002E0090000F
:10E9E000BE009000020278000301780080017800E8
:10E9F00081007800030062008100610081047800DA
:10EA0000000478000800BE000080700000F0A7003D
:10EA10000000EA000000EA004F00DE001047980006
:10EA20001E009000E20F500005003A001E409000CA
:10EA30000080FB000000E9004F00DE001047980056
:10EA40009E4090001E40780032FF07001E4FE800F5
:10EA50001E407800E64F5000BFFF360080918000D6
:10EA6000919180006E7D0200000000004F04BE0006
:10EA70000080FA00000006000200FA00000F780093
:10EA800080918000919180001E0178000089BE0075
:10EA90000080FA00000006000800FA0060479800B5
:10EAA000714798000000EB00100798006E4090003E
:10EAB0000004E0007C0032006E409000EF4F5000F8
:10EAC00079003E006E4090000080FB008000400016
:10EAD000E0C6230000804000904078004147980045
:10EAE0006E4090000080FB0080004000E0C62300E4
:10EAF00000804000104090000080FB00100798004C
:10EB0000FE429000554798005E4090000004E000EF
:10EB1000150032006E4090000082FB0010002000C3
:10EB200001002000F002120004003B008502EA0010
:10EB30008501DD000001EB00040037008502DE00E6
:10EB40000401DD008409DD00838172008091800072
:10EB50009191800000007100818071008091880097
:10EB6000919188001D0037006E4090000083FB00EB
:10EB700014002000050020007001130004003B0079
:10EB80000201EA008220DD000000EB0004003700F3
:10EB90000221DE000620DD008628DD0081007100F4
:10EBA0000082EA008182EA008091800091918000D9
:10EBB0000403780005027800800278008100780064
:10EBC0000500630081006200810178000001780087
:10EBD0000200BE0080918800919188000040EB0007
:10EBE000004F780010C0B300104798002100370094
:10EBF0001E4090000080FB0080004000E0C6230023
:10EC000000804000904078004E40900080CF50003F
:10EC100015003A0082918000939180001E40900080
:10EC20000082FB00F002120004003B008502EA00B3
:10EC30000518DE008000EB0004003700851ADD00B7
:10EC40000410DE00008072008418DE0000007800EE
:10EC500061006000004078000004E0000200320023
:10EC600010C0B300004F78001E4090000040E80044
:10EC7000104798001E409000EF4F5000DCFF360018
:10EC80001E009000E20F500004003A001E80FB00BE
:10EC90000000E9004F00DE00004F78009E40780041
:10ECA0004E4090009BFE07000080FA000000060026
:10ECB0000200FA00004F78001E80FB00E30F5000B6
:10ECC00014003200E30F500005003C00E10F50003B
:10ECD00008003200E20F50000A003200190037002D
:10ECE000E40F50000F003200E50F50001100320019
:10ECF00014003700F0332F009639020002000000A4
:10ED00001400370050342F00963902000200000032
:10ED100010003700B0342F009639020002000000C6
:10ED20000C00370010352F00963902000200000059
:10ED30000800370070352F009639020002000000ED
:10ED40000400370060D22E00963902000200000055
:10ED5000000000000080FA00000006000200FA0037
:10ED6000004F7800114798001E4090000004E0001A
:10ED70003A0032001E80FB00E60F50001E003200F9
:10ED8000E60F500007003C00E20F50001200320076
:10ED9000E30F500014003200E10F50000A0032006F
:10EDA0002A003700E80F50001B003200E80F500027
:10EDB00015003500E90F50001B003200EA0F50002B
:10EDC0001D00320021003700D0352F009639020097
:10EDD000020000005A00370030362F00963902003A
:10EDE000020000005600370090362F0096390200CE
:10EDF0000200000052003700D0362F009639020082
:10EE0000020000004E00370030372F009639020014
:10EE1000020000004A00370090372F0096390200A8
:10EE20000200000046003700F0372F00963902003C
:10EE3000020000004200370070382F0096390200AF
:10EE400002000000000000003D003700D0EE2E0060
:10EE50009639020002000000390037001E80FB00D6
:10EE6000E60F50001E003200E60F500007003C0085
:10EE7000E20F500012003200E30F50001400320085
:10EE8000E10F50000A00320029003700E80F50005F
:10EE90001B003200E80F500015003500E90F50004C
:10EEA0001B003200EA0F50001D0032002000370026
:10EEB000D0382F00963902000200000020003700F1
:10EEC00030392F0096390200020000001C00370084
:10EED00090392F0096390200020000001800370018
:10EEE000D0392F00963902000200000014003700CC
:10EEF000303A2F009639020002000000100037005F
:10EF0000903A2F0096390200020000000C003700F2
:10EF1000F03A2F0096390200020000000800370086
:10EF200060D22E0096390200020000000400370073
:10EF3000D0EE2E0096390200020000000000000012
:10EF40000080FA00000006001200FA00889FBE0050
:10EF5000200798003107980042079800530798004F
:10EF60006407980075079800065798000040EB006A
:10EF7000104798000040EB00004F78001B0137005D
:10EF80001E82FB002E019000BE019000F0021200D4
:10EF900004003B008502EA000518DE008000EB005B
:10EFA00004003700851ADD000410DE0000807200C6
:10EFB0008418DE00000078006100600000407800E6
:10EFC0000004E000080132001E409000E54F5000B0
:10EFD00005003600703B2F00963902000200000049
:10EFE00010C0B300104798001E4090000004E000DD
:10EFF00003003200D0EE2E0096390200020000001D
:10F000001E82FB004E019000DE019000F002120013
:10F0100004003B008502EA000518DE008000EB00DA
:10F0200004003700851ADD000410DE000080720045
:10F030008418DE0000007800610060000040780065
:10F040000004E0001C003200B03C2F0096390200A2
:10F05000020000001E82FB006E019000FE01900085
:10F06000F002120004003B008502EA000518DE00F1
:10F070008000EB0004003700851ADD000410DE007C
:10F08000008072008418DE000000780061006000DB
:10F090008004EB00000478000800BE0000807000CF
:10F0A00000F0A7000000EA000000E9004F00DE00C9
:10F0B00020479800100037001E82FB006E01900070
:10F0C000FE019000F002120004003B008502EA00FD
:10F0D0000518DE008000EB0004003700851ADD0013
:10F0E0000410DE00008072008418DE00004078000A
:10F0F00061406000204798000E5090000004E0003E
:10F100005D0032002E4090000004E0005A00320002
:10F110001E80FB006101B900E0FF2F00F1FF2F000E
:10F12000020040008380480002012000030020000C
:10F13000820F5000838F58004A003E0000060100F5
:10F1400010003700170037001A003700450037005D
:10F15000440037001B0037001E0037002100370035
:10F1600024003700270037002A0037002D00370021
:10F1700030003700330037003A0037000500370011
:10F1800034003700D03C2F00963902000200000006
:10F1900038003700403D2F00963902000200000081
:10F1A00034003700803D2F00963902000200000035
:10F1B00030003700C03D2F009639020002000000E9
:10F1C0002C003700003E2F0096390200020000009C
:10F1D00028003700703E2F00963902000200000020
:10F1E00024003700103F2F00963902000200000073
:10F1F00020003700903F2F009639020002000000E7
:10F200001C00370000402F00963902000200000069
:10F210001800370080402F009639020002000000DD
:10F220001400370000412F00963902000200000050
:10F230001000370080412F009639020002000000C4
:10F240000C003700F0412F00963902000200000048
:10F250000800370070422F009639020002000000BB
:10F260000400370030432F009639020002000000EE
:10F2700000000000590037001E80FB006101B9004A
:10F28000E0FF2F00F1FF2F000200400083804800C4
:10F290000201200003002000820F5000838F5800DD
:10F2A0004A003E000006010010003700170037003A
:10F2B0001A00370045003700440037001B003700B4
:10F2C0001E003700210037002400370027003700D8
:10F2D0002A0037002D003700300037003300370098
:10F2E0003A003700050037003400370050432F0044
:10F2F000963902000200000038003700C0432F009A
:10F3000096390200020000003400370000442F004C
:10F3100096390200020000003000370040442F0000
:10F3200096390200020000002C00370080442F00B4
:10F33000963902000200000028003700F0442F0038
:10F3400096390200020000002400370090452F008B
:10F3500096390200020000002000370010462F00FE
:10F3600096390200020000001C00370080462F0082
:10F3700096390200020000001800370000472F00F5
:10F3800096390200020000001400370080472F0069
:10F3900096390200020000001000370000482F00DC
:10F3A00096390200020000000C00370070482F0060
:10F3B000963902000200000008003700F0482F00D4
:10F3C00096390200020000000400370030432F008D
:10F3D0009639020002000000000000001E4090006C
:10F3E0000040E800104798001E4FE8001E407800DB
:10F3F000F24F5000E2FE36004F04BE000080FA00DB
:10F40000000006000C00FA00889FBE00204F980004
:10F41000314F98002E4890000004E000480132006F
:10F420002E489000E64F500045013E000040EB00A2
:10F43000504798000000EB001007980010C0B30080
:10F4400060479800160037006E4090000080FB0077
:10F4500080004000E0C6230000804000904078001B
:10F460002E48900080CF50000A003A00EE409000F5
:10F47000514798006E4090000080FB0080004000E3
:10F48000E0C6230000804000104090000080FB0098
:10F49000100798006E4090000040E8006047980018
:10F4A0005E4090000004E00003003A006E409000CF
:10F4B000EF4F5000E4FF36002E489000E54F50001B
:10F4C00003003E005E4090000004E00003003A00AC
:10F4D0003E4890000004E00019013200D0ED2E00FB
:10F4E00096390200020000002E489000F0FD07004F
:10F4F000D0ED2E0096390200020000003E48900038
:10F500000004E000D10032001E009000E30F500024
:10F5100031003A0067004700800078005E409000AC
:10F520005BF807000004E000FF0032007E4090001E
:10F530000080FB0041C0B300EE2802000200000082
:10F54000D0ED2E00963902000200000011C0B30079
:10F550005E40900001FE07005E409000E84F5000C2
:10F5600003003A0064CD020001000000F100370002
:10F570005E409000E24F5000ED003A00E900470085
:10F5800068004700681F020001000000B0492F001A
:10F5900096390200020000000E4890000000FB00B7
:10F5A0003E09020001000000304A2F009639020097
:10F5B000020000001E4890000080FB0011C0B30054
:10F5C000EE28020002000000604A2F009639020077
:10F5D00002000000D70037001E009000E40F50002A
:10F5E00010003A00804A2F00963902000200000005
:10F5F0002170800000402000008060000000E000DA
:10F6000004003200404B2F00963902000200000037
:10F61000C8003700C04B2F009639020002000000DE
:10F62000C40037000040EB00404798002E4890008F
:10F630000080FB00E30F500016003200E30F500083
:10F6400005003C00E10F500008003200E20F5000BE
:10F650000B00320020003700E40F5000120032008F
:10F66000E50F5000150032001B003700C07080000D
:10F670004A00DE0061406000004F7800190037004A
:10F68000C07080004D00DE0061406000004F7800D7
:10F6900014003700C07080004F00DE00004078008A
:10F6A000004F78000F003700607180004900DE00D5
:10F6B00061406000004F78000A0037002070800031
:10F6C0004700DE0061406000004F780010C0B300CA
:10F6D00040479800030037000040EB00004F7800DF
:10F6E000000000004E4090000004E0000B003200DB
:10F6F0001E4078000004E00004003200504C2F004F
:10F7000096390200020000000E003700B04C2F00B6
:10F7100096390200020000000A0037001E407800FF
:10F720000004E00004003200104D2F009639020062
:10F730000200000003003700B04C2F009639020091
:10F7400002000000D0EE2E009639020002000000F8
:10F750005E409000E34F50000F003A009E4078005A
:10F7600030C0B3007DFD0700E90047006800470096
:10F77000681F020001000000B0492F009639020006
:10F78000020000000E4890000000FB003E0902004D
:10F7900001000000670037005E409000EA4F500013
:10F7A000260036005E409000EF4F500023003E00E0
:10F7B0001E009000E20F500003003A00704D2F0031
:10F7C000963902000200000082918000939180002F
:10F7D0002E4890000080FB004300DD00E400400064
:10F7E00060C323000080400090009000100078006B
:10F7F0002E4A90000482FB00C322DD0064C3230074
:10F8000004824200140478009404900016C0B300EF
:10F810000202BE000001BE000800BE00CAFD0700D3
:10F820001E009000E20F500042003A00A04D2F0051
:10F8300096390200020000003E0037009E4078002A
:10F840005E40900045FD07003A003700C04D2F0094
:10F8500096390200020000005E409000EA4F50001E
:10F860000A003E001E009000E20F500003003A0024
:10F87000B03C2F0096390200020000008040EB00EF
:10F880005E40900035FD07002A0037005E40900082
:10F890006A405000204F98002E489000E54F5000DD
:10F8A00024003E001E009000E20F500003003A00CA
:10F8B000704D2F0096390200020000002E48900083
:10F8C0000080FB004300DD00E400400060C3230033
:10F8D0000080400090009000100078002E499000B9
:10F8E0000281FB00C311DD0062C3230002814100DD
:10F8F00012047800920490000043EB006022B800EC
:10F900000001BE000800BE008FFD07001E00900031
:10F91000E20F500007003A00A04D2F009639020078
:10F920000200000003003700000000000100370063
:10F930000000000000ED2E009639020002000000D9
:10F940004F04BE000080FA00000006000400FA0028
:10F950002047980010C0B300004F78000400370023
:10F96000AE4090001E407800A6FE07001E4FE80043
:10F970001E407800E64F5000F9FF36000080FA0084
:10F98000000006000200FA0010C0B300004F78002B
:10F99000060037001E40780093F607008040EB0019
:10F9A0001E4078005BFB07001E4FE8001E407800F9
:10F9B000E84F5000F7FF36000080FA000000060014
:10F9C0000200FA0010C0B300004F780019003700A1
:10F9D0001E80FB0080004000E0C623000080400045
:10F9E00010409000E34F500007003A001E80FB00DB
:10F9F00080004000E0C623000080400010407800F6
:10FA000094F607000A0037001E407800E14F5000CE
:10FA100004003A0011C0B30010C0B3001EFC070080
:10FA2000030037008040EB001E4078001AFC0700FE
:10FA30001E4FE8001E407800EF4F5000E4FF3600F4
:10FA40000080FA00000006000000FA000000EB0051
:10FA5000B0DF89000000EB0040E08900A00F21002A
:10FA600030E089004076260010E089002010210057
:10FA7000C0DF890060102100D0DF8900A0102100C4
:10FA8000E0DF8900E0102100F0DF89002011210073
:10FA900000E089006011210020E08900803226000A
:10FAA00050E08900E011210060E089002078260004
:10FAB00070E089006012210080E089008032260019
:10FAC00090E08900AFFF0700BDFF07003032EF0074
:10FAD0003232EF000080FA00000006001800FA0041
:10FAE000889FBE008A9FBE008C9FBE00008FBE0014
:10FAF0000040EB00282F0200020000000040EB0055
:10FB0000622F0200020000000040EB009E2F020066
:10FB10000200000002802000030020001E00780088
:10FB20009E00900080027800010278008200780038
:10FB30000300780081806200000062008004780089
:10FB4000010478000800BE00E00F5000E08F58006C
:10FB50000C00320080C0B30064F2B700F003200054
:10FB6000309388006832EF0020C0B300282F0200D5
:10FB70000200000010C0B300622F0200020000006B
:10FB8000CA00370002002100030020001E00780098
:10FB90009E009000800278000102780082007800C8
:10FBA0000300780081806200000062008005780018
:10FBB000010578000A00BE00E00F5000E08F5800F9
:10FBC0000C00320000C1B30064F2B700F0FF230064
:10FBD000309388006832EF0020C0B300282F020065
:10FBE0000200000010C0B3009E2F020002000000BF
:10FBF000AE00370002002200030020001E00780043
:10FC00009E00900080027800010278008200780057
:10FC100003007800818062000000620080067800A6
:10FC2000010678000C00BE00E00F5000E08F580085
:10FC30000900320000C1B30064F2B700F0FF2000F9
:10FC4000309388006832EF0020C0B300282F0200F4
:10FC500002000000950037008240200003002000D1
:10FC60001E0078009E00900080027800010278005B
:10FC7000020078008300780000806200810062004A
:10FC800031079800200798002E009000BE009000D9
:10FC9000E00F5000E08F58000C00320040C0B3006D
:10FCA00064F2B70030002000309388006832EF0023
:10FCB00020C0B300282F02000200000010C0B300D3
:10FCC0009E2F020002000000780037000021200073
:10FCD000010020001E0178009E01900002027800C1
:10FCE0000301780080017800810078000300620041
:10FCF0008100610051079800400798004E00900075
:10FD0000DE009000E00F5000E08F58000C00320041
:10FD100080C0B30064F2B700F00020003093880088
:10FD20006832EF0020C0B300282F0200020000005C
:10FD300010C0B3009E2F0200020000005B003700DD
:10FD400000002C00010020001E0178009E019000A0
:10FD500002027800030178008001780081007800B9
:10FD6000030062008100610071079800600798003D
:10FD70006E009000FE009000E00F5000E08F5800F1
:10FD80000A00320040C0B30064F2B700F000200067
:10FD900030938800300020004093880020C0B300DA
:10FDA000282F020002000000400037000010200051
:10FDB000010020001E0178009E01900002027800E0
:10FDC0000301780080017800810078000300620060
:10FDD00081006100110F9800000F98000E0890003C
:10FDE0009E089000E00F5000E08F58000D00320098
:10FDF00000C1B30064F2B700C0FF2F003093880049
:10FE0000300020004093880020C0B300282F02005B
:10FE10000200000010C0B3009E2F0200020000008C
:10FE2000220037001E0078009E009000000078003D
:10FE3000640060008000EB00310F9800200F9800F4
:10FE40002E089000BE089000E00F5000E08F580090
:10FE50000700320000C1B30064F2B700F00F2000C9
:10FE6000309388000080EB00409388000F0037003B
:10FE70001E00780061006000004078000004E0008F
:10FE80000600320000C1B30064F2B7006632EF0032
:10FE9000F0FF2700409388000400370020C0B30023
:10FEA00064F2B7006632EF006832EF004F06BE0022
:10FEB0004F05BE004F04BE000080FA00000006009F
:10FEC0000000FA006232EF0010C0B30064F2B70025
:10FED0006632EF006832EF000080FA000000060092
:10FEE0000600FA00C08D80004300DE00000F78009D
:10FEF000109380009E007800808F50003A003200FE
:10FF000064D2BF000080FB009E00780000017800F2
:10FF1000110009008280D800100798001E007800A8
:10FF2000804078001E0090000040780042262100AA
:10FF3000124178000281FB008090B90000407800F7
:10FF400000C05000404798004E4090000080FB00E9
:10FF5000110020000008DD00800078004093800040
:10FF60000080600000F0A7000000EA000000EA0046
:10FF70004F00DE00004078000080FB006100600060
:10FF80004200DD00617180000120A10001007000CD
:10FF9000607188004E4090000080FB00110020003E
:10FFA0000008DD0080007800309380000080600051
:10FFB00000F0A7000000EA000000EA004F00DE00A9
:10FFC000004078000080FB006100600000004000FD
:10FFD000617180000110A100010070006071880053
:10FFE0009E007800119388000080FA00000006004F
:020000040001F9
:10000000202A00002A2A00000D0A0000002000001B
:100010002A2A00002A2000002020000020200000C2
:1000200020200000202000002020000020200000D0
:1000300020200000202000002020000020200000C0
:10004000747300006D320000353000003020000075
:10005000505200004F470000524100004D4D00003B
:10006000494E000047200000202000002020000012
:100070002020000020200000202000002020000080
:100080002020000020200000202000002020000070
:10009000202000002A2A00002A0D00000A0000008B
:1000A000202A00002A2A00002057000041520000A8
:1000B0004E4900004E4700003A20000054680000FE
:1000C00069730000206300006F6D00006D61000027
:1000D0006E64000020630000686100006E6700002D
:1000E0006573000020740000686500002043000074
:1000F000414E000020490000442000006F660000CF
:10010000206100002043000048340000313000002E
:100110003020000063680000617200006765000025
:1001200072200000202A00002A2A00000D0A000088
:10013000002000002A2A00002A2000004F4E000064
:100140004C590000204F00004E4500002074000074
:10015000736D000032350000303000002063000075
:100160006861000072670000657200002073000083
:10017000686F0000756C000064200000626500007C
:10018000207000006F770000657200006564000059
:1001900020750000702000006174000020740000D1
:1001A0006869000073200000746900006D6500003C
:1001B00020200000202000002A2A00002A0D000034
:1001C0000A000000202A00002A2A00000D0A000070
:1001D0000D0A0000507200006F63000065650000AA
:1001E000642000005B5900002F4E00005D200000DD
:1001F0003F20000000500000726F00006772000096
:10020000616D00006D6900006E67000020740000E1
:1002100068650000206300006861000072670000EC
:1002200065720000202E00002E2E0000200000002D
:10023000646F00006E6500002E0D00000A5400007F
:1002400068650000206300006861000072670000BC
:1002500065720000206D00007573000074200000BE
:100260006E6F0000772000006265000020700000C3
:100270006F77000065720000206300007963000062
:100280006C650000642E00000D0A00000074000080
:10029000736D000032350000303000002020000077
:1002A00020000000747300006D3200003530000043
:1002B000305F00003431000000740000736D0000F6
:1002C00032350000303000005F34000032000000A2
:1002D000747300006D32000035300000305F0000A4
:1002E00034330000006500006C6300006F6E000096
:1002F000202000002020000020000000656C00008D
:10030000636F00006E5F0000653700002020000072
:10031000006500006C6300006F6E00005F65000008
:100320003820000020000000656C0000636F0000B2
:100330006E5F00006539000020200000006C0000A6
:1003400065610000722000002020000020200000D5
:10035000200000006E6C00006735000020200000C7
:100360002020000020200000007600006F6C0000BC
:100370007420000020200000202000002000000049
:1003800073740000656100006C7400006820000058
:10039000202000000062000061730000696300001B
:1003A00020200000202000002000000063680000E2
:1003B00061720000676500006D6F00002020000082
:1003C000003F00003F20000020200000202000000F
:1003D0002020000020000000204C00003100000020
:1003E000204C000032000000204C000033000000D0
:1003F000202000002000000072780000206500002E
:1004000072720000006800007766000061690000F9
:100410006C00000068690000746500006D700000E9
:10042000006900006E700000757400002076000006
:100430006F6C0000746100006765000020650000BB
:100440007272000000700000616300006B20000009
:10045000766F00006C74000061670000652000008A
:1004600065720000720000006E6F000074200000D2
:100470006368000061720000676900006E67000039
:10048000002C00002000000045720000726F000088
:10049000723A00002063000068610000726700008B
:1004A0006572000020000000206E00006F740000E4
:1004B000206300006F6E0000666900006775000031
:1004C00072650000642100000D0A0000003A00007F
:1004D000205600003D0000002C200000413D00009F
:1004E000002C0000205700003D0000002C200000E0
:1004F000576800003D000000200000002C20000094
:10050000544D0000503D0000002D0000004300004D
:100510000078000000430000484300004150000004
:10052000203A0000206D00003D000000562C000025
:10053000004100002C200000743D00000056000027
:100540002C200000696400003D0000000D0A00003E
:10055000004300004853000054410000543A00009A
:10056000206300003D000000412C000020730000CB
:10057000663D000000630000687200006720000014
:10058000006600006C740000200000006C6F00002A
:10059000636B000020000000696E00006320000013
:1005A00000730000666C00007420000000730000FF
:1005B000746F000070200000002C00002063000019
:1005C000723D0000002C0000206300007232000029
:1005D0003D0000002C200000696400003D00000088
:1005E0004348000041520000474500004D4F0000C5
:1005F000002C0000205400003D0000002C200000D2
:10060000544D000050680000693D000000430000A8
:100610002C200000544D0000506C00006F3D000085
:10062000004300002C2000006C6900006D69000090
:10063000743D0000004300004300000043560000EA
:100640000043000054000000657600006363000072
:100650002D3E0000430000004556000043430000CB
:10066000206300006F6E000066690000672E0000C6
:100670002E0000007265000073650000740D00001C
:100680000A00000044490000534300004F4E0000A0
:100690004E45000043540000454400000043000064
:1006A0004F4E00004E4500004354000045440000FA
:1006B000004C00004F4300004B4500004400000088
:1006C00044490000534300004F4E00004E450000D7
:1006D000435400005F5700004149000054000000EF
:1006E00041430000544900005645000000530000FB
:1006F00054410000525400005550000000530000C7
:10070000544100004E4400004259000000430000E4
:1007100048410000524700004500000046490000E3
:100720004E490000534800002043000048410000AB
:100730005247000045000000464C00004F410000B9
:10074000542000004348000041520000474500008B
:1007500000570000415200004D4400004F57000078
:100760004E00000043480000415200004745000091
:100770002F5400004F500000424100004C41000047
:100780004E43000045000000434800004152000075
:10079000474500004D4F000020430000414E00003F
:1007A0002057000041490000540000004348000069
:1007B00041520000474500004D4F0000205300000B
:1007C000455100003220000057410000495400000C
:1007D000004300004841000052470000454D000022
:1007E0004F200000434800004152000047490000EC
:1007F0004E470000004300004841000052470000FF
:10080000454D00004F20000057410000524D0000B0
:10081000444F0000574E00000043000048410000D4
:1008200052470000454D00004F2000004F5000008F
:10083000454E0000204300004F4E00005441000090
:10084000435400004F520000530000004E4F000080
:100850004E4500000048000057460000415500008A
:100860004C54000000430000434500004E5300007C
:100870005553000000540000434500004E53000053
:10088000555300000048000056430000004C000093
:10089000564300000048000049540000454D000048
:1008A000500000004C4F000057540000454D000020
:1008B000500000004E4F0000544C00004F43000019
:1008C0004B45000044000000484900005041000032
:1008D000434B000000490000534F00004C41000012
:1008E000544900004F4E00002046000041550000D2
:1008F0004C540000004E00004F5200004D410000DB
:100900004C000000504C00005547000020440000FF
:1009100049530000434F00004E4E00004543000085
:100920005445000044000000434500004C4C0000CA
:10093000204C00004F4F00005000000045560000C2
:100940005345000020540000494D0000454F000071
:100950005554000000430000484100005247000089
:100960004552000020520000582000005449000069
:100970004D4500004F550000540000004E4F000050
:1009800020500000414300004B000000434800009D
:10099000415200004745000052200000535400001F
:1009A0004F50000000430000484100005247000043
:1009B00045200000544900004D4500004F550000FF
:1009C000540000004E4F0000204900005345000035
:1009D0004E5300004F520000004E00004F20000018
:1009E00054480000455200004D4900005354000097
:1009F0004F520000004E00004F2000005345000001
:100A000051310000004E00004F200000534500000F
:100A100051320000005300005953000020450000EF
:100A2000525200004F520000004F00005554000089
:100A30005055000054200000435500005252000061
:100A4000454E0000542000004C4F000057000000AD
:100A50004F55000054500000555400002043000042
:100A600055520000524500004E540000204800003E
:100A700049470000480000004F5500005450000056
:100A8000555400002043000055520000524500001C
:100A90004E540000204E0000454700004154000025
:100AA0004956000045000000564F00004C5400001D
:100AB00041470000452000004D490000534D000013
:100AC000415400004348000000450000562000004B
:100AD000494E0000434F00004D50000041540000BB
:100AE000494200004C45000000430000484100001E
:100AF0005247000045520000204E00004F540000B5
:100B000020520000554E00004E4900004E470000A4
:100B10000045000056200000535400004F500000D4
:100B2000004E00004F5200004D4100004C5F00009D
:100B3000530000004E4F0000524D0000414C000099
:100B40005F56000000200000202000004E4F0000F3
:100B50004E45000020200000200000002020000062
:100B60006877000066610000756C0000742000006A
:100B70000020000020630000636500006E73000029
:100B80007573000020000000202000007463000046
:100B9000656E0000737500007320000000200000E7
:100BA00020200000204800005643000020200000C4
:100BB0002000000020200000202000004C560000F3
:100BC00043200000202000000020000020680000DA
:100BD00069740000656D00007020000020000000B6
:100BE000202000006C6F000077740000656D00002D
:100BF00070200000002000006E6F0000746C000088
:100C00006F6300006B65000064000000202000009E
:100C10006869000070610000636B00002020000024
:100C200000200000697300006F660000617500001D
:100C30006C7400002000000020200000206E0000E6
:100C40006F7200006D6100006C2000000020000049
:100C5000706C00007567000020640000697300007C
:100C60006300000020630000656C00006C20000041
:100C70006C6F00006F7000000020000045560000FF
:100C800053450000207400002F6F0000200000007A
:100C9000206300006867000072200000742F0000CD
:100CA0006F20000000200000206E00006F20000078
:100CB00070610000636B00002000000020630000F2
:100CC0006867000072200000737400006F700000FD
:100CD000006300006861000072670000652000008A
:100CE000742F00006F0000006E6F0000206900008C
:100CF000736500006E7300006F720000002000003A
:100D00006E6F00002074000068650000726D0000C6
:100D100020000000202000006E6F00002053000023
:100D2000455100003120000000200000206E00002E
:100D30006F200000534500005132000020000000E9
:100D400020730000797300002065000072720000BB
:100D50006F720000002000006368000067720000EE
:100D6000206600006C74000020000000206C000071
:100D70006F770000206300007572000020200000E3
:100D80000020000068690000676800002063000020
:100D90007572000020000000206E000065670000F2
:100DA0002063000075720000202000000056000043
:100DB000206D0000697300006D6100007463000025
:100DC0006800000065760000696E0000636F000037
:100DD0006D70000061740000006300006820000076
:100DE0006E6F0000742000006F6E00002000000095
:100DF0002020000020730000746F000070200000AD
:100E000020200000002000006E6F0000726D0000C6
:100E1000616C00002053000020000000206E0000E4
:100E20006F7200006D6100006C2000005620000011
:100E30000020000020200000203F00003F20000094
:100E400020200000200000004368000061720000C4
:100E500067650000205300007461000074650000A5
:100E60003A200000002000003D3E0000200000006D
:100E70002C20000074650000726D000020720000DC
:100E8000736E00003D000000506C000075670000AC
:100E90002053000074610000746500003A200000D7
:100EA000007A000065760000636300007320000094
:100EB00020200000203A000020430000435300009F
:100EC0005F4300004D4400003B20000063750000BC
:100ED000726C0000696D00003D000000410D0000D3
:100EE0000A0000007A65000076630000637300006A
:100EF00020200000202000003A2000004343000092
:100F0000535F000044490000414700003B200000BF
:100F100062760000733D0000005600002C200000A7
:100F200063760000733D0000005600002C20000096
:100F3000643D00000045000056420000415400009E
:100F4000543A0000206D00003D000000412C0000DC
:100F50002072000061740000653D00000045000043
:100F600056540000494D0000453A0000206500003D
:100F70003D0000006D6900006E2C0000206D000037
:100F8000313D0000006D0000696E00002C20000063
:100F90006D3200003D00000073650000632C00000E
:100FA000004B000077480000004500005653000049
:100FB00054410000543A00002076000065720000A1
:100FC0003D000000412C0000205300004F43000072
:100FD0003D0000002C200000663D0000002C0000B9
:100FE00020730000747300003D0000000D0A000033
:100FF0002041000063740000756100006C20000057
:10100000766F00006C7400006167000065000000EE
:101010000D0A0000204300006861000064650000C4
:101020006D6F0000207600006F6C0000746100009E
:101030006765000000200000202000002020000044
:1010400020200000202000002020000073790000F4
:1010500073200000737400006174000065200000BC
:101060003D000000682C0000206500007620000094
:10107000737400006174000075730000203D00006F
:10108000006800002C20000065760000206600004B
:10109000617500006C740000203D000000680000D5
:1010A0002C200000636800002073000074610000C1
:1010B00074750000732000003D000000680D000002
:1010C0000A0000004A3100003737000032200000DB
:1010D000006C00006F6300006B650000642000007E
:1010E000006300006F6E00006E6500006374000016
:1010F0006564000020000000646900007363000064
:101100006F6E00006E65000063740000656400008F
:10111000200000004A310000373700003254000040
:101120003220000000430000484100005247000008
:10113000454D00004F200000006300006F6E00006E
:101140006E650000637400006564000000640000C8
:1011500069730000636F00006E6E0000656300003D
:101160007465000064000000410000002C200000B5
:10117000707200006F660000696C0000653D000041
:101180000070000072650000736500006E7400005E
:10119000006E00006F740000207000007265000097
:1011A000736500006E740000002000002000000045
:1011B000203A0000005600002020000020200000FF
:1011C000202000000041000020200000202000001E
:1011D000202000000020000020200000696E000098
:1011E00066200000202000002020000020200000B9
:1011F0000068000072200000202000002020000075
:10120000006D0000696E000020200000202000001A
:10121000002000003F3F00002020000020200000B0
:1012200020200000202000002020000000200000DE
:1012300020200000202000002020000020200000AE
:1012400020200000202000002000000020200000BE
:101250005345000074200000504C0000554700002A
:10126000203C0000703E00002020000020200000F4
:101270002020000020200000202D0000206300001E
:10128000686100007267000065200000706C00005B
:10129000756700002074000079700000650D000083
:1012A0000A20000020530000457400002045000083
:1012B00056530000455700004149000054200000EB
:1012C0003C6D00003E200000202000002020000097
:1012D0002D200000455600005345000020770000F7
:1012E0006169000074200000746900006D650000F1
:1012F0000D0A00002020000053450000742000006B
:1013000043480000415200004745000052200000C1
:10131000202E00002E2E00002020000020200000A3
:10132000202D00002064000065660000696E00004A
:1013300065730000206300006861000072670000B0
:1013400065720000203100000D0A0000002000003E
:101350002053000045740000204300004841000075
:101360005247000045520000322000002E2E00009F
:101370002E20000020200000202000002D20000052
:1013800064650000666900006E650000732000005F
:101390006368000061720000676500007220000051
:1013A000320D00000A2000002053000045740000A8
:1013B0002043000048410000524700004552000011
:1013C000332000002E2E00002E20000020200000E0
:1013D000202000002D2000006465000066690000E8
:1013E0006E650000732000006368000061720000F9
:1013F0006765000072200000330D00000A20000025
:1014000020530000457400002043000048410000C4
:101410005247000045520000342000002E2E0000EC
:101420002E20000020200000202000002D200000A1
:1014300064650000666900006E65000073200000AE
:1014400063680000617200006765000072200000A0
:10145000340D00000A000000202000005345000069
:10146000742000004C4900004E450000562000004A
:101470003C7600003E2000002020000020200000DC
:1014800020200000202D0000206C0000696E00006C
:1014900065200000766F00006C740000616700003A
:1014A000650D00000A200000205300004574000074
:1014B000204C0000494E000045430000203C000045
:1014C000633E0000202000002020000020200000BB
:1014D000202000002D2000006C6900006E650000D7
:1014E0002063000075720000726500006E740000D9
:1014F0000D0A000020200000534500007420000069
:101500004D41000058560000203C0000763E00008F
:1015100020200000202000002020000020200000CB
:10152000202D0000206D000061780000696D000032
:10153000756D0000206300006861000072670000A4
:10154000696E000067200000766F00006C74000078
:1015500061670000650D00000A20000020530000B4
:1015600045740000204D0000415800004320000059
:101570003C6100003E2000002020000020200000F0
:1015800020200000202000002D2000006D610000C0
:10159000786900006D7500006D2000006368000030
:1015A00061720000676900006E6700002063000040
:1015B00075720000726500006E7400000D0A000074
:1015C0002020000053450000742000005445000016
:1015D000524D0000432000003C6100003E2000000E
:1015E000202000002020000020200000202D0000EE
:1015F00020740000657200006D6900006E610000DB
:10160000746900006F6E00002063000068610000D4
:1016100072670000696E00006720000063750000BB
:1016200072720000656E0000740D00000A20000058
:101630002053000045740000205400004552000073
:101640004D540000203C0000743E000020200000AB
:101650002020000020200000202000002D2000007D
:101660006D610000786900006D7500006D2000005C
:10167000636800006172000067650000207400006C
:10168000696D0000650D00000A00000020200000C8
:101690005345000074200000464900004E5F0000E2
:1016A0004D41000058560000203C0000763E0000EE
:1016B0002020000020200000202D000020660000D7
:1016C000696E000069730000686900006E670000C1
:1016D0002063000068610000726700006520000060
:1016E0006D61000078200000766F00006C740000CF
:1016F00061670000650D00000A2000002053000013
:101700004574000020460000494E00005F4D000077
:1017100041580000432000003C6100003E200000D2
:1017200020200000202000002D200000666900001D
:101730006E69000073680000696E00006720000099
:10174000636800006172000067650000206D0000A2
:10175000617800002063000075720000726500006F
:101760006E7400000D0A00002020000053450000A8
:1017700074200000464900004E5F00005445000000
:10178000524D0000542000003C7400003E20000038
:1017900020200000202D000020660000696E00005F
:1017A00069730000686900006E6700002063000034
:1017B0006861000072670000652000006D61000034
:1017C0007820000063680000617200006765000017
:1017D00020740000696D0000650D00000A20000003
:1017E0002053000045740000204600004C540000C7
:1017F0005F4D000041580000562000003C7600007C
:101800003E20000020200000202000002D200000AD
:10181000666C00006F6100007420000063680000C7
:101820006172000067650000206D000061780000B3
:10183000207600006F6C0000746100006765000096
:101840000D0A000020200000534500007420000015
:10185000464C0000545F00004D410000584300001A
:10186000203C0000613E00002020000020200000FD
:10187000202D0000206600006C6F000061740000E5
:1018800020630000686100007267000065200000AE
:101890006D61000078200000637500007272000026
:1018A000656E0000740D00000A2000002053000047
:1018B00045740000204600004C5400005F540000B6
:1018C000455200004D540000203C0000743E0000D2
:1018D00020200000202000002D200000666C000069
:1018E0006F610000742000006368000061720000F6
:1018F00067650000206D0000617800002063000033
:1019000068610000726700006520000074690000D3
:101910006D6500000D0A000000200000205300004B
:1019200045740000205000004D4100005020000090
:101930003C700000733E0000203C00006964000021
:101940003E200000202000002D2000006D610000DE
:101950007020000070730000656C0000656300007B
:1019600074200000746F000020700000726F00008F
:10197000666900006C6500000D0A00000020000090
:10198000204500004449000054200000505200004F
:101990004F460000494C0000452000003C6E00000E
:1019A0003E20000020200000202000002D2000000C
:1019B000636800006F6F0000736500002070000016
:1019C000726F0000666900006C6500002074000002
:1019D0006F20000065640000697400003B20000077
:1019E0003C690000643E0000203A00003D200000F9
:1019F0005B3100007C3200007C3300007C3400004E
:101A00007C4F000046460000424F0000415200005B
:101A1000445D00000D0A000000200000204400008A
:101A2000454C000045540000452000005052000085
:101A30004F460000494C0000452000003C6E00006D
:101A40003E200000202000002D20000063680000E0
:101A50006F6F00007365000020700000726F00005F
:101A6000666900006C650000207400006F200000B3
:101A7000646500006C650000746500003B20000098
:101A80003C690000643E0000203A00003D20000058
:101A90005B3200007C3300007C3400005D0D0000F0
:101AA0000A00000020200000454E00006162000096
:101AB0006C650000205A00004556000043430000BA
:101AC000532000003C630000696600003E200000D7
:101AD000202D0000205A000045560000434300001E
:101AE0005320000063680000617200006769000015
:101AF0006E6700000D0A000020200000454E000027
:101B0000616200006C650000204300004841000055
:101B100052470000454D00004F2000003C6300008C
:101B2000696600003E2D000020430000484100008F
:101B300052470000454D00004F2000006368000040
:101B400061720000676900006E6700000D0A000006
:101B500020200000454E0000616200006C6500001E
:101B6000204F00004243000048410000524700005F
:101B7000452000003C630000696600003E2D000027
:101B8000206F00006E6200006F6100007264000050
:101B9000206300006861000072670000696E000049
:101BA000670D00000A200000204500004E61000083
:101BB000626C000065200000544F0000504200009D
:101BC000414C0000414E0000434500002020000031
:101BD000202000002D20000073650000652000001B
:101BE000646F0000637500006D6500006E74000096
:101BF00061740000696F00006E0D00000A20000093
:101C0000204500004E610000626C0000652000006D
:101C1000534C00004F570000535400004152000045
:101C20005420000020200000202000002D20000073
:101C30007365000065200000646F0000637500009C
:101C40006D6500006E74000061740000696F000033
:101C50006E0D00000A000000202000004449000032
:101C600053610000626C0000652000005A450000CE
:101C700056430000435300002020000020200000B5
:101C800020200000202D0000205A000045560000B2
:101C900043430000532000006368000061720000AD
:101CA000676900006E6700000D0A00002020000038
:101CB0004449000053610000626C00006520000090
:101CC0004348000041520000474500004D4F0000CE
:101CD0002020000020200000202D000020430000D4
:101CE0004841000052470000454D00004F200000D1
:101CF0006368000061720000676900006E670000A1
:101D00000D0A00002020000044490000536100003B
:101D1000626C000065200000544F0000504200003B
:101D2000414C0000414E00004345000020200000CF
:101D3000202D000020730000656500002064000075
:101D40006F630000756D0000656E00007461000037
:101D5000746900006F6E00000D0A00002020000072
:101D60004449000053610000626C000065200000DF
:101D7000534C00004F5700005354000041520000E4
:101D80005420000020200000202D000020730000BF
:101D900065650000206400006F630000756D000041
:101DA000656E000074610000746900006F6E0000D1
:101DB0000D0A000000200000202D00002D6F000003
:101DC00070740000696F00006E7300002D2D00001C
:101DD0000D0A0000002D00002D6500007663000054
:101DE000632D00002D2D00002D2D00002D2D000055
:101DF0002D2D00002D2D00002D2D00002D2D00007B
:101E00002D2D00002D2D00002D2D00002D2D00006A
:101E10002D2D00002D2D00002D2D00002D2D00005A
:101E20002D2D00002D2D00002D0D00000A2000009A
:101E300020530000486F00007720000020200000A1
:101E40002020000020200000202000002020000092
:101E50002020000020200000202000002D20000075
:101E60006368000061720000676500002073000075
:101E70007461000074750000730D00000A200000FA
:101E800020530000486F000077200000434F0000FF
:101E90004E6600006967000020200000202000003E
:101EA0002020000020200000202000002D20000025
:101EB0006368000061720000676500002063000035
:101EC0006F6E0000666900006775000072610000B7
:101ED000746900006F6E00000D0A00000020000011
:101EE000205200004573000065740000204300008C
:101EF0004F4E0000666900006720000020200000AF
:101F00002020000020200000202000002D200000C4
:101F100072650000736500007420000045560000E3
:101F200043430000206300006F6E000066690000FC
:101F30006775000072610000746900006F6E000038
:101F40000D0A0000002D00002D6300006F6E0000E0
:101F50006669000067750000726100007469000026
:101F60006F6E00002D2D00002D2D00002D2D000086
:101F70002D2D00002D2D00002D2D00002D2D0000F9
:101F80002D2D00002D2D00002D2D00002D2D0000E9
:101F90002D2D00002D2D00002D0D00000A00000049
:101FA000202000002D2D000020620000756C000034
:101FB0006B2000006368000061720000676500002C
:101FC0002070000061720000616D00006574000007
:101FD00065720000732D00002D0D00000A00000046
:101FE000202000002D2D00006C65000061640000C1
:101FF0002061000063690000642000006368000045
:1020000061720000676500002070000061720000CE
:10201000616D00006574000065720000732D0000A2
:102020002D0D00000A000000202000002D2D0000D2
:10203000707200006F660000696C0000657300003C
:102040002D2D00000D0A000000200000204400009B
:1020500049530000616200006C650000203C0000F4
:102060006F700000746900006F6E00003E20000079
:1020700020200000202000002D20000064690000C6
:1020800073610000626C000065200000616E00005A
:10209000206F000070740000696F00006E0D00007A
:1020A0000A0000002D2D0000646900006167000037
:1020B0006E6F00007374000069630000732D0000F0
:1020C0002D2D00002D2D00002D2D00002D2D0000A8
:1020D0002D2D00002D2D00002D2D00002D2D000098
:1020E0002D2D00002D2D00002D2D00002D2D000088
:1020F0002D2D00002D2D00000D0A000000200000F5
:1021000020530000486F000077200000484900007D
:10211000537400006F72000079200000202000003E
:102120002020000020200000202000002D200000A2
:1021300063680000617200006765000020680000AD
:1021400069730000746F0000727900000D0A0000CE
:10215000202000005245000073650000742000003C
:1021600048490000537400006F720000792000009D
:10217000202000002020000020200000202D000052
:102180002072000065730000657400002063000089
:102190006861000072670000652000006869000047
:1021A000737400006F720000790D00000A000000D7
:1021B00020200000545200006163000065200000F0
:1021C0004348000061720000676500007220000053
:1021D000202000002020000020200000202D0000F2
:1021E000206500006E610000626C00006520000048
:1021F0006F6E0000626F00006172000064200000DA
:1022000063680000617200006765000072200000D2
:102210007472000061630000696E0000670D0000C9
:102220000A000000202000005452000061630000FA
:10223000652000004348000041520000474500006F
:102240004D4F000020200000202000002020000032
:10225000202D0000206500006E610000626C00000F
:10226000652000004348000041520000474500003F
:102270004D4F000020730000746100007465000081
:102280002074000072610000636900006E67000046
:102290000D0A0000002000002054000052610000E0
:1022A00063650000205300005441000054450000C5
:1022B000202000002020000020200000202000001E
:1022C000202000002D200000656E000061620000EB
:1022D0006C650000206F00006E6200006F610000FE
:1022E00072640000206300006861000072670000F3
:1022F00065720000207300007461000074650000C6
:102300002074000072610000636900006E670000C5
:102310000D0A0000202000005452000061630000FC
:10232000652D0000203C0000743E000020200000CD
:10233000202000002020000020200000202000009D
:10234000202D00002064000069730000616200001D
:102350006C6500007320000074720000616300006F
:10236000650D00000A2000002054000052610000AA
:1023700063650000204F000046460000202000005A
:10238000202000002020000020200000202000004D
:10239000202000002D20000064690000736100000F
:1023A000626C000065730000206100006C6C00002E
:1023B0002074000072610000636900006E67000015
:1023C0000D0A000000200000202000002020000056
:1023D000202000002020000020200000203A0000E3
:1023E000200000002D2D00006F66000066620000D6
:1023F0006F610000726400002063000068610000EB
:1024000072670000696E0000672000002865000008
:1024100064690000742900002D2D00002D2D00009E
:102420002D2D00002D2D00002D2D00002D2D000044
:102430002D2D00002D2D00000D0A0000002D0000A4
:102440002D6F000066660000626F00006172000080
:10245000642000006368000061720000676900008A
:102460006E6700002D2D00002D2D00002D2D000089
:102470002D2D00002D2D00002D2D00002D2D0000F4
:102480002D2D00002D2D00002D2D00002D2D0000E4
:102490002D0D00000A0000002020000070720000D6
:1024A0006F7400006F6300006F6C0000202000005C
:1024B0003A200000006300006861000072670000BD
:1024C000656D00006F0D00000A0000002020000074
:1024D00020200000637300006571000031200000BF
:1024E000202000003A200000006E00006F74000001
:1024F000206D000061700000706500006400000045
:10250000202000002020000063730000657100009F
:1025100032200000202000003A20000000200000AF
:10252000202000002063000070650000726D000034
:1025300020200000203A00002000000020200000A1
:1025400020200000636300006F6E00007420000014
:10255000202000003A200000007A0000657600008C
:1025600063630000730D00000A0000006D6100004D
:1025700078760000202000002020000020000000CD
:102580006D61000078630000202000002020000022
:102590002000000074650000726D000074200000CF
:1025A000202000002000000074650000726D000013
:1025B0006320000020200000200000002D2D0000DE
:1025C0006F6E0000626F0000617200006420000006
:1025D0006368000061720000676900006E670000B8
:1025E000202800006564000069740000292D0000A7
:1025F0002D2D00002D2D00002D2D00002D2D000073
:102600002D2D00002D2D00002D2D00002D2D000062
:102610000D0A0000002D00002D6F00006E6200000A
:102620006F610000726400002063000068610000B8
:1026300072670000696E0000672D00002D2D0000FC
:102640002D2D00002D2D00002D2D00002D2D000022
:102650002D2D00002D2D00002D2D00002D2D000012
:102660002D2D00002D2D00002D0D00000A00000072
:102670002D2D000063680000617200006769000092
:102680006E6700002D2D00002D2D00002D2D000067
:102690002D2D00002D2D00002D2D00002D2D0000D2
:1026A0002D2D00002D2D00002D2D00002D2D0000C2
:1026B0002D2D00002D2D00002D2D00002D2D0000B2
:1026C0002D2D00000D0A00000020000020700000E9
:1026D0006C75000067200000202000002020000012
:1026E000203A0000200000004A3100003737000087
:1026F000320D00000A0000004A31000037370000A8
:1027000032540000320D00000A000000646900002D
:1027100072650000637400000D0A0000003F0000B5
:102720003F0D00000A00000020200000706C000037
:1027300075670000696E0000202000002020000066
:102740003A20000000200000206F0000707400009C
:10275000696F00006E73000020200000203A000026
:1027600020000000746F000070620000616C0000C7
:10277000616E0000636500000D0A00000073000038
:102780006C6F0000777300007461000072740000C9
:102790000D0A00000020000020700000726F000091
:1027A000666900006C65000020200000203A0000EF
:1027B0002020000000200000202000002000000059
:1027C000202800002A2900002020000020200000EE
:1027D0002020000020000000202000002020000019
:1027E0002020000020200000202000002000000009
:1027F00063680000617200006765000072200000DD
:10280000200000006368000061720000676500003E
:102810007232000020000000636800006172000056
:10282000676500007233000020000000636800004C
:102830006172000067650000723400002000000033
:102840006C6900006E65000076200000202000000A
:10285000200000006C6900006E650000632000002D
:102860002020000020000000657600007365000055
:1028700077610000697400002000000066690000B4
:102880006E5F00006D61000078760000200000009F
:10289000666900006E5F00006D61000078630000F3
:1028A00020000000666900006E5F00007465000093
:1028B000726D000074000000666C0000745F000020
:1028C0006D6100007876000020000000666C00005A
:1028D000745F00006D61000078630000200000005C
:1028E000666C0000745F000074650000726D00008B
:1028F0007400000020200000706D00006170000076
:102900002020000020200000202000003A0D0000C0
:102910000A0000002020000020200000696E000056
:102920006620000020200000202000003A00000067
:10293000780D00000A000000202000002020000088
:10294000323000004B20000020200000202000003A
:102950003A0000002020000020200000354B00003D
:102960002020000020200000202000003A0000006D
:102970002020000020200000302000002020000047
:1029800020200000202000003A00000070720000AB
:102990006F660000696C0000650000006572000051
:1029A000726F0000723A0000206F00006E6C000031
:1029B000792000006F6E0000652000006F66000047
:1029C0002043000048410000444500004D4F0000F6
:1029D000206F0000722000005A450000564300009E
:1029E00043530000206D0000617900002062000068
:1029F00065200000656E0000616200006C650000EB
:102A0000640D00000A0000006D610000707000009D
:102A1000696E000067200000494E0000332000006E
:102A2000746F000020430000534500005131000046
:102A30000D0A000000430000534500005131000022
:102A4000206E00006F740000206D000061700000B7
:102A500070650000642C0000204900004E33000027
:102A6000206100006C720000656100006479000064
:102A70002061000073730000696700006E6500004C
:102A8000640D00000A0000006D610000707000001D
:102A9000696E000067200000494E000034200000ED
:102AA000746F0000204300005345000051320000C5
:102AB0000D0A0000004300005345000051320000A1
:102AC000206E00006F740000206D00006170000037
:102AD00070650000642C0000204900004E330000A7
:102AE000206100006C7200006561000064790000E4
:102AF0002061000073730000696700006E650000CC
:102B0000640D00000A0000006D610000707000009C
:102B1000696E0000672000004F550000543200002D
:102B2000207400006F200000435000004552000058
:102B30004D0D00000A000000435000004552000007
:102B40004D2000006E6F0000742000006D610000D9
:102B500070700000656400002C2000004F550000DC
:102B600054320000206100006C72000065610000BA
:102B70006479000020610000737300006967000041
:102B80006E650000640D00000A0000006D61000029
:102B900070700000696E0000672000004F55000053
:102BA00054330000207400006F20000043430000F5
:102BB0004F4E0000540D00000A0000004343000087
:102BC0004F4E0000542000006E6F00007420000083
:102BD0006D61000070700000656400002C20000032
:102BE0004F55000054330000206100006C7200005B
:102BF00065610000647900002061000073730000CB
:102C0000696700006E650000640D00000A000000A6
:102C10006D61000070700000696E000067200000A8
:102C2000504C000055470000207400006F20000049
:102C30005A45000056430000435300000D0A0000AF
:102C4000006D000061700000706900006E67000098
:102C5000204900004E330000207400006F20000067
:102C6000504C000055470000494E00000D0A00007E
:102C7000005000004C550000474900004E20000065
:102C80006E6F0000742000006D6100007070000025
:102C9000656400002C200000494E00003320000035
:102CA000616C000072650000616400007920000022
:102CB0006173000073690000676E000065640000C6
:102CC0000D0A0000006D00006170000070690000D6
:102CD0006E670000205000004C55000047200000A7
:102CE000746F0000204A00003137000037320000C6
:102CF0000D0A000000640000656C000065740000AF
:102D0000696E0000672000006D6100007020000007
:102D1000746F0000205000004C550000474900002F
:102D20004E0D00000A000000646500006C650000A4
:102D3000746900006E670000206D00006170000083
:102D4000207400006F200000435300004551000034
:102D5000310D00000A000000646500006C65000091
:102D6000746900006E670000206D00006170000053
:102D7000207400006F200000435300004551000004
:102D8000320D00000A000000646500006C65000060
:102D9000746900006E670000206D00006170000023
:102DA000207400006F2000004350000045520000D6
:102DB0004D0D00000A000000646500006C65000015
:102DC000746900006E670000206D000061700000F3
:102DD000207400006F200000434300004F4E0000AD
:102DE000540D00000A000000317C0000327C00001D
:102DF000337C0000347C00004F4E0000424F000046
:102E000041520000447C00004F4600004642000052
:102E10004F4100005244000000730000796E000032
:102E200074610000783A000020270000454400004B
:102E30004954000020500000524F00004649000055
:102E40004C450000203C00006E3E0000273B000087
:102E5000202000003C6E00003E2000003A3D0000B3
:102E6000205B0000317C0000327C0000337C0000DD
:102E7000347C00004F460000464200004F410000F5
:102E8000524400005D0D00000A000000737900004C
:102E90006E740000617800003A20000027440000B2
:102EA000454C0000455400004520000050520000F1
:102EB0004F460000494C0000452000003C6E0000D9
:102EC0003E2700003B200000203C00006E3E00003A
:102ED000203A00003D2000005B3200007C330000FF
:102EE0007C3400005D0D00000A00000065720000E7
:102EF000726F0000723A0000206E00006F20000028
:102F00004F460000464200004F410000524400007E
:102F100020630000686100007267000065720000B5
:102F2000206F000070740000696F00006E73000075
:102F30002061000072650000206500006E610000E5
:102F4000626C0000656400000D0A0000006500006E
:102F5000727200006F7200003A200000636100008E
:102F60006E6E00006F740000206400006973000042
:102F7000616200006C650000207400006869000058
:102F800073200000707200006F660000696C000022
:102F9000650D00000A000000747300006D3200002F
:102FA00035300000307C0000747300006D3200008A
:102FB00035300000305F0000343100007C740000C8
:102FC000736D000032350000303000005F340000C7
:102FD000327C0000747300006D3200003530000058
:102FE000305F0000343300007C6500006C6300003B
:102FF0006F6E00007C6500006C6300006F6E000067
:103000005F650000377C0000656C0000636F0000A6
:103010006E5F0000653800007C6500006C63000096
:103020006F6E00005F650000397C00007374000063
:10303000656100006C740000687C00006C65000035
:10304000617200007C6E00006C670000357C00003F
:10305000766F00006C7400007C62000061730000F9
:10306000696300007C6E00006F6E00006500000068
:10307000737900006E740000617800003A2000004F
:103080002773000065740000203C000063680000A6
:103090006172000067650000723E0000203C000085
:1030A0006D6F0000646500006C3E00005B3C00003A
:1030B0007068000061730000653E00005D2700003D
:1030C0000D0A000020200000202000002020000029
:1030D000202000002020000020200000203C0000D4
:1030E000636800006172000067650000723E0000C6
:1030F000203A00003D2000005B43000048410000F2
:1031000052470000455200007C4300004841000047
:103110005247000045520000327C00004348000046
:103120004152000047450000523300007C4300003C
:10313000484100005247000045520000345D000045
:103140000D0A0000002000002020000020200000C8
:10315000202000002020000020200000202000006F
:10316000202000003C6D00006F640000656C0000D2
:103170003E2000003A3D0000205B00005453000058
:103180004D32000035300000307C00005453000008
:103190004D32000035300000305F00003431000057
:1031A0007C540000534D00003235000030300000E8
:1031B0005F340000327C0000545300004D320000A8
:1031C00035300000305F0000343300000D0A00008D
:1031D00020200000202000002020000020200000EF
:1031E00020200000202000002020000020200000DF
:1031F00020200000202000002020000020200000CF
:10320000202000007C4500004C4300004F4E000091
:103210007C4500004C4300004F4E00005F4500001D
:10322000377C0000454C0000434F00004E5F00001B
:10323000453800007C4500004C4300004F4E000024
:103240005F450000390D00000A200000202000002A
:10325000202000002020000020200000202000006E
:10326000202000002020000020200000202000005E
:10327000202000002020000020200000207C0000F2
:1032800053540000454100004C540000487C0000AD
:103290004C450000415200007C4E00004C470000AD
:1032A000357C0000564F00004C5400007C4200006A
:1032B00041530000494300000D0A00002020000097
:1032C00020200000202000002020000020200000FE
:1032D00020200000202000002020000020200000EE
:1032E00020200000202000002020000020200000DE
:1032F0007C4E00004F4E0000455D00000D0A0000AE
:1033000000200000202000002020000020200000DD
:1033100020200000202000002020000020200000AD
:103320003C70000068610000736500003E200000F2
:103330003A3D0000205B00004E4F00004E4500006B
:103340007C4C0000317C00004C3200007C4C0000C2
:10335000335D00000D0A0000002000002020000066
:1033600020200000202000002027000073650000BE
:10337000742000003C630000686100007267000078
:10338000657200003E2000004E4F00004E450000D8
:1033900027200000746F000020640000656C0000AE
:1033A0006574000065200000612000006368000073
:1033B0006172000067650000720D00000A000000E5
:1033C0006E6F00006E6500007C4C0000317C0000D8
:1033D000317C00004C3200007C3200007C4C00004C
:1033E000337C0000337C0000707200006F670000C7
:1033F000726100006D00000065720000726F0000D5
:10340000723A000020630000616E0000206F00002F
:103410006E6C000079200000707200006F67000081
:10342000726100006D200000747300006D320000B6
:103430003530000030200000636800006172000039
:1034400067650000727300000D0A0000006500004F
:10345000727200006F7200003A2000006361000089
:103460006E6E00006F74000020640000656C000048
:10347000657400006520000074680000652000008D
:103480006669000072730000742000006368000029
:103490006172000067650000720D00000A00000004
:1034A00065720000726F0000723A00002064000034
:1034B000757000006C6900006361000074650000B5
:1034C0002063000068610000726700006572000000
:1034D0002074000079700000650D00000A000000F3
:1034E00065720000726F0000723A000020620000F6
:1034F000616400002070000061720000616D0000D6
:10350000657400006572000020280000276D00002F
:103510006F640000656C0000272900000D0A0000A0
:10352000006A000031370000373200007C6A00007A
:103530003137000037320000743200007C64000034
:103540006972000065630000740000007379000078
:103550006E740000617800003A20000027730000BC
:1035600065740000207000006C750000672000008A
:103570005B4A000031370000373200007C4A00000F
:103580003137000037320000543200007C44000024
:103590004952000045430000545D0000270D000023
:1035A0000A00000065720000726F0000723A0000AD
:1035B0002062000061640000207000006172000061
:1035C000616D000065740000657200000D0A000066
:1035D000006900006E6600007C320000304B000085
:1035E0007C3500004B7C0000307C0000616C0000EA
:1035F0006C000000737900006E74000061780000B8
:103600003A200000275300004574000020500000BD
:103610004D410000502000003C700000733E00004F
:10362000203C0000696400003E2700003B200000B1
:10363000203C0000707300003E2000003A3D000076
:10364000205B0000696E0000667C000032300000E4
:103650004B7D0000354B00007C3000007C61000099
:103660006C6C00005D0D00000A20000020200000AE
:10367000202000002020000020200000202000004A
:10368000202000002020000020200000202000003A
:10369000202000002020000020200000202000002A
:1036A00020200000202000003C690000643E000053
:1036B000203A00003D2000005B3100007C32000019
:1036C0007C3300007C3400005D0D00000A00000027
:1036D00065720000726F0000723A000020700000F6
:1036E000726F0000666900006C6500002000000039
:1036F00020690000732000006E6F0000742000003D
:1037000064650000666900006E650000640D0000DD
:103710000A0000000A000000737900006E740000C7
:10372000617800003A2000002773000065740000F3
:10373000206C0000696E000065760000203C0000EF
:10374000763E0000273B0000203C0000763E000053
:10375000206900006E200000766F00006C7400008D
:103760007320000028300000207400006F2000004B
:103770006469000073610000626C0000652900004C
:103780000D0A0000006C0000696E00006576000004
:1037900000730000796E000074610000783A000048
:1037A0002027000073650000742000006C69000091
:1037B0006E650000632000003C6100003E270000B1
:1037C0003B2000003C6100003E200000696E0000CC
:1037D000206100006D7000007320000028300000A0
:1037E000207400006F200000646900007361000015
:1037F000626C0000652900000D0A0000006C0000EA
:10380000696E00006563000000730000796E0000BF
:1038100074610000783A0000202700007365000002
:10382000742000006D61000078760000203C0000EC
:10383000763E0000273B0000203C0000763E000062
:10384000206900006E200000766F00006C7400009C
:10385000730D00000A00000065720000726F000026
:10386000723A000020630000616E00006E6F00007D
:1038700074200000646500006C6500007465000041
:1038800020700000726F0000666900006C65000027
:10389000203100000D0A0000006D0000617800007A
:1038A00076000000737900006E74000061780000FB
:1038B0003A2000002773000065740000206D0000AE
:1038C00061780000632000003C6100003E2700009A
:1038D0003B2000003C6100003E200000696E0000BB
:1038E000206100006D700000730D00000A000000F0
:1038F0006D6100007863000000730000796E0000C5
:1039000074610000783A0000202700007365000011
:103910007420000074650000726D000063200000D8
:103920003C6100003E2700003B2000003C6100009D
:103930003E200000696E0000206100006D700000F4
:10394000730D00000A00000074650000726D000035
:1039500063000000696E0000667C0000646A00007D
:103960006D000000737900006E7400006178000043
:103970003A200000277300006574000020740000E6
:10398000657200006D740000203C0000743E000071
:10399000273B0000203C0000743E0000206900002E
:1039A0006E2000006D6900006E75000074650000F7
:1039B000730D00000A2000002020000020200000DD
:1039C0002020000020270000736500007420000004
:1039D00074650000726D000074200000696E0000C4
:1039E000662700003B2000006E6F0000206C000086
:1039F000696D0000697400000D0A00000074000089
:103A0000657200006D74000000730000796E0000A4
:103A100074610000783A0000202700007365000000
:103A200074200000666900006E5F00006D61000098
:103A300078760000203C0000763E0000273B000026
:103A4000203C0000763E0000206900006E2000004F
:103A5000766F00006C7400007320000028300000B6
:103A6000207400006F200000646900007361000092
:103A7000626C0000652900000D0A0000006600006D
:103A8000696E00005F6D0000617800007600000044
:103A9000737900006E740000617800003A20000025
:103AA000277300006574000020660000696E000046
:103AB0005F6D000061780000632000003C61000041
:103AC0003E2700003B2000003C6100003E2000003B
:103AD000696E0000206100006D700000730D000031
:103AE0000A000000666900006E5F00006D61000062
:103AF0007863000000730000796E000074610000BC
:103B0000783A000020270000736500007420000050
:103B1000666900006E5F000074650000726D000051
:103B2000742000003C7400003E2700003B20000091
:103B30003C7400003E200000696E0000206D000013
:103B4000696E000075740000657300000D0A0000C6
:103B500000730000796E000074610000783A000084
:103B6000202700007365000074200000666C0000D0
:103B7000745F00006D61000078760000203C00005A
:103B8000763E0000273B0000203C0000763E00000F
:103B9000206900006E200000766F00006C74000049
:103BA0007320000028300000207400006F20000007
:103BB0006469000073610000626C00006529000008
:103BC0000D0A0000006600006C7400005F6D0000CC
:103BD0006178000076000000737900006E740000C8
:103BE000617800003A20000027730000657400002F
:103BF000206600006C7400005F6D000061780000BA
:103C0000632000003C6100003E2700003B200000D4
:103C10003C6100003E200000696E00002061000051
:103C20006D700000730D00000A000000666C00005B
:103C3000745F00006D61000078630000006900009F
:103C40006E66000000730000796E00007461000071
:103C5000783A0000202700007365000074200000FF
:103C6000666C0000745F000074650000726D0000F7
:103C7000742000003C7400003E2700003B20000040
:103C80003C7400003E200000696E0000206D0000C2
:103C9000696E000075740000657300000D0A000075
:103CA0002020000020200000202000002020000014
:103CB0002773000065740000206600006C7400002B
:103CC0005F740000657200006D74000020690000E0
:103CD0006E660000273B0000207300007461000046
:103CE00079200000696E000020270000666C00004B
:103CF0006F61000074270000206900006E640000FE
:103D000065660000696E000069740000656C000063
:103D1000790D00000A000000737900006E74000045
:103D2000617800003A2000002773000065740000ED
:103D3000206500007673000065770000616900006F
:103D4000742000003C6D00003E2700003B20000076
:103D50003C6D00003E200000696E0000206D0000F8
:103D6000696E000075740000657300000D0A0000A4
:103D7000006500007673000065770000616900004F
:103D800074000000202000006368000061720000E1
:103D90006765000072000000202000003A2000004B
:103DA000002000002020000020730000746100004B
:103DB0007475000073200000203A0000200000000D
:103DC0000D0A00002020000020200000766F000077
:103DD0006C74000061670000652000003A2000005C
:103DE000005600000D0A0000002000002020000006
:103DF0002063000075720000726500006E740000A0
:103E0000203A000020000000726500006365000099
:103E10006976000065200000746900006D6500008F
:103E20006F750000740D00000A000000206D000096
:103E30007367000073200000736500006E7400005B
:103E40003B200000002000006D730000677300003D
:103E5000207200006563000065690000766500005F
:103E6000640D00000A000000202000002020000057
:103E7000766F00006C740000616700006520000030
:103E80003A200000002000002020000020630000F5
:103E9000686100007267000065200000203A0000A1
:103EA00020000000576800000D0A000000200000FC
:103EB0002020000020200000666C000061670000E8
:103EC00073200000203A0000200000006E6F000008
:103ED0002063000068610000726700006520000038
:103EE00068690000737400006F720000790D0000B3
:103EF0000A000000202000002020000020200000F8
:103F00007C2000002020000074650000726D00001D
:103F100020200000207C00002020000063680000BA
:103F20006172000067650000207C00002020000016
:103F30002020000020200000202000002020000081
:103F40007C200000202000007761000074740000D5
:103F5000207C0000206D000061780000696D000089
:103F6000756D00007C2000006D6100007869000024
:103F70006D7500006D7C000020200000656E000063
:103F8000646900006E6700007C0D00000A000000FC
:103F9000202000006E7500006D2000007C200000D5
:103FA0002072000065610000736F00006E20000049
:103FB000207C00002020000020740000696D0000BB
:103FC00065200000207C00002020000063680000C5
:103FD0006172000067650000722000007C20000014
:103FE000206800006F75000072730000207C0000E4
:103FF000207600006F6C00007461000067650000AF
:104000007C2000006375000072720000656E000085
:10401000747C00002063000075720000726500006F
:104020006E7400007C0D00000A0000002D2D0000C1
:104030002D2D00002D2D00002D2D00002D2D000018
:104040002D2D00002D2D00002D2D00002D2D000008
:104050002D2D00002D2D00002D2D00002D2D0000F8
:104060002D2D00002D2D00002D2D00002D2D0000E8
:104070002D2D00002D2D00002D2D00002D2D0000D8
:104080002D2D00002D2D00002D2D00002D2D0000C8
:104090002D2D00002D2D00002D2D00002D2D0000B8
:1040A0002D2D00002D2D00002D2D00002D2D0000A8
:1040B0002D2D00002D2D00002D2D00002D2D000098
:1040C0000D0A0000002000006C6100007374000005
:1040D000207C000000200000202D000000200000B7
:1040E0007C0000007C000000206D0000696E000074
:1040F000737C000000200000202000002020000031
:1041000020200000202000002020000020200000AF
:10411000202000002020000020200000202000009F
:104120002020000020200000202000007C00000053
:10413000202000002020000020200000202000007F
:10414000202000002020000020200000202000006F
:10415000202000002020000020200000202000005F
:1041600020200000207C0000544F0000544100003B
:104170004C20000020200000202000007C000000D7
:10418000576800007C000000562000007C00000002
:10419000412000007C000000412000007C0D000058
:1041A0000A00000020200000737400006174000009
:1041B0006520000020200000202000003A200000A0
:1041C000002C000020430000430000002C200000D1
:1041D00043560000002C0000204300005400000063
:1041E00020200000706C0000756700002073000044
:1041F00074610000746500003A2000000020000097
